:020000040000FA
:10000000305A001001020000050200000702000043
:10001000090200000B0200000D020000A299FFEF90
:100020000000000000000000000000000F020000BF
:100030001102000000000000130200001502000081
:10004000170200001702000017020000170200004C
:10005000170200001702000017020000170200003C
:10006000170200001702000017020000170200002C
:10007000170200001702000017020000170200001C
:10008000170200001702000017020000170200000C
:1000900017020000170200001702000017020000FC
:1000A0003F230000170200001702000017020000A3
:1000B00017020000170200001702000017020000DC
:1000C00017020000170200001702000000F002F8FB
:1000D00000F05EF80AA090E8000C82448344AAF184
:1000E0000107DA4501D100F053F8AFF2090EBAE882
:1000F0000F0013F0010F18BFFB1A43F0010318475C
:10010000DC370000FC3700000A444FF0000C10F808
:10011000013B13F0070408BF10F8014B1D1108BF85
:1001200010F8015B641E05D010F8016B641E01F825
:10013000016BF9D113F0080F1EBF10F8014BAD1C75
:100140000C1B09D16D1E58BF01F801CBFAD505E093
:1001500014F8016B01F8016B6D1EF9D59142D6D3ED
:10016000704700000023002400250026103A28BF15
:1001700078C1FBD8520728BF30C148BF0B60704719
:100180001FB59DE8030002F0B9FF1FBD10B510BDFB
:1001900003F004F81146FFF7F3FF00F0BBFB03F098
:1001A00022F803B4FFF7F2FF03BC03F053F800009A
:1001B000D0F800D0D0F804F0024600200B21C3078D
:1001C00000D0802303EB500012F8013B491E184475
:1001D00009B2C0B20029F2D17047000006480221DE
:1001E00041600021016741610B22C260C1630121AE
:1001F000416000207047000000800040443322111D
:1002000008480047FEE7FEE7FEE7FEE7FEE7FEE7F9
:10021000FEE7FEE7FEE7FEE703480449044A054B14
:1002200070470000CD000000300A0010305A001066
:10023000304A0010304A001070B5284C607820B366
:100240000026274D012810D002280DD1A86861682A
:10025000401A2449884215D32348406B400011D5E9
:10026000012001F097FF667070BDA8686168401AB0
:100270001E498842F8D3002001F08CFFA868606016
:100280000220607026700C2005E020780028EBD159
:10029000012020700D20BDE8704001F05DB90028FC
:1002A00002D10E4901204870704710B501F01AFEC6
:1002B0000A490020487010BD0848012141700849D2
:1002C00089684160704770477047022803D003284F
:1002D00003D100F0D9BE00F0F4BE7047A4010010B5
:1002E00000800040A086010000C0092040420F00AD
:1002F000704770477047704770477047FFFFFFFFB8
:100300001948062101610721016000214161416214
:1003100002214160C168C906FCD400E08168C1685F
:100320004907FBD4002070470F498860C868C006A1
:10033000FCD48868704700B50B46024604E000BF55
:1003400012F8010BFFF7F0FF5B1EF9D200BD00B5FC
:100350000B46024604E00020FFF7E6FF02F8010B1F
:100360005B1EF8D200BD00000080084070B5064654
:1003700000F036F8056806F10B0020F00704B442DF
:100380009CBF002070BD2B466A68BAB11068A042BD
:1003900010D304F1080188423CBF5068586007D36D
:1003A0005168101941601168091B016058601460A0
:1003B000101D70BD13465268002AE7D12146284619
:1003C00002F088FE0028DED170BD10B591FBF2F47A
:1003D00091FBF2F302FB1411C0E9003110BD0000E3
:1003E00000487047D809001000210160C0E90110E1
:1003F000704710207047000000487047D009001077
:1004000000000000A71B000010B50178427801EB46
:10041000810102EB4101C902A1F5C0318AB2C17864
:100420000479303901EB810104EB41014901A1F567
:10043000C06101F4FC611143C27980796FF02F0330
:10044000303800EB800003EB40001044C0F3440060
:10045000084310BDF0B58DB004463022F949684616
:1004600002F004FEE079A17A00EB4002C2EBC0107A
:1004700001EBC001207A64225043627A102302EB20
:10048000820200EB420008444002742100EB41204C
:100490002179627901EB810103EB4101114480B2C2
:1004A00001F01F010143237800206D4655F82020FC
:1004B0001678B3420DD166785778BE4209D1A67836
:1004C0009278964205D14001203000F4F07001434B
:1004D00003E0401CC0B20C28E8D30DB00846F0BDC4
:1004E000D94910B5486D00050CD4D84A906843F638
:1004F00098239468241A9C42FBD3486D000501D4CC
:10050000012010BD052001F027F8002010BD70B5B6
:10051000CE4CA668042001F01FF8CD4D03E000BFCB
:10052000FFF7DEFF48B1A068801BA842F8D308E0BF
:10053000FFF7D6FF08B1012070BDA068801BA8425C
:10054000F6D3002070BD10B5092001F005F8C149AF
:100550000120487010BD2DE9F041002506462C46CB
:10056000BD4F0BE040222146BB4800F0ECFE0020CE
:100570003958001D0D444028FAD34034B442F1D319
:100580002846BDE8F081B5A086B00FC88DE80F0001
:10059000B6A0B74900680490086800264FF6FF022D
:1005A0001040B44A40F4807010430860B249B34F21
:1005B0004FF4C8200E60B3493860B1480860B249B2
:1005C0004012B24D0860F8202870FF206870A870B3
:1005D000AF48B046D0F8109001F0EAF89D4CDFF833
:1005E000B4A24FF0010B606801280FD14FF4C8206E
:1005F000FFF7B1FFE0B3D4F8042020204346514672
:1006000051F822703B54401C4028F9D36268002006
:100610005AF822102A180B5C401C82F8003460281B
:10062000F8D301F091FD012001F0B4FD4FF4E17A1F
:100630005546514640F2491001F01FF9294640F253
:100640009F1001F01AF9A046FFF7F6FD98F8010097
:1006500045460028F8D100218FA000F07EFD04005F
:10066000F2D08E49087A66287DD046287BD0DCE01F
:10067000FFE784F800B003223B680221104601EB3B
:10068000932740F6FF7E13E0B0EB932F01D3714622
:1006900000E0411CC0F3032C4CEA0118A85405EB00
:1006A000020C09098CF80180801C8CF80210D21C05
:1006B0008742E9D8402240F20441674800F043FEF7
:1006C00065498878032802D3584681F802B0C0B241
:1006D00004AA5746125C60685AF8203083F8432019
:1006E0005AF8203083F827204B786A4602EB131320
:1006F0005AF820C01B788CF844305AF820C08CF887
:1007000029304B7857F820C003F00F031DF8033051
:100710008CF8453057F820C08CF82E300B7857F8FD
:1007200020C002EB13131B788CF8463057F820C01A
:100730008CF83030097801F00F01515C57F8202017
:1007400082F8471057F8202082F8321057F820001E
:100750004030FFF731FD616857F8211081F82D0016
:100760003D480C3000E01CE0FFF774FE616857F86C
:100770002120A2F8580057F82120A2F8520057F87B
:100780002110A1F8500034481C30FFF73DFE61688D
:1007900057F82120A2F8560057F82110A1F84E0072
:1007A00034E7487A722801D052283ED1887A6D28E1
:1007B00006D04D2804D0782801D0582835D10126FC
:1007C00036480078662801D046282ED140221101F3
:1007D000214800F0B8FD012E03D140211E4800F051
:1007E000BDFD1D492D484F7A001D091D00F05BFD20
:1007F000D8B16868A84628B14FF4C820FFF7ABFE0F
:10080000F8B112E03846254900F024FD50B11248F5
:100810002249807900F02CFD20B14FF4C820FFF769
:100820009AFE28B1092000F097FEFFF78CFE0BE737
:100830000A2000F091FE00273D46072000F08CFEC4
:100840003EE056E0A836000000C0092000800040CD
:1008500080841E00C8000010B00700103031323311
:100860003435363738394142434445464B4E4600CD
:100870000CED00E00000FA0510010010000100106E
:10088000005C0600F8000010FC000010B001001031
:10089000D8360000C0000010463131005C0800105E
:1008A000A8050DD1204600F032FC0446A0F570608A
:1008B000FF381ED0032C1CD340F6F870844218D2A7
:1008C000402229464F4800F03EFD4035012E03D11D
:1008D00040214C4800F042FD09EB07004022494905
:1008E00000F0B2FD0720403700F036FE002DE7D0C3
:1008F000D6E70B2000F030FE5446514640F29F10E0
:1009000000F0BBFF214640F2491000F0B6FF88F826
:1009100001B099E600F09EFE00F0DEFFFFF75EFCFE
:1009200000F0E0FD002000F017FEFFF7E9FC36487C
:10093000C16821F44021C160C16C21F4402141F41F
:100940000021C164314D4FF00070A863286A40F067
:1009500000702862FFF7C4FD2D4E2E4CDFF8B880E2
:10096000002768B3042000F0F7FD686D000514D47B
:10097000FFF7CDFD20B3FFF7CAFD08B3FFF7C7FDB2
:10098000F0B1042000F0E8FDA06841466A6D120550
:1009900003D4A268121A8A42F8D3A06842F21071F6
:1009A000A268121A8A42FBD36869400314D401205A
:1009B000706000F09AFC4FF4C820FFF7CCFD58B1EE
:1009C00000F076FD00284FF002000AD000F0C4FDD0
:1009D0007068401C02D00AE07760F1E700F062FD29
:1009E00005E000F0B9FD7068401C00D1776000F0B0
:1009F0007CFCA0684146A268121A8A42FBD3FFF72A
:100A0000C2FD0000B007001000C0024000C0092075
:100A1000C80000100080004080841E002DE9F843CB
:100A200000250E460446FE4FA84634E0B4F5007F8C
:100A300019D2132C0DD0142C0ED0B4F5FF7F0ED08C
:100A4000A4F58070FF380CD03E2C1CD8F548005D12
:100A500012E097F820000FE0388C000A0CE05520D7
:100A60000AE0AA2008E0B4F5006F08D2EE4820445E
:100A7000A0F5805090F8000E8DF8000005E0EB48DE
:100A8000006801280BD08DF80080E9499DF800002E
:100A9000641C48556D1CB542C8D3BDE8F8830122DB
:100AA000A4F50061684600F04EFCEEE770B5DC4D41
:100AB0002C6B402C00D94024E86AE96902198A426B
:100AC00002D90C1A042169702146FFF7A7FF2246BC
:100AD000D749822001F009FCE86A2044E862286BCB
:100AE000011BD348296300F19F008268A2EB040236
:100AF000826005D06978022901D00021017370BDA0
:100B000003216970F9E7CA4910B59F31C9480860E7
:100B10000D22822001F0E9FBC1490520487010BD7B
:100B200070B50D46C449496D490521D4B0F5007F23
:100B30001ED3C24BBA4CB0F5006F1AD29968A269A5
:100B4000891ABF4A914204D39968A161002161606A
:100B50006161B74A00214032B34B07E044181C449E
:100B6000565CA4F58054491C84F8006EA942F5D364
:100B700070BD616921B99968A16199686161A060DE
:100B8000AA49096829B10129F2D1AE490978002999
:100B9000EED199686269891AAB4A914217D2996875
:100BA000A16199686161A168401A6168884203D9AE
:100BB000616A884200D26060062000F0CDFC2A46BF
:100BC0006168BDE870409A48403000F0AABBBDE8BB
:100BD00070400C2000F0C0BC10B5914CA178E06AC8
:100BE0004218E1698A4206D9081AA070052060708F
:100BF000022001F035FBA178E06AFFF791FFA178B0
:100C0000E06A0844E062206B421A8948226300F1DE
:100C10009F008368A3EB0101816002D06178052900
:100C200004D100210173BDE810406CE710BD2DE92F
:100C3000F0417B4CA178E06A4218E1698A4206D90A
:100C4000081AA07005206070022001F009FB784BA3
:100C50000021A07803F14005E26A08E056186F5CB5
:100C60009E5DBE4202D00021A16202E0491C814289
:100C7000F4D31118E162216B0A1A6D49226301F164
:100C80009F018B68A3EB0000886002D06078052884
:100C900008D1A06A20B100200873BDE8F04132E716
:100CA0000120F9E7BDE8F081614810B58030D0F847
:100CB0001110027D09BA21F0FF011143584A49027F
:100CC000D162C18A49BA49021163806888420DD055
:100CD000822001F0C5FA022001F0C2FA5449022034
:100CE0009F310873FFF70FFF002010BD012010BDDA
:100CF00070B54F4880300224816800F11F0529B18A
:100D0000007B000607D4022001F0AAFA2C73FFF73B
:100D1000FAFE002070BD012070BD10B54448404C63
:100D200080308068A178884200D2A0704049A278C3
:100D30004031822001F0D9FA032060703C48A2784B
:100D40009F308168891A81600021017310BD384885
:100D500010B58030816839B1007B000601D5822052
:100D600000E0022001F07CFA314900209F31087335
:100D7000BDE81040C7E610B5FFF7BAFF00281FD046
:100D80002B48702140300222017000214170827096
:100D9000C1700171417181710A22C2710172417287
:100DA0008172C17230220273012242738173C17356
:100DB000017441741A4912208870BDE81040ACE7F4
:100DC00010BD1CB5FFF794FF002869D01F480A2208
:100DD0000621008883B2684600F020FA14480022F9
:100DE000403080230270437082700121C170202145
:100DF000017143718271C2714122027254224272A6
:100E00004F2282724C22C272017341738173C1738B
:100E1000462202745023437472238374692317E0BB
:100E2000DC00001068360000B0010010CC0000109B
:100E3000B00700105553425300C009200080004005
:100E4000A0860100C800001020A1070004040000D3
:100E5000C3746E230375742343758175C2756C2248
:100E6000027661224276732282766822C276017708
:100E700041778177C1779DF8011080F820109DF8A7
:100E8000021080F821109DF8031080F822109DF8C0
:100E9000041080F82310DD4924208870FFF73DFFFF
:100EA0001CBD10B5FFF724FF00280CD0D848032143
:100EB0000170002141708170C170D4490420887094
:100EC000BDE8104029E710BD10B5FFF711FF00285D
:100ED00010D0CF4800210622017042708170C1708D
:100EE000017141718171C171C84908208870BDE8E4
:100EF000104012E710BD10B5FFF7FAFE002815D01C
:100F0000C24AC348116A491E0B0E03700B0C437092
:100F10000B0A8370C170002101714171022383713A
:100F2000C17108209070BDE81040F6E610BD10B504
:100F3000FFF7DEFE002819D0B5480021B34B017041
:100F4000417081700822C2701A6A140E0471140C68
:100F50004471140A8471C271022202724172827257
:100F6000C1720C209870BDE81040D6E610BD2DE986
:100F7000F041A64DA64C0021A8784034A44A02E0D6
:100F8000535C6354491C03468142F9D31F2B72D131
:100F90002068A04988426ED19D4E60685F364FF050
:100FA00001087060A068B060607B18B9A07B08B1D0
:100FB000102802D986F80C8059E0E07B1E28F9D071
:100FC0000FDC12282ED005DC48B30328F2D1BDE88F
:100FD000F041D0E61528EDD01A28EBD1BDE8F0415C
:100FE0005FE702272A2828D010DC23281DD02528D7
:100FF0001ED02828DED1FFF757FE002826D0207B00
:10100000000618D56F70BDE8F0414FE52F281ED0BF
:101010005528CFD05A28CDD1BDE8F04154E7BDE8DE
:10102000F04194E6BDE8F041CBE6BDE8F0417EE753
:10103000BDE8F0415FE7022016E0FFF735FE00282B
:1010400004D0207B00060ED485F801802AE6FFF745
:101050002BFE0028FAD0207B000604D485F80180FE
:10106000C5F828801EE6822001F0FAF83773BDE843
:10107000F04148E5FFE7822001F0F2F8022001F09C
:10108000EFF8062068700DE6604810B54178022937
:1010900008D003290ED004290FD0052901D1002141
:1010A000417010BD5A484030C07B2828F9D1BDE8B6
:1010B0001040FBE4BDE8104025E5822001F0D0F8A7
:1010C000F8E710B55249022001F0DEF84F49887068
:1010D000487858B101280CD0022001F0C1F84C49E1
:1010E00002205F310873BDE810400CE5BDE81040F8
:1010F0003DE747484030C07B2A2804D02F2805D13F
:10110000BDE8104093E5BDE8104065E510BDFFB5B2
:101110000246002002EB420501464FF400666C4691
:1011200003AA6B1844F82130B34202DD002004B05A
:10113000F0BD394F07EB6307DB073F78575401D009
:101140003B095354535C8F0003F00F035354BB40CF
:10115000491C18440329E4DBE9E7F0B50546002003
:10116000044602462C4B4FF4007700E0641C2E5DD1
:1011700036B102EB040C9C449CF800C4B445F5D095
:10118000032C3ED302F580601844047F457FC67F60
:1011900004EB0524857F2D0405EB06652C4451EAFC
:1011A00004052AD021B91949496840318C4224D814
:1011B000174C00216C3455181D4495F800546554A3
:1011C000491C0C29F7D3817EC27E01EB0221027DEE
:1011D000407D120402EB00600C182046FFF797FFD9
:1011E00040F6F57502E000BFFFF791FFC11EA9426E
:1011F000FAD3A0F57061FF3901D00020F0BD204680
:10120000F0BD2032BA42B2D3F0BD0000DC000010C5
:10121000F007001055534243B0010010FFB559A626
:101220000446E1CE8DE8E100022902DA002004B094
:10123000F0BD6018002100F8011D6946B3FBF2F50E
:1012400002FB1535B3FBF2F34D5D00F8015DA042E2
:10125000F4D8ECE702460020332A01D0432A06D115
:101260004A78312A03D18978312900D10120704789
:1012700002004FF0000009D0012A0ED0022A04D14A
:10128000C978662907D0462905D07047C9786B29E7
:1012900001D04B29F9D101207047C9786E29FAD0C5
:1012A0004E29F8D07047F0B50646002004460546A2
:1012B0000346F25CA2F13007092F01D8FDB209E024
:1012C000A2F14107052F02D8373AD5B202E0613AC0
:1012D000052A05D95B1CDBB205EB0414042BE8D30B
:1012E0000988A14200D10120F0BD10B501F093F9A9
:1012F0002848294C006840B101F0FCFAA0F5C8204C
:10130000206001F0F7FA606010BD01F0F3FA6FF4AD
:1013100048210844206001F0EDFA6FF4C821084428
:10132000F1E7F8B51C4D034600242E687018696873
:1013300087188F4200D9881A00920246304601F081
:10134000F6F92046F8BD0B460146134810B5006873
:101350000024184401F01AFC204610BD70B500228C
:101360000D4C134608340AE0E65C855C5B1C754056
:10137000DBB28554402B00D30023521CD2B28A42E8
:10138000F2D370BD303132333435363738394142DB
:1013900043444546CC000010140100104B4A10474E
:1013A00010B572B633244A4B10C307C349484FF4F3
:1013B0007A710068B0FBF1F01860191D4448FFF71E
:1013C000EDFF62B610BD424A32231360C2E901014B
:1013D00040484FF47A710068B0FBF1F0D06002F140
:1013E00014011046DAE73A4A34231360C2E90101D6
:1013F00038484FF47A710068B0FBF1F0D06002F128
:1014000014011046CAE710B572B60424324900BF71
:1014100051F82420824212D92F49783951F82410EA
:10142000814207D121460846FFF7CDFF21460846F5
:10143000FFF7D9FF21460846FFF7C5FF02E0641C0D
:101440001D2CE5D962B610BD2DE9F041234C23686F
:1014500003B920601E4D00202835636803E00F5C4F
:101460001E18401CAF559042F9D398184FF480765F
:101470006060B04213D12068FFF7C5FF144D1435EA
:10148000286800B1FEE71249324628312068FFF78C
:1014900087FF286800B1FEE7002060602060002020
:1014A000BDE8F0810E494FF480400860FEF780BE31
:1014B00000214FF480404FF4D02208C890421944D4
:1014C000FBD309B10020704701207047F11FFF1FB7
:1014D0006808001074010010503700005C01001013
:1014E00008ED00E0002070475849C20702D04FF4D1
:1014F00080028A61800702D54FF4001088610020C5
:1015000070475249C20702D04FF48002CA61800777
:1015100002D54FF40010C86100207047014600203A
:101520004A4ACB0703D053695B0200D501208907E3
:1015300004D55169890201D540F00200704710B509
:101540000446FFF7EBFF0346FFF7DBFF24EA030047
:10155000FFF7CAFF002010BD10B53D4B38B15968E8
:101560000424042906D2DFE801F0061D37540020C8
:101570005860986010BD042807D005280AD00124BF
:1015800002285ED001284CD010BD0320FFF7B9FF20
:1015900001201EE0BDE810400120B2E7FFF7A4FFE4
:1015A0005C6010BD062808D00328FAD00928ECD0CA
:1015B0000D280AD00C28E8D010BD0320FFF7A1FFAA
:1015C0000220FFF791FF022021E00320FFF799FF9F
:1015D0000220BDE8104087E7062808D00A280FD06F
:1015E00009281ED00C28D0D00D28EED010BD986848
:1015F00010F01F0F00F101009860F7D102201DE0EC
:101600000320FFF77EFF0120FFF76EFF03205860E5
:1016100010BD07280AD00A28B7D00B2811D00928F6
:10162000F6D10320FFF76DFF0120B7E7986810F0AF
:101630001F0F00F101009860EAD10120BDE81040C1
:101640007DE70320FFF75DFF0220A7E700C0092028
:10165000640100104F4810B52021C0F8A01100BF50
:10166000D0F8A0114906FBD50521C0F804114FF0B0
:101670004472C0F8A8214FF48062C0F8AC21012266
:10168000C0F80C210B23C0F88430C0F88020AA22B7
:10169000C0F88C205523C0F88C3000BFD0F88840AB
:1016A0006401FBD50324C0F88040C0F88C20C0F84A
:1016B0008C30C0F808113849C0F8C4100021C0F8B7
:1016C000C811D0F888106FEA11618A073349D0F841
:1016D0000C2102F0030207D07AB3012A44D0022A77
:1016E00047D0032A4ED13AE02AB1012A13D0022A68
:1016F00024D0032A46D1D0F88820D0F80431C2F390
:101700000742DBB2521C5B1C5A43D0F88830244C91
:10171000C3F30E030EE0D0F88820D0F80431C2F3F2
:101720000742DBB2521C5B1C5A43D0F888301D4C78
:10173000C3F30E035B1C634321E010E0D0F8882064
:10174000D0F80431C2F30742DBB2521C5B1C5A438F
:10175000D0F888304FF47A44C3F30E03EAE7D0F8A8
:101760000421114BD2B209E0D0F804210F4BD2B2C0
:1017700004E0D0F804214FF4FA43D2B2521CB3FB78
:10178000F2F20A60016821F4704141F400510160F5
:1017900010BD000000C00F40DC966883740100108B
:1017A00000127A0000366E0100093D00001BB700F0
:1017B000424900200867C86002224A6188613022DD
:1017C000CA633F498A683F49C1E900203E49086031
:1017D0003E49086078463E490860002070472DE980
:1017E000F04341F288320024374F384E384B904254
:1017F00008D8642800D228B942F21072914201D868
:10180000052907D286203860784634601860862023
:10181000BDE8F083DFF8A890D9F80850294AD2F83B
:1018200000C0A5EB0C05D2F804C00CEB4C08C8EBCB
:10183000CC1CB5EBCC0F06D205203860784634605E
:1018400018600520E4E71D4D4FF0020CC5F804C0F8
:1018500048B1DFF88080B8FBF0F04010A861C5F80F
:1018600004C001206860D9F80800C2E900013C60AA
:101870007846346018600020CAE770B5114C002526
:101880000E466560FFF7ABFF0F49000601D50868FB
:1018900070BD0B4B06EB46022068C2EBC6129E6879
:1018A000361AB6EBC20FFAD3044802224260C26B6A
:1018B00002F0FE02C2636560E9E700000000094033
:1018C0000080004078010010D0000010D40000100B
:1018D000D8000010001BB700F0B5FF48002181625E
:1018E000016821F440310160016C21F4403141F480
:1018F00000310164F9498215CA610B6843F48073B1
:101900000B60036823F440530360036C23F44053DB
:1019100043F4005303644024CC610B6843F040035C
:101920000B60036823F440630360036C23F440639B
:1019300043F4006303642023CB610B6843F020036E
:101940000B60036823F440730360036C23F440735B
:1019500043F4007303641023CB610D6845F0100558
:101960000D60C56825F00C05C560C56C25F00C053B
:1019700045F00805C5645502CD630E6A46F400368D
:101980000E62066926F440560661066D26F440563E
:1019900046F4005606658C650C6C44F040040C64FB
:1019A000046924F00304641C0461046D44F003041E
:1019B0000465046924F00C04241D0461046D44F0E2
:1019C0000C040465046924F0300444F0100404613C
:1019D000046D44F030040465046924F0C00444F04C
:1019E00040040461046D44F0C0040465046924F4F7
:1019F000407444F480740461046D44F440740465DC
:101A0000046924F4406444F480640461046D44F483
:101A100040640465046824F4404444F400440460D1
:101A2000046C24F440440464046824F4402444F422
:101A300000240460046C24F440240464446824F00A
:101A40000C044460446C24F00C044464CD610C68C4
:101A500024F400340C60446824F030044460446C86
:101A600024F0300444F0200444649402CC610D68F6
:101A700025F480250D60C56845F44025C560C56C1A
:101A800025F4402545F40025C564C56845F040456A
:101A9000C560C56C25F0404545F00045C564056846
:101AA00025F0300545F010050560056C25F0300582
:101AB00045F020050564056825F0C00545F04005A2
:101AC0000560056C25F0C0050564056925F04065D5
:101AD00045F080650561056D25F040650565056883
:101AE00025F0404545F080450560056C25F04045F2
:101AF00045F000450564456825F003056D1C45600B
:101B0000456C25F003054564056925F4403545F429
:101B100000350561056D25F4403545F40035056552
:101B2000056925F4402545F400250561056D25F47A
:101B300040250565056825F00305AD1C0560056CAD
:101B400025F00305AD1C0564056825F00C0545F07E
:101B500008050560056C25F00C050564C56845F4AD
:101B60004035C560C56C25F4403545F40035C56485
:101B7000C56845F44045C560C56C25F4404545F44D
:101B80000045C564C56845F44075C560C56C25F45D
:101B9000407545F40075C564C56825F44055C560B9
:101BA000C56C25F44055C56495038D630E6A46F4F3
:101BB00080060E62C66826F44066C660C66C26F4CF
:101BC0004066C66456038E630F6A47F400170F62BF
:101BD000C76827F44017C760C76C27F44017C7646D
:101BE00097048F630F6A47F080670F62C76827F01A
:101BF0003007C760C76C27F03007C7648C630C6A76
:101C000044F480240C62446824F0407444F08074EE
:101C10004460446C24F040744464446824F44004F8
:101C200044F480044460446C24F4400444644468F4
:101C300044F440744460446C24F440744464446844
:101C400044F0C0044460446C24F0C004446444681C
:101C500024F0406444F080644460446C24F04064A8
:101C600044F000644464446824F0405444F08054D8
:101C70004460446C24F0405444F000544464C4680C
:101C800024F0405444F00054C460C46C44F0405408
:101C9000C464C46924F44024C461C46D44F4402481
:101CA000C4655404CC670C6E44F000740C66446840
:101CB00024F4401444F480144460446C24F440142C
:101CC00044F400144464446824F4404444F48044DC
:101CD0004460446C04E0000000C0024000C00920E1
:101CE00024F4404444F400444464446824F440240C
:101CF00044F480244460446C24F4402444F40024DC
:101D00004464446824F4403444F480344460446CB3
:101D100024F4403444F400344464446824F44054CB
:101D20004460446C24F4405444F400544464CD6151
:101D30000C6844F480040C60446824F440644460FB
:101D4000446C24F4406444F400644464CE610C6840
:101D500044F400140C60446A24F0407444F00074AD
:101D60004462446E24F0407444F000744466446A53
:101D700024F0406444F000644462446E24F0406403
:101D800044F000644466846824F00C048460846C2D
:101D900024F00C0444F0080484640224CC630C6A2C
:101DA00044F002040C62846824F003048460846CB0
:101DB00024F0030484640124CC630C6A24F001043D
:101DC0000C62C46824F00304C460C46C24F00304EF
:101DD000A41CC4641402CC630C6A44F480340C6206
:101DE000046924F440040461046D24F4400404658F
:101DF000C414CC650C6C24F400640C64046924F4F1
:101E000040140461046D24F4401404650415CC6589
:101E10000D6C25F480650D64C56825F4400545F416
:101E20008005C560C56C25F4400545F40005C56412
:101E3000C56825F0C005C560C56C25F0C00545F036
:101E40008005C564D502CD630E6A46F400260E6295
:101E5000C66826F0C006C660C66C26F0C00646F00E
:101E60008006C664CD630D6A45F400250D62856861
:101E700025F440758560856C25F4407545F4007542
:101E80008564CB630B6A43F010030B62836823F411
:101E900040338360836C23F4403343F40033836422
:101EA0008A630A6A42F480720A62826822F04052AF
:101EB0008260826C22F04052826422018A630A6A44
:101EC00042F480420A62826822F440128260826C8C
:101ED00022F4401282648C63086A40F480600862D5
:101EE000F0BD0000664800214FF0011281800170B2
:101EF0004170C0E90221704761491C31002000F0A7
:101F0000C3B910B55E4C1434A288402A00D94022CF
:101F10008020216800F0E9F9216801442160A1884E
:101F2000081AA08010BD10B5554C0020143421684B
:101F300000F0AAF9216801442160A188081AA08054
:101F400010BD00221146802000F0CFB94D4900207D
:101F500000F09AB92DE9F041494C00271C34484D56
:101F60002178A4F10806082863D2DFE800F06204B3
:101F7000647262628381FFF7BFFF2078C00900F0BE
:101F800050F9E088B0802078C0F34111F1BB61784E
:101F90000C294AD2DFE801F00609490B49101A1D45
:101FA0001F25314201F0B8F94DE0002000E001208A
:101FB00001F0F2F950B306E010F01F0F35D1A07810
:101FC00040F080002870BDE8F041BAE701F068F900
:101FD00039E000202AE010F01F0F26D12848401CCD
:101FE0001AE010F01F0F20D101F01EFA70B1FFF7B8
:101FF000A8FFBDE8F041FEF767B900F01F00012817
:1020000013D1687810B12079A97800E00DE08842FA
:102010000BD21B491031084430601CE000F01F0057
:10202000012802D101F0A8FAC4E7802000F018F9D5
:10203000B780BDE8F081080608D4B0880028F8D041
:10204000FFF771FFB0880028EFD0F2E7BDE8F0415C
:102050007CE7080602D5BDE8F04152E72878010682
:10206000E7D500F07F002870BDE8F04100F041B8EE
:10207000802000E00020BDE8F04100F0FBB8000047
:10208000800100109009001001460007C00E0906EB
:1020900000D5401C7047DA491022C1F80822C1F867
:1020A000100200BFD1F80002C006FBD57047D44A29
:1020B0001023C2F80832C2F8100200BFD2F80002A2
:1020C000C006FBD5C2F80832C2F81012D2F80002DE
:1020D000C006FBD57047CA493022C1F80822C1F8B2
:1020E000100200BFD1F800028006FBD5D1F814021F
:1020F000704730B5C349C44D41EA004421462846E3
:10210000FFF7D5FF21462846BDE83040CFE7BC4861
:102110000021C0F848124021C0F84C120122C0F83A
:102120004822C0F84C1200BFD0F80012C905FBD5F8
:102130004FF0FF31C0F83812C0F83412C0F808125E
:102140000C21C0F804127047B04800B5C16821F0F6
:10215000405141F00051C160C16C41F04051C16437
:10216000AB491A200860091D0A6830EA0202FBD157
:102170004FF0E0214FF08070C1F88002A54B202283
:1021800083F80024C1F80001FFF7C1FF00205DF8CB
:1021900004EBAEE710B5040001D0012000E0002000
:1021A0004FF4807141EA00419B48FFF780FF9B4953
:1021B0004FF000700CB1886710BDC86710BD704744
:1021C00010B500B101204FF4807444EA00419448F6
:1021D000FFF76DFF8A480321C0F84412D0F80012BF
:1021E000C905FBD5C0F8084210BD10B5024680787D
:1021F000FFF74AFF8249D1F8443201248440234347
:10220000C1F84432C1F848029088C1F84C0200BFBE
:10221000D1F80002C005FBD54FF48070C1F8080268
:1022200010BD704700B5FFF72FFF7E495DF804EB46
:1022300041EA004089133AE700B5FFF725FF7949E5
:102240005DF804EB41EA0040774930E700B5FFF75D
:102250001BFF74495DF804EB41EA0040891326E74F
:1022600000B5FFF711FF6F495DF804EB41EA00404C
:102270006E491CE700B5FFF707FF6A495DF804EBFC
:1022800041EA0040891312E700F00F02012370B504
:1022900003EB82035A4AC2F8283200BFD2F8203238
:1022A0001C05FBD5C3F309030024DD1C05E000BFBA
:1022B000D2F8186241F8046B641CB4EB950FF7D3A5
:1022C0000021C2F8281241F24821C140C9070AD1B1
:1022D000FFF7DAFE4FF4A06141EA0040FFF7DBFEB2
:1022E0005348FFF7D8FE184670BD70B51346054633
:1022F000434C00F00F00022202EB8000C4F82802D9
:10230000C4F824320020DA1C05E000BF51F8046B49
:10231000C4F81C62401CB0EB920FF7D30020C4F845
:1023200028022846FFF7B0FE4FF4A06141EA0040C2
:10233000FFF7B1FE3F48FFF7AEFE184670BD2DE92E
:10234000F0412F4DD5F80032C5F80832180721D5D5
:102350003148FFF7A0FE3848FFF7BDFEC10605D59E
:10236000FFF7D5FEBDE8F041FDF79FBF810705D51A
:10237000BDE8F04100F00100FDF791BF010709D56C
:10238000400703D5BDE8F041FDF796BFBDE8F04139
:10239000FDF799BF294E58074FF001071CD4BDE83F
:1023A000F0810024D5F8302207FA04F10A4210D057
:1023B0006008C5F8381200BFD5F800128906FBD5B1
:1023C000D5F81412E2070CD056F8201009B10320FA
:1023D0008847641C202CE5D3D5F830020028E0D1D2
:1023E000DDE73CB9490705D5316819B101208847B7
:1023F0000124D7E756F820100029EAD00220E7E7A9
:1024000000C00050000180000005D00000C0024064
:10241000F4CF005018E000E00005FE0000C00920E5
:102420000005D80000054000000120000001010067
:102430000005F2000005FA000002FE006C38000002
:102440002DE9F047FE4E80464FF080773068BC1192
:10245000FC4DB84249D100BF00BF00BF00BF00BF64
:1024600000BF00BF00BF00BF00BF00BF00BF00BF74
:1024700000BF00BF00BF00BF00BF00BF00BF00BF64
:1024800000BF00BF00BF00BF00BF00BF00BF00BF54
:1024900000BF00BF00BFEC631520FDF745FF002023
:1024A000FDF742FF00F0FF09AC6300BF00BF00BFB3
:1024B00000BF00BF00BF00BF00BF00BF00BF00BF24
:1024C00000BF00BF00BF00BF00BF00BF00BF00BF14
:1024D00000BF00BF00BF00BF00BF00BF00BF00BF04
:1024E00000BF00BF00BF00BF00BF00BF00BF00BFF4
:1024F00000BF00BF00BF00BF00BF00BF00BF00BFE4
:1025000000BF00BF00BF00BF00BF00BF00BF00BFD3
:1025100000BF00BF00BF00BF00BF00BF00BF00BFC3
:1025200000BF00BF00BF00BF00BFEC630620FDF787
:10253000FBFEAC6300BF00BF00BF00BF00BF00BF19
:1025400000BF00BF00BF00BF00BF00BF00BF00BF93
:1025500000BF00BF00BF00BF00BF00BF00BF00BF83
:1025600000BF00BF00BF00BF00BF00BF00BF00BF73
:1025700000BF00BF00BF00BF00BF00BF00BF00BF63
:1025800000BF00BF00BF00BF00BF00BF00BF00BF53
:1025900000BF00BF00BF00BF00BF00BF00BF00BF43
:1025A00000BF00BF00BF00BF00BF00BF00BF00BF33
:1025B00000BF00BFEC630120FDF7B6FE4FEA8800C4
:1025C000FDF7B2FE3068B84202D14846FDF7ACFED6
:1025D000AC6300BF00BF00BF00BF00BF00BF00BFB3
:1025E00000BF00BF00BF00BF00BF00BF00BF00BFF3
:1025F00000BF00BF00BF00BF00BF00BF00BF00BFE3
:1026000000BF00BF00BF00BF00BF00BF00BF00BFD2
:1026100000BFBDE8F0872DE9F0474FF0000900BF8B
:1026200000BF00BF00BF00BF00BF00BF00BF00BFB2
:1026300000BF00BF00BF00BF00BF00BF00BF00BFA2
:1026400000BF00BF00BF00BF00BF00BF00BF00BF92
:1026500000BF00BF00BF00BF00BF00BF00BF794E7A
:102660004FF48025F5639F20FDF75EFE0020FDF707
:102670005BFE00F0FF080020FDF756FEC4B200200C
:10268000FDF752FEC1B2B56300BF00BF00BF00BF7F
:1026900000BF00BF00BF00BF00BF00BF00BF00BF42
:1026A00000BF00BF00BF00BF00BF00BF00BF00BF32
:1026B00000BF00BF00BF00BF00BF00BF00BF00BF22
:1026C00000BF00BF00BF00BF5F4D604E604FB8F15C
:1026D000C20F01D1202C07D0822028602120306039
:1026E00078463860822094E75548142912D015297D
:1026F00013D0162915D0182916D0C0F80090002044
:10270000FFF79EFEC5F800907846C6F80090386046
:1027100000207EE74FF4801101E04FF400110160CA
:10272000EDE74FF48001FAE74FF08071F7E72DE90C
:10273000FF4F8DB00D46DDF868900026424C0793A0
:102740005FEA09013FD04FF4805701463A46684698
:10275000FDF73BFEDDE900B10C913A46691C684685
:10276000FDF733FEDDE90010CDE904013A46684685
:102770000F99FDF72AFEDDE9008500BFA9EB0607EA
:10278000C5F58050B84200D2074625B1D84556D18C
:102790000C98854253D14FF48050FDF7E7FD5FEA76
:1027A000000A1CD0D8455CD10C98854259D12A46E4
:1027B0004FEA0830514600F0F1F8000619D55046AE
:1027C00000F0E8FB84E086202060204809210160B9
:1027D00078461F490860862011B0BDE8F08F82203E
:1027E00020601A4822210160794619480160822040
:1027F000F2E70598804509D1049901EB0030C1F555
:102800008052514400F0CAF80006D8D4404600F087
:1028100042F90006D3D407983A46811905EB0A001D
:1028200000F0DFFBEA194FEA0830514600F01AFBCE
:102830000006C4D4059988453DD104980AE03EE0DD
:10284000AC01001000C00920D0000010D40000101E
:10285000D800001000EB01300499C1F580525144BA
:1028600025E0059988450AD1049800EB01300499C8
:10287000C1F58052514600F091F800069FD44046C1
:1028800000F009F900069AD407983A4681190F9882
:10289000304400F0E7FA000691D4059988450AD142
:1028A000049800EB01300499C1F58052514600F0C4
:1028B000D9FA000683D4504600F06CFB0AE0079872
:1028C0003A4681190F98304400F0CCFA000601D541
:1028D000206881E73E44002508F101084E45FFF4D9
:1028E0004DAF064900202060086078460449086022
:1028F000002071E70348006870470000D400001012
:10290000D8000010AC01001070B500BF00BF00BFC0
:1029100000BF00BF00BF00BF00BF00BF00BF00BFBF
:1029200000BF00BF00BF00BF00BF00BF00BF00BFAF
:1029300000BF00BF00BF00BF00BF00BF00BF00BF9F
:1029400000BF00BF00BF00BF00BFD04C4FF48025C8
:10295000E5630620FDF7E8FCA56300BF00BF00BFEC
:1029600000BF00BF00BF00BF00BF00BF00BF00BF6F
:1029700000BF00BF00BF00BF00BF00BF00BF00BF5F
:1029800000BF00BF00BF00BF00BF00BF00BF00BF4F
:1029900000BF00BF00BF00BF00BF70BD2DE9FC5FDE
:1029A000BB4DBC4EBC4F5FEA020A8B4604464FF05B
:1029B00000080DD001A9B94800F002F980B18220C9
:1029C000286021203060784638608220BDE8FC9F76
:1029D000C5F800807846C6F8008038600020F5E72A
:1029E00003208DF80000200C8DF80100200A8DF8DE
:1029F00002008DF8034000BF00BF00BF00BF00BF52
:102A000000BF00BF00BF00BF00BF00BF00BF00BFCE
:102A100000BF00BF00BF00BF00BF00BF00BF00BFBE
:102A200000BF00BF00BF00BF00BF00BF00BF00BFAE
:102A300000BF00BF00BF954C4FF48029C4F83C9004
:102A400004216846FDF777FC51465846FDF77FFCA8
:102A5000C4F8389000BF00BF00BF00BF00BF00BF78
:102A600000BF00BF00BF00BF00BF00BF00BF00BF6E
:102A700000BF00BF00BF00BF00BF00BF00BF00BF5E
:102A800000BF00BF00BF00BF00BF00BF00BF00BF4E
:102A900000BF00BF9CE72DE9FC47044601A97F4821
:102AA00000F08EF87A4D7B4EDFF8EC9148B1822031
:102AB00028602220794630608220C9F80010BDE8E5
:102AC000FC879DF80400800701D4FFF71DFF20203C
:102AD0008DF8000020098DF8010020018DF802001A
:102AE00000248DF8034000BF00BF00BF00BF00BF3F
:102AF00000BF00BF00BF00BF00BF00BF00BF00BFDE
:102B000000BF00BF00BF00BF00BF00BF00BF00BFCD
:102B100000BF00BF00BF00BF00BF00BF00BF00BFBD
:102B200000BF00BF00BFDFF864814FF48027C8F802
:102B30003C7004216846FDF7FEFBC8F8387000BF02
:102B400000BF00BF00BF00BF00BF00BF00BF00BF8D
:102B500000BF00BF00BF00BF00BF00BF00BF00BF7D
:102B600000BF00BF00BF00BF00BF00BF00BF00BF6D
:102B700000BF00BF00BF00BF00BF00BF00BF2C6090
:102B8000794634600020C9F8001098E770B5414DCF
:102B9000414E3F4C2AB1FFF701FF000609D52068DE
:102BA00070BD86202060092028607846306086202D
:102BB00070BD00202060286078463060002070BD25
:102BC0002DE9F041364C0F460646A56806E0A068A0
:102BD000401BB04202D30120BDE8F081384600F02E
:102BE00003F80028F3D1F7E770B5044600BF00BF33
:102BF00000BF00BF00BF00BF00BF00BF00BF00BFDD
:102C000000BF00BF00BF00BF00BF00BF00BF00BFCC
:102C100000BF00BF00BF00BF00BF00BF00BF00BFBC
:102C200000BF00BF00BF00BF00BF00BF174E4FF482
:102C30008025F5630520FDF777FB0020FDF774FB89
:102C40002070B56300BF00BF00BF00BF00BF00BF62
:102C500000BF00BF00BF00BF00BF00BF00BF00BF7C
:102C600000BF00BF00BF00BF00BF00BF00BF00BF6C
:102C700000BF00BF00BF00BF00BF00BF00BF00BF5C
:102C800000BF00BF207800F0010070BD00C0092027
:102C9000D0000010D4000010D8000010A086010061
:102CA000008000402DE9F34F85B0044603A9B348E6
:102CB00000F0FDF8B24DB34EB34F4FF0820B18B198
:102CC0002120C5F800B060E0FFF71EFE42208DF81D
:102CD00000004FF0000ACDF801A0CDF805A0ADF836
:102CE00009A000BF00BF00BF00BF00BF00BF00BF02
:102CF00000BF00BF00BF00BF00BF00BF00BF00BFDC
:102D000000BF00BF00BF00BF00BF00BF00BF00BFCB
:102D100000BF00BF00BF00BF00BF00BF00BF00BFBB
:102D200000BFDFF868924FF48028C9F83C800B217F
:102D30006846FDF700FBC9F8388000BF00BF00BF40
:102D400000BF00BF00BF00BF00BF00BF00BF00BF8B
:102D500000BF00BF00BF00BF00BF00BF00BF00BF7B
:102D600000BF00BF00BF00BF00BF00BF00BF00BF6B
:102D700000BF00BF00BF00BF00BF03A97F4800F035
:102D800096F848B12220C5F800B030607846386027
:102D9000822007B0BDE8F08F9DF80C00800701D4B9
:102DA000FFF7B2FD02208DF80000200C8DF8010025
:102DB000200A8DF8020006988DF803408DF8040073
:102DC00000BF00BF00BF00BF00BF00BF00BF00BF0B
:102DD00000BF00BF00BF00BF00BF00BF00BF00BFFB
:102DE00000BF00BF00BF00BF00BF00BF00BF00BFEB
:102DF00000BF00BF00BF00BF00BF00BF00BF00BFDB
:102E00004446C846C9F83C4005216846FDF793FA98
:102E1000C8F8384000BF00BF00BF00BF00BF00BF00
:102E200000BF00BF00BF00BF00BF00BF00BF00BFAA
:102E300000BF00BF00BF00BF00BF00BF00BF00BF9A
:102E400000BF00BF00BF00BF00BF00BF00BF00BF8A
:102E500000BF00BFC5F800A07846C6F800A03860E3
:102E6000002096E72DE9F05F454EDFF81891DFF876
:102E700018A1150083460F464FF000080ED000241D
:102E80000AE0395D0BEB0400FFF70CFF000602D5EA
:102E90003068BDE8F09F641CAC42F2D3C6F80080F5
:102EA0007946C9F800800020CAF80010F1E72DE942
:102EB000F041374C0F460646A56806E0A068401B67
:102EC000B04202D30120BDE8F081384600F003F89B
:102ED0000028F3D1F7E770B5044600BF00BF00BF7C
:102EE00000BF00BF00BF00BF00BF00BF00BF00BFEA
:102EF00000BF00BF00BF00BF00BF00BF00BF00BFDA
:102F000000BF00BF00BF00BF00BF00BF00BF00BFC9
:102F100000BF00BF00BF00BF00BF1C4E4FF48025A4
:102F2000F5630520FDF700FA0020FDF7FDF920709C
:102F3000B56300BF00BF00BF00BF00BF00BF00BF40
:102F400000BF00BF00BF00BF00BF00BF00BF00BF89
:102F500000BF00BF00BF00BF00BF00BF00BF00BF79
:102F600000BF00BF00BF00BF00BF00BF00BF00BF69
:102F700000BF207800F0010070BD0000A0860100B5
:102F8000D0000010D4000010D800001000C00920AC
:102F90000080004070B50446051FFDF721FA006867
:102FA000002C14BF446870BD002C18BFAC423CBF5D
:102FB00020466468F8D301680A18AA4218BF456021
:102FC00003D12A6805461144016028684119A142CD
:102FD0001CBF6C6070BD616869602168084428602E
:102FE00070BD032A40F2308010F0030C00F0158011
:102FF00011F8013BBCF1020F624498BF11F801CBFC
:1030000000F8013B38BF11F8013BA2F1040298BF60
:1030100000F801CB38BF00F8013B11F0030300F0CA
:103020002580083AC0F0088051F8043B083A51F86E
:1030300004CBA0E80810F5E7121D5CBF51F8043B73
:1030400040F8043BAFF30080D20724BF11F8013BE6
:1030500011F801CB48BF11F8012B24BF00F8013B48
:1030600000F801CB48BF00F8012B704710B5203A9B
:10307000C0F00B80B1E81850203AA0E81850B1E831
:103080001850A0E81850BFF4F5AF5FEA027C24BFE7
:10309000B1E81850A0E8185044BF18C918C0BDE8DE
:1030A00010405FEA827C24BF51F8043B40F8043BA7
:1030B00008BF7047D20728BF31F8023B48BF11F85C
:1030C000012B28BF20F8023B48BF00F8012B7047B6
:1030D0007047704738B504460A4600206946AFF38A
:1030E0000080002808BF38BD02460099204600F045
:1030F00034F8012038BD012000F049B8F8B5AFF32D
:103100000080054600200C46102000BF0646A81986
:10311000A0420DD9324669460020AFF30080070077
:1031200008BF00F034F80098A04218BF0546C41943
:10313000FDF756F905600746F01D20F00700461917
:103140002846FDF751F9B44208BFF8BDA21B31462D
:103150003868BDE8F840AFF30080034640688C460D
:10316000002818BF88423CBF03464068F8D318685F
:103170001844884207D00CF1030020F00700001D1E
:10318000411A521A0146081D0A60FFF703BF10B525
:1031900000F038F8BDE8104000F02EB87546FDF795
:1031A0002BF9AE4605006946534620F007008546D8
:1031B00018B020B5FDF730F8BDE820404FF000060C
:1031C0004FF000074FF000084FF0000B21F007010F
:1031D000AC46ACE8C009ACE8C009ACE8C009ACE852
:1031E000C0098D46704710B50446AFF300802046F5
:1031F000BDE81040FCF7D5BF002801D000F02AB888
:103200007047000010B5012805D0002103A000F090
:1032100027F8012010BD09A1F8E7000053494752E3
:10322000544D454D3A204F7574206F662068656196
:1032300070206D656D6F7279000000003A2048655E
:103240006170206D656D6F727920636F7272757039
:103250007465640001491820ABBEFEE72600020039
:1032600070B505460C460A2000E06D1C00F011F810
:1032700035B128780028F8D102E0641C00F009F884
:1032800014B120780028F8D1BDE870400A20AFF3CF
:10329000008008B569468DF800000320ABBE08BD6C
:1032A000194810B5007810F01F0F1748C07829D1C1
:1032B00015490839012806D0134A0228937806D008
:1032C00003281FD112E011480860122012E01048B4
:1032D000002204E004780CB144882044521C93423C
:1032E000F8D1027872B10860408803E009481844B8
:1032F000086000788A88824200D98880FEF701FE43
:10330000012010BD002010BD9C010010C837000036
:10331000DA370000FB37000070B51D481C4D0078FF
:10332000A5F1080510F01F040AD01948A5F11401F1
:10333000184B4A780079012C06D0022C26D109E0DE
:103340001348183828601DE002B3897888421DD2DE
:10335000002015E000F08F04200605D504F00F06CC
:103360004FF48030B04001E00120A0400AB92207AC
:103370000CD18A68024209D0C9680142E8D0012014
:1033800018802B60FEF7BDFD012070BD002070BDD0
:103390009C0100109009001070B502462148A0F170
:1033A0001C04017811F01F030146498804D0012B49
:1033B00029D0022B27D111E0012924D132B10120DB
:1033C000FEF7FDFEA08840F0020005E00020FEF7B9
:1033D000F6FEA08820F00200A08021E0007900F035
:1033E0008F00030605D500F00F034FF480359D4094
:1033F00001E00125854063782BB1030703D0A36862
:103400002B4200D009B1002070BD22B1FEF728FF89
:10341000E068284303E0FEF72DFFE068A843E06082
:10342000012070BD9C0100102DE9F84F504F002085
:103430000090B8784FF000094FF0010A4FF4803B3C
:10344000A7F11C0600286AD04A4C64E06078022884
:1034500004D0042840D005285BD140E06179B878D9
:10346000814237D170702079B070414900200C3909
:1034700001F80090401C0428FAD301254FEA060801
:103480000AFA05F0D8F80810084202D02846FEF7DC
:10349000D3FED8F808100BFA05F0084203D045F027
:1034A0008000FEF7C9FE6D1C102DE9D34FF001100E
:1034B000C8E902090120FEF783FEE0794006B8F86A
:1034C000040002D540F0010001E020F00100A8F85E
:1034D00004001EE060881DE0E078009019E000988C
:1034E000B8B9A07800F08F05280604D505F00F01C3
:1034F0000BFA01F001E00AFA05F0B1680143204639
:10350000B160FEF772FE2846FEF78CFE2846FEF7F5
:103510009DFE207804442078002897D11FE086F88B
:10352000019001245546D846B16805FA04F00842D6
:1035300002D02046FEF780FEB16808FA04F0084287
:1035400003D044F08000FEF777FE641C102CEBD310
:103550004FF00110C6E902090020FEF731FEB878ED
:103560007178884202D10120BDE8F88F0020FBE786
:103570009C010010DA3700002DE9FC5F384D002770
:103580003E466878BB46B846002866D0BA46354CF9
:1035900005F11C095DE06078022804D0042808D0F9
:1035A000052854D119E06079697888424FD0608845
:1035B0004EE0A77899F80410E6784FF00008B94279
:1035C00045D199F80200B04241D125484FF0010A97
:1035D000103010F807B0C65539E099F80410B94218
:1035E00035D1A17801F08F010191090605D5019926
:1035F00001F00F024FF4803101E0019A0121914066
:10360000009199F80200B04213D1A8680843A8605D
:10361000E968009881432046E960FEF7E6FD0198DD
:10362000FEF700FE0198FEF711FE009948EA010836
:103630000DE05E450BD118EA010F08D1A868884358
:10364000A860E8688843E8600198FEF7F5FD2078F7
:103650000444207800289ED15046BDE8FC9F00001D
:1036600080010010DA370000EB3C904D53444F537B
:10367000352E3000020201000110000004F80200A3
:10368000010001000000000000000000000029EF20
:10369000BEADDE41544F4C20465072696E744641B7
:1036A0005431322020200000BC380000AC3800002B
:1036B000C8380000CC380000D8380000C0380000FE
:1036C000B8380000B4380000C4380000D03800001A
:1036D000D4380000B03800000000000000100000E6
:1036E00000200000003000000040000000500000FA
:1036F00000600000007000000080000000900000EA
:1037000000A0000000B0000000C0000000D00000D9
:1037100000E0000000F00000000001000080010057
:10372000000002000080020000000300008003008F
:103730000000040000800400000005000080050077
:10374000000006000080060000000700008007005F
:10375000FF0F0000FF1F0000FF2F0000FF3F0000D1
:10376000FF4F0000FF5F0000FF6F0000FF7F0000C1
:10377000FF8F0000FF9F0000FFAF0000FFBF0000B1
:10378000FFCF0000FFDF0000FFEF0000FFFF0000A1
:10379000FF7F0100FFFF0100FF7F0200FFFF02002B
:1037A000FF7F0300FFFF0300FF7F0400FFFF040013
:1037B000FF7F0500FFFF0500FF7F0600FFFF0600FB
:1037C000FF7F0700FFFF070012011001000000400B
:1037D00051C2031300010420480109022000010125
:1037E00000803209040000020806506207058202C8
:1037F0004000000705020240000000040309041C09
:1038000003410054004F004C002000200020002005
:103810000020002000200020002000280346005047
:1038200000720069006E007400200046006C0061A8
:1038300000730068002000200020002000200020ED
:103840000020001A034600690072006D00770061D5
:10385000007200650030003000300030000E034D73
:103860000065006D006F007200790000551F0000B8
:1038700000000000CB02000000000000000000007B
:103880000000000000000000000000000000000038
:103890000000000000000000000000000000000028
:1038A000000000000000000000000000466562000B
:1038B00044656300417567004A756C004A616E009B
:1038C0004A756E00536570004D6172004170720060
:1038D0004F6374004E6F76004D617900FC38000034
:1038E00000000010B0010000080100009439000041
:1038F000B00100108058000064010000A00D415488
:103900004F4C20465072696E74280546D4284B3DB2
:1039100039609F4574616C6F6E60992012661A3130
:1039200002124E1230120F1BDE30071230122E120E
:10393000663272326D1E4631314E30011546524D9F
:10394000202008BC419737383738263D6E2B380287
:103950004340061B106004411AFF01014C100D4545
:103960005F5553494E475F4D4F5645B81328085889
:1039700038365F54554E455F4550494C4F47551FAB
:103980008A291F1753484946543103192A08033915
:10399000093D000043928B4AEDB7A5C2340B9AC68D
:1039A0005150E2CAA6F135636FDB77013200A209FC
:1039B0007CA9FB6E7B5A5019B5EABAC86D158740D1
:1039C000E36E8E48A7D4421E46A7F962C86337B992
:1039D000735D885874DC980C3FE9A5C87BBB5DEE2D
:1039E000640E46A38C5334C5F22709C356BCF4D7E2
:1039F0006AAFE360915536CD23F9505C88F8D198D1
:103A00000EE4703FA74A2F0E166A69765132565A55
:103A1000B9E2709B6138B4CA65C90DEF6973169C31
:103A2000A80B7EDC2079137E71957ECD6E918097F8
:103A3000D7FAE0A2F1D627E1FC02E15E18C9C7FA85
:103A40009A546858677921E93F2D0F56AB002B9A9D
:103A500066DC1BA8AA116B347E55F75B90AC0FF3A4
:103A60000DD03EC0EE3B153F3C985013C2C1F0CC88
:103A700005FAC82817C074CDEAF6F7D55D24695C4D
:103A8000FDE3B1A49D58867AC4A091DB05119DE8A1
:103A90000029C07639CF996ABB73F17971474C2BF5
:103AA0008BE3CEC61F9B72790A53AB773F282A6FF0
:103AB00076AAB5474E1DA0A48244184FE233204B8E
:103AC000BCC9E8A4F19F70F71AC15D8DAAD420ACDF
:103AD00081AEEB20E5F7A4CC78BF3981F817098FC8
:103AE0004107F94245105B35C9018FB8017699A2AB
:103AF00060A84CC373DD18AC69DA15EB6940EF8C34
:103B000021CB410804F282F6D2F4F8EC6062DCC00A
:103B1000F2BEC73FDAD343B8C7397E0F3F33606187
:103B2000ED7204E4A33FD0A5FDC72A831647654A7A
:103B30007B8BBC738B0DD6AF7FD768BBA84BD10EE8
:103B400044C2C56D96962CE27F745DB0FE2D70B2B6
:103B5000A65D43BDB9243F4AC18F9771B18B90B820
:103B60002B5FADC951FFA6FE306E41BF88FBAF6928
:103B700024285114CD1FAA5C61053B5EFF6F50EEF7
:103B800063BCF2A3664FDB70098BE486A0FB373978
:103B90001CFE9742C5578F693A5A7275D86DB8188E
:103BA000088CC42C90138D23E85BC6459BDE4689A8
:103BB000184771620C347E4A5CFC119C14C0535A45
:103BC0005F22B179963CF45CB8A24FE3FE05BED308
:103BD00036B7D6F04029CFA5F95176EA7F9BC22BA4
:103BE000D186731485BC7E18751FBF02681570F5E9
:103BF00032BA5EA5ED46F1DF3A4401B2B8028FA6B3
:103C0000832F5661C0CCD2E7206DBFAFB131921087
:103C10007E6ACA64A84F8B0917A93586F99BB4BC84
:103C2000B07EC4CA250E04C85692A6FC957D239288
:103C3000A4F0FD156A40423FF794D4F49F177E77B5
:103C4000E5ECE12DE03786FDDD5A37ED6F2B5E0A9E
:103C5000DB07A66103D43243DD1493B07ABC2B5A40
:103C6000A3688D8E940242DDE682CCE27779D29110
:103C7000ED949059EA542A1974653EC9CC0084EE3B
:103C80002C7EC1FF63C3799F435330E04B44EDE486
:103C90009B1DB9F82C376DB5F96FA23E1CD53FBC02
:103CA00000659C058A152D22C17AF656AE69CDAD08
:103CB0000A1A1C5D5747F64310AB8831E3E9BC1E76
:103CC0008FC6E865EE74583A2E85DF3EAF1DB112FF
:103CD000F34465FCC49865F3D843C25E6C2E343A55
:103CE0000E195B4C1183797D93B596CFBAE782E4C8
:103CF00077A7DB73E3952D082AC52DC28D65B75ACA
:103D000067EE75461937338B6B8147C0920AE62000
:103D10005212433D0CD9234425E74614EE30DE8091
:103D2000CF30A9269F1811E789EACF524E77C26893
:103D30006015D2717769A1A2D2DA008798DDA5302B
:103D40009F420937C87E99028933936C459270630C
:103D50003684628AFB8708500B31DDC889422D1AF0
:103D600003E371FADA6310075773EB786A0FBCDE6E
:103D700096FE3310FC1AC9105129E88767E8FD1F29
:103D80006B53FEEB595A96C4455242B6E574DD3288
:103D900000A1F47BC140A9C6F1B02B6C88A7D73134
:103DA000CF1619A6119054F6B2EA89282E376EEC78
:103DB0007007BE3CF1D2EACD0452EC2F78FD07B279
:103DC00057832B833E4A3B56878D0BBC8CBCEBD66E
:103DD00040039D4C0C1DEE8F79E3546E80145D7E84
:103DE0009C636027B5EF6C63AD26E1FA7D265E59D2
:103DF00048DB7297E371489422A6171C21EFE92A49
:103E00001D0B94B2E3EA0BB6B4B57F6E97F8F37F5F
:103E10007A81FB414A5126136F2373E34A794E8915
:103E2000DF8AFF543DE864653986CB538C1F6D5F94
:103E3000F5CDF76E1FC6D00C9368CC84CC5A8E1F7C
:103E40001C5AF0282D802F4C836B51D97E3BB75DD7
:103E500073012935E40F23E478DA8C3D777AC616AE
:103E600085BCABBB2D8F19B450254E9191EF61BC31
:103E70001B0586213E01CA056D5B91804202593FB8
:103E800082C7048402D665190D20B17141C9BBC433
:103E9000905EA9D6BBA50F61B6C16305DB6BA340DD
:103EA000B431F602278C4C360CC6D8ED8FF7FC7D6A
:103EB000778142E6A8069AD85BC7D21811FDB5C62D
:103EC000F861874F37CD1EFC699B11497A70E97FF5
:103ED000680C2A84B438737FE9A639A4795404584D
:103EE0007110911C9200229E8C8BCFA5349AB5E65E
:103EF000D4CA211A41C515BFB7FE32AA09C2A0E52E
:103F00003FB2D0EC7A34D176077492E8F8D25ECB27
:103F10006A65D6DE2869C7BA096F0B2EBC1AE90696
:103F2000B2B4DEADD90E94974B56E26D387300AE45
:103F30002E4A1597CCD49DBAAEF3044682AC1787AF
:103F40007A86C244C90AD2C68B361FE6CAE0D17748
:103F500017ACE9722039BF35B42C9BA81226D98939
:103F6000A3D7D1AD96E03B80C11F14CD8CF8245C63
:103F7000618A056EA26C053B616CEDE168AB648EF5
:103F80003F1D007923FD022453AF7AF71AA8E1D32D
:103F9000EB19D99100718B4D82C66BE883C6C5843D
:103FA000DD4D845BFACF75ABA1B071E3671BAD2526
:103FB0005D679051AFEDA7B4085458DF6AD93BE371
:103FC00091A9627F2F72CF0BDC75D7DEBA7D624E6E
:103FD000216F39712C721AB33E7DC101E5F9245F5E
:103FE000496112997DD3975EE14B1FE03171164C08
:103FF000ECD7F42B33DD1DFD92892FA6E1A2B0F1A1
:1040000028070820A5910200A9910200AB910200A7
:10401000AD910200AF910200B1910200D28EE8DFB3
:10402000000000000000000000000000B39102004A
:10403000B591020000000000B7910200B9910200A2
:10404000BB910200BB91020041360300BB9102000C
:10405000BB910200450A03004D0D0300031003004D
:104060008F120300BB910200BB910200BB910200C2
:10407000BB910200BB910200BB910200BB91020008
:10408000BB910200BB910200BB910200BB910200F8
:10409000BB910200733C0300BB910200BB91020084
:1040A000CF540300BB910200BB910200BB91020000
:1040B000BB910200BB910200BB910200BB910200C8
:1040C000BB910200BB910200BB91020000F002F81C
:1040D00000F088F80AA090E8000C82448344AAF11A
:1040E0000107DA4501D100F07DF8AFF2090EBAE818
:1040F0000F0013F0010F18BFFB1A43F0010318471C
:104100003CE704007CE704000A444FF0000C10F880
:10411000013B13F0070408BF10F8014B1D1108BF45
:1041200010F8015B641E05D010F8016B641E01F8E5
:10413000016BF9D113F0080F1EBF10F8014BAD1C35
:104140000C1B09D16D1E58BF01F801CBFAD505E053
:1041500014F8016B01F8016B6D1EF9D59142D6D3AD
:10416000704700000023002400250026103A28BFD5
:1041700078C1FBD8520728BF30C148BF0B607047D9
:1041800069293DF0318164293DF02E8175293DF08A
:104190002B816F293DF0C28178293DF0E9810368C8
:1041A000DB0928BF41F0800163293DF04A8673296D
:1041B0003DF04F86E3293DF05A86002070471FB539
:1041C0009DE803003DF074FD3DF019FB3DF056FD08
:1041D0000400002000213EF0CFFA401C60601FBDAB
:1041E00010B510BD3DF02FFF1146FFF7E8FF00F0BE
:1041F0001DF93DF04DFF03B4FFF7F2FF03BC3DF0A6
:104200007DFF00000B49D1F800C04A685CF8043B10
:104210001068184442F8040B8C4528BFA1F1DC0C4F
:104220008A4228BFA1F1DC02C1F800C04A6020F038
:1042300000407047AC06001010B5782119483DF0D9
:10424000EDFC19494FF0FF30088010BD1648018879
:10425000491C09B201800A290CD001EB4102114925
:10426000436841F8223001EB820183684B60C068EB
:1042700088607047FEE70C4910B5B1F90000421C98
:104280000ED0084A00EB4003401E52F8234002EBD8
:1042900083024C6053688B609268CA60088010BDCE
:1042A000FEE700003C04001004C00720334850F82B
:1042B000C01F21F0030101603148016821F00401B1
:1042C000016030BF70472D4951F8C42F82430A6006
:1042D0001046704700B56FF40040FFF7F4FF28491F
:1042E0000420086025490820C1F8C00030BF00BD87
:1042F000224951F8C42F02430A60104670471F49F3
:10430000D1F8C410014201D001207047002070474D
:1043100010B51DF002F905281FD12FF08AFCE0B975
:1043200006F02BF9C8B900203CF042FAA8B90120E8
:104330003CF03EFA88B902203CF03AFA68B9032012
:104340003CF036FA48B907202CF03DFB052804D193
:1043500007202CF038FB052807D02FF06AFC002836
:104360000AD1BDE810402FF06DBC0648406DC0F387
:10437000C0202FF067FC30BF10BD000000C00F4010
:1043800010ED00E000C0092038B50546684606F08B
:104390008DFB0D4C000611D49DF80000032809D0B8
:1043A00087200A4920600020086078460849086094
:1043B000872038BD0CF0EEFD000601D5206838BD21
:1043C000284609F037FA38BD08C007200CC007207E
:1043D00010C00720074802214160002101674161A8
:1043E0000B22C260C16301214160002070470020A0
:1043F000704700000080004000487047B40600107D
:10440000C06DBCAEAB1B02000033704770477047F5
:104410004A756E20203220323031360070477047A6
:1044200031353A30363A30370000000088B0C24C9F
:104430000027039720883E4640F002002080BF48B6
:1044400026F033FBBE48007802281CD1FFF7FEFEA1
:1044500003A825F046F9000601D502F0A0FEFFF7FB
:104460000AFF0398B0F58C7F0DDAFFF7EFFE00210D
:10447000B4A030F07DF8000601D502F090FEFFF701
:10448000FAFE02F08CFEAD4D288830F4504010D07A
:104490000127FFF7DBFE32201BF079F8012012F034
:1044A000C1FB10B1032030F066FAFFF7E4FE02F022
:1044B00076FE2888810B06D001270FF059FA0006F6
:1044C00001D502F06CFE2E801FF02AF8000601D5FF
:1044D00002F065FE01F0AEFA07F0C4FA000601D55D
:1044E00002F05DFEA24DAE6805A826F006FA01F0C6
:1044F00059FA10B1012702F052FE01F0DDFADFF89F
:104500007482C0B1FFF7A2FE01F02EFCFFF7B3FEEC
:10451000D8F80000062802D0002197A004E09B49AB
:104520000220087000219AA030F022F8208840F084
:10453000020020800CE001F0DCFC38B1FFF786FEC1
:1045400001F012FCFFF797FE02F029FE01F05AFF7E
:104550009448A968891B8142FBD306A826F0CDF9AF
:10456000914EDFF84892307800EB400159F8310065
:104570008047000601D502F012FE01F0A9FF0006F7
:1045800001D502F00CFE9DF81A009DF81610884225
:1045900001D0012000E0002001F0DCFF00B1012784
:1045A00002F036F800F0C0FD02A953201BF09AF982
:1045B000000601D502F0F3FD9DF8080000F00100AF
:1045C0008DF808006FB9B0B1012012F02BFB000686
:1045D00001D502F0E4FD11F031FE000601D502F034
:1045E000DEFD9DF8080030B1012012F01BFB000633
:1045F00001D502F0D4FD24F024FF4F464FEA0D0907
:104600003BF0A2FC2EF03AFA307800EB400007EBCA
:10461000C000C0688047000601D502F0C0FD3078B8
:1046200000EB400007EBC00040688047000601D562
:1046300002F0B5FD307800EB400007EBC000806869
:104640008047000601D502F0AAFD00202FF046FCAD
:10465000D8F800000C2805D005F0C0FE000601D5F2
:1046600002F09DFD207840071ED501202FF036FC7A
:10467000D0B9684606F0A5FA50B909F1020006F073
:10468000B1FA28B909F1040006F0BDFA000601D517
:1046900002F085FD46499DF804000870684607F061
:1046A0004FFC08B908F0B0FA35F097FE207810F00A
:1046B000B80F35D001202FF011FC000630D4A868C7
:1046C0003C49AA68121A8A42FBD32078000701D518
:1046D00011F05EFE2088010614D5810612D4C006B2
:1046E00013D411F0AFFE000601D502F058FD0020F2
:1046F00008F074FB000601D502F051FD208820F07F
:10470000810020802078C00601D507F0BBFB20780F
:10471000800605D501200AF071F8012012F082FA16
:1047200024F0F5FE000601D502F039FD30F02AFA3A
:10473000FFF7EEFD64E700000200001000C0072054
:1047400008C207208E9888818A802081809280907C
:104750008588209780918E820A8E8190809288929F
:1047600085919C20822096928E0A0A0A0A000000F7
:10477000008000400CC007208E9888818A80208F9E
:10478000808C9F9288208F840A0A0000000000100D
:10479000878D208D852082828584858D0A0A0A0A6C
:1047A0000A000000E0C8100076020010A8C107202F
:1047B0006D020010A086010000F00F01000900EB5F
:1047C000800001EB4000C0B270470A21B0FBF1F25B
:1047D00001FB1202B0FBF1F002EB0010C0B2704717
:1047E000002210B511460A2309E000BFB0FBF3F424
:1047F00003FB1404B0FBF3F08C402244091D002895
:10480000F4D1104610BD2DE9F047FA4DFA4EFB4F9A
:104810009046C3B15C1E0BD4DFF8E49364220023FE
:104820003CF0B2FC19F8023008F80430641EF5D5EB
:10483000084310D089202860042030607846386012
:104840008920BDE8F08788202860092030607846FC
:1048500038608820F5E700202860306078463860AE
:104860000020EEE710B500220BE0835C03F00F049C
:10487000092C03D803F0F003902B01D9002010BDC0
:10488000521C8A42F1D3012010BD2DE9FF4FD94CB3
:10489000D94DDA4E83B08246082A31D87AB3002047
:1048A000CDE9000001214FF0860B4FF0200E00BF34
:1048B0000AEB020313F8019C09F00F03092B14DC27
:1048C000A1FB03784FEAD37C00FB038301FB0C338D
:1048D000DDE9008C18EB07074CEB030CCDE9007CFD
:1048E0004FEA1919B9F1090F12DDC4F800B0784682
:1048F000C5F800E03060862007B0BDE8F08FFFE724
:104900008820206009202860784630608820F3E7FE
:104910004FF00A0CA1FB0C3800FB0C80002701FBB8
:104920000700A3FB091800FB09874FEAE97C03FB9A
:104930000C77DDE9008C18EB01014CEB070CCDE99D
:10494000001C4FF00A0CA3FB0C18002700FB0C8086
:1049500003FB0700521EABD10698DDE90023C1001E
:1049600001208840401EC117801A994107D2892032
:10497000206004202860784630608920BCE76946C2
:10498000069A04983DF026F80020206028607846BA
:1049900030600020B0E730B500B90120401E80B281
:1049A00040F2B553B0FBF3F2B0FBF3F403FB140099
:1049B0009206401C120E80B24FF4B77398420BD986
:1049C000521CD2B2A0F5B77003E0521CD2B2A0F2D2
:1049D0006D1080B29842F8D2202801D2012319E04C
:1049E0001F3880B2930701D01C2300E01D2398429A
:1049F00001D802230EE0C01A814D002380B2643535
:104A000003E0001B5B1C80B2DBB2EC5C8442F8D399
:104A1000DB1CDBB20A704B7088707649002008609E
:104A200075490860784675490860002030BD10B5AA
:104A3000027840F26D135A430A80714C43786E3409
:104A400034F813301A440A8083781A4493B20B80E6
:104A50000278940705D14078022802D803EB92002F
:104A600003E0012000EB9200184408806149002017
:104A7000086061490860784660490860002010BD00
:104A800010B581784FF0FF32C9B143780D2B18D2A1
:104A9000DFE803F017070D070A070A07070A070AE6
:104AA00007001F290BD80FE01E2908D80CE000785A
:104AB000800702D01C2902D806E01D2904D910461F
:104AC00010BD6FF0010010BD002010BD18B50288A8
:104AD0000024B2F5FA6F0ED9C2788DF802208278E0
:104AE0008DF801200078A0F5FA608DF80000684686
:104AF000FFF79DFF00E00C803E4804603E480460E4
:104B000078463E490860002018BD18B50C46694635
:104B1000FFF741FF9DF80200E0709DF80100A070D2
:104B20009DF80000334900F5FA60208000200860FD
:104B300031490860784631490860002018BDC0F34B
:104B40000722C0B2C0EB001002EB800008802949A8
:104B5000002008602849086078462849086000203D
:104B600070473C22B0FBF2F30B70B0FBF2F302FB98
:104B7000130048701F49002008601F4908607846EC
:104B80001E490860002070472DE9F04F884600213B
:104B9000184D194E194F82464FF08609B3EB420F5C
:104BA00016D301201FE000BFA2EB000B1AF80B4048
:104BB00004F00F04092C0BDCA3EB400E0EEB080CE9
:104BC00030348CF801401AF80B402409092C06DD1A
:104BD000C5F8009078463160386086208DE6303424
:104BE00008F80E40401C9042DED9012000EB420044
:104BF00030220CE008C007200CC0072010C007209E
:104C00005A370400A3EB000C401C08F80C20984213
:104C1000F8D9296078463160386000206DE62DE9CA
:104C2000F84F82468B4601204FF08609B54DB64EAF
:104C3000B64F00212BE000BFA2EB000E1AF80E4089
:104C4000303C092C14DC04F0FF0C00EBD074A3EB17
:104C5000640808EB0B04A4F10108CDF8008004F807
:104C600001CC0EEB0A0414F8014C303C092C07DD92
:104C7000C5F800907846316038608620BDE8F88F2E
:104C80004CEA0414DDF800C0801C8CF8004090420F
:104C9000D2DD521C9A4203DC9C1A0BF80410F8E790
:104CA00029607846316038600020E7E77CB50D4622
:104CB00001A9FFF770FE934C000601D520687CBD6A
:104CC0009DF8040000909DF805309DF8062090A105
:104CD00028463CF0F5FA8C490020206008607846B0
:104CE0008A49086000207CBD3C2310B5B0FBF3F27C
:104CF000B0FBF3F403FB1403D2B20A20B2FBF0F4CE
:104D000030340C70B2FBF0F400FB142230324A70E5
:104D10003A228A70B3FBF0F23032CA70B3FBF0F281
:104D200000FB123030300871764900200860764967
:104D30000860784675490860002010BD3C2310B516
:104D4000B0FBF3F2B0FBF3F403FB1400744BD2B2EC
:104D50009A5C0A70185C48706A49002008606A49C9
:104D60000860784669490860002010BD02784078E4
:104D700002F00F03120902EB820203EB420200F081
:104D80000F03000900EB8000D2B203EB4000C0B279
:104D9000C2EB021200EB820008805A490020086032
:104DA000594908607846594908600020704718B58D
:104DB0000C466946FFF7EFFD5249000601D5086829
:104DC00018BD9DF802205648825C22709DF8012093
:104DD000825C62709DF80020805CA07000200860FA
:104DE00049490860784649490860002018BD70B5F7
:104DF000044611B93CF078FD0146002220230DE065
:104E0000A05CF02801DB103802E0C02802DB40384B
:104E1000A05402E0802800DBA354521C8A42EFDB3E
:104E2000002070BD70B5044611B93CF05DFD01462F
:104E30000020202311E0225CF02A01DB23540BE048
:104E4000E02A01DB103206E0B02A01DB403A02E042
:104E5000802A01DB40322254401C8842EBDB0020D8
:104E600070BD10B5044600200146012202FA01F38C
:104E7000234205D0C1F1070302FA03F30343D8B27A
:104E8000491CC9B20829F1D310BD20280BD009282C
:104E900009D00A2807D00B2805D00C2803D00D28EC
:104EA00001D0002070470120704770B505460446C8
:104EB00000E0641C2078FFF7E8FF0028F9D12046C5
:104EC0003CF012FD421C214628463CF0C8FD284615
:104ED00070BD10B504463CF007FD011900E0491E05
:104EE000A14205D011F8010CFFF7CFFF0028F6D141
:104EF00000200870204610BD10B5FFF7D6FFBDE8B2
:104F00001040E6E708C007200CC0072010C00720AB
:104F1000253032752D253032752D25303275000043
:104F20005A370400F8B56A4E0D4607460222694614
:104F300030462BF079FA674C000615D4BDF8000016
:104F40002A4640F0804039462BF079FA00060BD40F
:104F5000BDF8000002222844ADF800006946304642
:104F60002BF06DFA000601D52068F8BD5A490020E3
:104F7000206008607846594908600020F8BD08B5EF
:104F80000020ADF800000222694651482BF057FA84
:104F900008BD014602224E482BF046BA2DE9F041E9
:104FA00088B00025022201A949482BF03DFA494C5E
:104FB00000064ED401202FF0DCF9000649D4484900
:104FC0000888420606D520F0400008801AF0FDFB54
:104FD00000063ED4002705A8059706F0FBFA000658
:104FE00037D406A8069706F006FB000631D43D49E3
:104FF0000220087004A962201AF074FC000628D46C
:1050000000264FF0200829E046F08040012203A945
:105010002BF00AFA9DF81000400714D49DF80C00FC
:1050200043280DD0F3280BD0F42809D0F5280AD155
:105030006D1CEDB28DF80C80022D04D1002502E02C
:105040000DB18DF80C80012103A82EF07EFF000623
:1050500003D5206808B0BDE8F081761CBDF80400D7
:105060008642D1D31C482760076078461B490860F8
:105070000020EFE710B5FFF782FF164C000604D4BE
:1050800005202FF076F9000601D5206810BD1249E1
:10509000002020600860784610490860002010BD9C
:1050A00010B50C4C18B1FFF76AFF000604D40120BC
:1050B0002FF05FF9000601D5206810BD06490020D9
:1050C00020600860784605490860002010BD000097
:1050D000780D002008C007200CC0072010C0072052
:1050E0000200001000000010F8B516460D460446F8
:1050F0008948012269462BF097F9000602D58748B6
:105100000068F8BD9DF80000204000D00120287004
:10511000022C06D08048401C022231462BF084F934
:10512000F8BD7D48C01CF7E710B59EB01BA80BF07A
:1051300022FF7A4C00064BD41AAA1CA90120FFF7C3
:10514000D3FF000644D49DF8700028B1BDF8680074
:10515000BDF86C10884209D97149002020600860B0
:1051600078467049086000201EB010BD02202EF065
:1051700091FF00062CD46C482FF0DCFB000627D4EE
:10518000694814302FF0D6FB000621D41AAA1CA9B6
:105190000220FFF7A9FF00061AD49DF87000C8B1DD
:1051A0001DA9BDF86800FFF7F6FB000610D49DF8B6
:1051B00074005D4900909DF875309DF87620263189
:1051C00001A83CF07DF801A82FF0B4FB000601D542
:1051D0002068C9E75548018841F00201018054491F
:1051E00002200870012011F01DFDBDE7FEB501A8E9
:1051F0000BF0C1FE494C000632D46A4602A90220D7
:10520000FFF772FF00062BD49DF80800444D454E71
:1052100028B1BDF80000BDF80410884206D900206E
:1052200020602860784630600020FEBD02202EF00D
:1052300031FF000614D43C482FF07CFB00060FD44D
:10524000394814302FF076FB000609D4374801881E
:1052500041F002010180012011F0E4FC000601D5BB
:105260002068FEBD91202060BE2028607846306016
:105270009120FEBD4FF0A0430146042218462BF0BA
:10528000D3B84FF0A0430146042218462BF0D7B8FC
:10529000F7B50446204882B00E460546012269460D
:1052A0002BF0C2F81D4F00060ED49DF800000EB181
:1052B000204300E0A0438DF8000001226946284603
:1052C0002BF0BDF8000602D5386805B0F0BD022C01
:1052D00006D01148401C022204A92BF0B0F8F4E7D4
:1052E0000D48C01CF7E738B50020012201460090A8
:1052F0001046FFF7CDFF094C000606D4012200211D
:105300000220FFF7C5FF000601D5206838BD6846BA
:10531000FFF7B7FF38BD00000400005008C00720A9
:105320000CC0072010C00720E23704000200001064
:10533000000000102DE9F04F99B0012400250C94D5
:10534000841A089571EB030404DA16461C460746D6
:105350000D4603E00C46064617461D4600218B46C7
:10536000059116E002220023304621463BF083FFE0
:1053700006460C4602220023384629463BF07BFFB6
:105380000D46012205991BEB020B41F10001074676
:105390000591F00701D1F807E4D001200021CDE903
:1053A000220124AA0846279482E84300711E64F172
:1053B0000000CDE91610CDE91475CDE9127500BFD6
:1053C000DDE9260180468946C00729D1DDE92201B1
:1053D000C20702D1249AD2070AD03A1845EB01003D
:1053E000CDE92220DDE9241071186041CDE92410B7
:1053F000DDE92201022200233BF03DFFCDE922013D
:10540000DDE92401022200233BF035FFCDE9240130
:1054100002220023404649463BF02DFFCDE92601FC
:10542000DDE91201C20704D0DDE92632181A8A41EB
:105430000BDA14A922A800F066FA16A924A800F035
:1054400062FA12A926A800F05EFADDE926011090A2
:105450000D91C007B4D00DF15008DDF85C2098E83C
:105460000B009E46DDE922C3E1469A46BCEB000CE8
:105470008B4106DBDDE9248CB8EB0E037CEB020CE0
:105480000DDA17EB090345EB0A0CCDE9223CDDE907
:10549000243CF31844EB0C0CCDE9243CE2E7B9EBD7
:1054A00000006AEB0103CDE922032598B8EB0E0159
:1054B00060EB0200CDE92410DDE91210109B0D9A7B
:1054C0005B1A62EB0002CDE926320023591A73EB16
:1054D0000002FFF675AF14E0DB1B60EB05004FF038
:1054E000000CB3EB0C0C70F1000C17DBCDE9223093
:1054F000901B61EB0401021E71F100020EDBCDE98D
:105500002401DDE92230D91B70EB050106DBDDE962
:105510002421B6EB020C74EB010CDDDB0021084604
:105520001AE000BFDDE922720C9B089DA3FB07C8AF
:1055300005FB078503FB0252CDE922C2DDE9267295
:10554000A3FB07C8089D491C05FB078503FB025206
:10555000CDE926C240F10000059AB1EB0B0370EBD8
:105560000202DFDBDDE9261081F00101014304D0F6
:105570004FF0FF3019B0BDE8F08FDDE92410711A4B
:1055800064EB00042898C0E900140020F2E72DE93C
:10559000FF5F9CB00020CDE90200CDE904009246F7
:1055A0002E9907AA0A20CDE90002994614AB0122E0
:1055B000491C1BF00CF900287DD114AB08AA195C1A
:1055C0000C0902F8104001F00F0402EB4001401CEE
:1055D0004C700828F3DB9DF82F70DFF840831146EC
:1055E0000E2000BF58F82740461C255CA45D801E95
:1055F0004E5D11F804C001F805C00E55F2D500202B
:1056000002EB400412F810106478904644EA01114D
:105610001954401C0828F3DB19460020079B0DE0B5
:105620001C1A0C440A5C14F8015D2E0146EA15159B
:105630000D54150145EA12122270401CB0EB530FB5
:10564000EED3082312A914A8079AFFF71EF9002821
:10565000B2D114A90EF080FB0028ADD10C2114A802
:10566000FFF700F900287DD0DDE91501CDE908013B
:10567000082208A90020131A0B440C5C13F8015DE2
:105680000D54401C1C70B0EB520FF4D300252C4677
:105690002F462E462846C3464FF00A0E1BF8001030
:1056A0007246303901EBC101B1FBF2F3B1FBFEFCF4
:1056B0000EFB1C1100E0AEE04FF0640CA5FB0C28C3
:1056C00001EB810103EB410104FB0C84002305FB8A
:1056D000034455185C4107910A23A7FB031C06FBF2
:1056E00003C3002207FB02321BF8003000F1010067
:1056F000303B5F1842EBE3760828CFDBDDE912018F
:10570000401B61EB0401864A0023CDE912013BF006
:105710003BFDCDE9122350EA01027CD01AAA069281
:10572000CDE90054DDE91C23FFF704FE002872D107
:10573000DDE91A50A7FB051206FB052207FB002432
:105740008346DDE91C23084621463BF01DFD144637
:105750009846DDE91223A2FB050603FB056302FB65
:105760000B3100E06CE0DDE91C233BF00DFD15463C
:105770009B4654EA080203D0DDE92A01012618E01D
:10578000012000211AE000BFDDE92A72A0FB073CDE
:1057900001FB07C100FB02111846BAEB000379EBCD
:1057A000010205D252464B463BF0EEFC104619462C
:1057B000761CF317371B73EB0803E5DBCDE91A0101
:1057C00080460C4655EA0B0003D0DDE92C0101268A
:1057D00017E00120002119E0DDE92C72A0FB073C55
:1057E00001FB07C100FB02111846BAEB000379EB7D
:1057F000010205D252464B463BF0C6FC1046194604
:10580000761CF317771B73EB0B03E5DBA0FB085348
:1058100001FB083100E012E000FB041152464B4648
:1058200028463BF0B1FC10461946DDE91C233BF04D
:10583000ABFCDDE9120150405940084303D0002081
:1058400020B0BDE8F09F0120FAE7F0B5411E85B019
:105850001E2932D2012404FA00F111F0D00F2CD00D
:10586000304FBE68401E2D4D8440083D69680C4293
:1058700029D1C1B204912C49002301EBC001D1E927
:105880000021CDE902212849284A383901EBC0011D
:10589000D1E90001CDE9000141F2E7001946FFF727
:1058A00076FE0028286801D0204300E0A04328604D
:1058B000B8681F49801B884202D3002005B0F0BDA4
:1058C00068682043686028682040F7E7411E1E2969
:1058D0000ED2012101FA00F212F0D00F08D0401EC2
:1058E00081400E48083842688A4342600120704770
:1058F0000020704700B501231846FFF7E7FF5B1C47
:105900001E2BF9DD00BD30B5D0E90023D1E90045FB
:10591000C0E90045C1E9002330BD00000C000010C3
:1059200000E1F505008000406038040063777B00EB
:10593000404B4C0038B50446684605F096F89DF893
:105940000000204038BD38B50446684605F08DF8A3
:10595000000602D5FD48006838BD9DF800002043D0
:105960008DF80000684605F077F838BD38B5044674
:10597000684605F07AF8000602D5F448006838BD9C
:105980009DF80000A0438DF80000684605F064F81B
:1059900038BD01B5FEF75AFC684605F07DF8FEF704
:1059A0006AFC08BD7CB5684605F080F8E74C000647
:1059B00038D49DF800000025082809D009280DD00A
:1059C000E348256005607846E249086000207CBD18
:1059D000684605F07CF8000624D40BE001A805F029
:1059E000B6FD00061ED49DF8040001281CD013202B
:1059F0008DF80000684605F04FF8000612D48DF8C7
:105A0000045001A805F099FD00060BD48DF8045050
:105A100001A805F088F8000604D4432019F0B7FD6A
:105A2000000603D520687CBD0220E1E7012011F0CB
:105A3000F9F87CBD2DE9F041002402202EF0B5FFDD
:105A4000C54DAE68C54F4FF4FA7811E0A868801BC9
:105A5000B8420DD3012024F00FFAC821404623F0AC
:105A6000D0FC012024F015FAAE68641C042C04DC80
:105A7000002024F0F3F90028E8D1012C06D0022CF4
:105A800007D0032C09D0042C11D10EE001F02EF91F
:105A90000DE002201FF03BFF09E0B14C0120207017
:105AA00003F013FC0020207001E026F0B1FABDE8FD
:105AB000F04101202EF079BF0EB568460EF0C7F810
:105AC00050B1932803D1A2480068062801D00E20C7
:105AD00000E01120FFF75DFF9C4800680EBD2DE936
:105AE000F34F002789B088460F703E4608A9384614
:105AF0000CF039FB954C000639D49DF82000DFF8F6
:105B00005092DFF850A2400607D407A804F0BDFF6A
:105B100000062CD49DF81C0068B3694609980DF066
:105B200088F8000623D40125EB4605A9284605F090
:105B3000C6FA00061BD405EB85015944052205A8C9
:105B4000491F3BF081FE00B101276D1CEDB2042D11
:105B5000EBD9C7B1834909980880452019F017FD92
:105B6000000604D4012011F05DF800060BD5206872
:105B70000BB0BDE8F08F26607946C9F800600020C0
:105B8000CAF80010F4E788F80070F4E72DE9F34F45
:105B900085B00320002408700E46274621460120C8
:105BA0000EF0A5F80106694802D5006807B0E0E7E5
:105BB0000168DFF89C91DFF89CA10025052913D02E
:105BC0008046EB46694601200EF06BF80006D8F8D7
:105BD0000000EBD405280DD005220BF10400059937
:105BE0003BF032FE18B103E0357005600DE0671C34
:105BF000641CE7E737B1BC4201D1022000E001207C
:105C0000307000E03570C8F800507946C9F800508F
:105C10000020CAF80010C9E730B5044685B000205E
:105C2000208002200EF079F8484D05280BD06946F7
:105C300002200EF036F800061ED4BDF800002188C0
:105C4000884200D9208001200EF067F8052802D094
:105C50006946012006E000200EF05FF805280BD011
:105C6000694600200EF01DF8000605D4BDF80000BE
:105C70002188884200D92080286805B030BD2DE9F0
:105C8000F04387B00646694600200EF065F82F4DB8
:105C9000000649D403A90B200CF065FA000643D492
:105CA0000C2203A968463BF0CFFD0227DFF8A08055
:105CB000DFF8A090002408B137703EE003A910205F
:105CC0000CF051FA00062FD4694604200EF044F877
:105CD000000629D4BDF80000BDF80C108842EBD1B5
:105CE000694606200CF03FFA00061DD4BDF80000FE
:105CF000BDF80C10401E8142DED169460E200CF02A
:105D000032FA000610D403A8FFF786FF00060BD472
:105D1000BDF80000BDF80C108842CDD369460020C4
:105D20000CF021FA000603D5286807B0BDE8F0831F
:105D30009DF800004007BFD534702C607946C8F844
:105D400000400020C9F80010EFE7000008C007205D
:105D50000CC0072010C0072000800040C0C62D00E6
:105D600014C00720E0010010FEB502A804F09EFE5A
:105D7000FC4C000637D49DF808000025FA4EFB4F76
:105D80001D2812D004F093FD08B104F012FD01A803
:105D900004F0D3FE000626D49DF8040028B10128A3
:105DA00009D002280BD003280ED025607846356034
:105DB00038600020FEBD012008F020FD01E009F060
:105DC0006BFB00060FD410E08DF80050684605F01C
:105DD000B4FB000607D4432019F0D9FB000602D417
:105DE0000BF090FFEDE72068FEBD012010F01AFFD8
:105DF000FEBD2DE9F0418AB0002606A80DF027FF70
:105E0000DFF86883D74CD84D932806D12868082836
:105E10006DD005286BD0062833D0002108460DF040
:105E200066FF000663D405A900200EF039FA0006CB
:105E30005DD4CF4F387858B1002101200DF057FFC5
:105E4000000654D405A901200EF02AFA00064ED40B
:105E500009A805F0CFFD000649D49DF8240038B309
:105E6000002101200DF043FF000640D469460120C7
:105E70000DF017FF05280DD00120397881430ED190
:105E80000AE00020206079462860C8F800100AB0B7
:105E9000BDE8F0810020F0E73978884308D09320EE
:105EA00020600820794628609320C8F80010EEE7AB
:105EB00002200DF032FF000619D4694602200DF0D1
:105EC000F0FE000613D4002102200DF010FF0006A2
:105ED0000DD405A902200EF0E3F92068932806D11D
:105EE0002868082803D1761CB6B2032EF1D32068A7
:105EF000CDE72DE9F04F97B012A804F0C6FD994CFC
:105F000000066ED413A805F075FD0006F9D4DFF87D
:105F100060821026DFF8549298F80000924D4FF0FE
:105F2000000A4FF0160B9227C0B107A80CF083F8B7
:105F300040F3C010401C8DF8300011D09DF82D00AA
:105F4000010637D59DF84C1099B38DF8006068466E
:105F500004F0A2FD032027602860ABE18DF830A09B
:105F60009DF84C0098F80010084217D028680328C4
:105F700011D004280FD08DF800B000BF9DF80000AC
:105F8000FFF707FD286809282BD9462019F0FFFAEA
:105F900030202760E0E78DF80060EFE7FFF7E4FED0
:105FA0008EE100BF8DF80000684604F075FD17B063
:105FB000DFE5FFE7C00603D50BF0A4FE0006A0D482
:105FC000FFF717FFDFF8AC8193280BD09DF82D0069
:105FD00000077DD50CA90AA8FFF7D8FD00285ED1DF
:105FE00014E06CE1FFF7C0FE00068AD40E208DF8A5
:105FF0000000684604F050FD000687D400215EA032
:106000002EF0B6FA614902200870C8E19DF8300010
:10601000022804D001287DD000287CD0E9E19DF839
:106020002D00400778D501A80BF083FF002874D11C
:1060300003E000BFFFF7ADFCD9E10FA904200DF08C
:106040008BFE0006F8D4BDF83C00BDF80410401CDF
:1060500081427CD19DF82D00800602D5FFF784FE99
:1060600011E015A804F069FD0006E5D49DF8540080
:10607000012815D0FFF778FE0006DDD412A804F041
:1060800004FD0006D8D4BDF8040014A9FFF727FDCD
:1060900020688228D0D0922863D093287AD133E127
:1060A00010A804F08EFD0006C6D410AEB01C04F09B
:1060B00099FD0006C0D4301D04F0A5FD0006BBD438
:1060C00033499DF844000870684604F0EFFC00E096
:1060D0006CE10006B0D49DF80000042809D0052822
:1060E0003AD01D282BD0FFF73FFE684604F0DEFCB7
:1060F000C7E704F0DCFB30B104F05BFB10A805F04F
:106100001FFF000698D4012600270EA9304604F090
:106110009FFE03E099E0A3E08EE0F1E000068BD45F
:106120000E98761CF6B20744102EEED93FB11D2012
:106130008DF80000684604F0AFFC000695D4B8F86E
:10614000001010A841F00401A8F8001000E022E0BF
:1061500005F0F6FE000688D406F056FD000684D44D
:10616000C3E753E008C007200CC0072010C0072079
:1061700008440000020000108E9888818A80208FD9
:10618000808C9F9288208F840A0A000000000010F3
:106190006D0200103DE0FFF7E7FD000684D49DF896
:1061A0002D009DF8481000F04000491E084306D11C
:1061B000BDF83C10BDF80400891C884214D00BF0D7
:1061C000A1FD00067BD414208DF80000684604F081
:1061D00063FC000673D44E2019F0D9F900066ED482
:1061E000012010F01FFDE2E6401E80B214A9FFF767
:1061F00076FC2068822862D0922802D0932803D1AE
:1062000082E0286808287DD11320CBE6286808287A
:1062100078D19DF8500008B11520C3E6684604F017
:1062200045FC00064BD49DF800001D2869D047E0CE
:106230000120B7E60220B5E68DF80060684604F05C
:106240002BFC00063BD4332007E08DF80060684645
:1062500004F022FC000632D4412019F098F99EE0A7
:10626000FFF782FD00062AD49DF82D004FF031067D
:1062700010F0600F29D09DF84C0008B38DF800B0E5
:10628000684604F009FC000619D4422019F07FF991
:106290006946532019F026FB000610D49DF8000033
:1062A00010F002008DF8000002D0012010F0BAFCBE
:1062B00027602E6079469220C9F8001077E680E0CA
:1062C0009DF848000028B5D0B2E701A80BF031FED8
:1062D000B0B914A8FFF7D3FC822872D0922811D04D
:1062E000932811D09DF8500080B1022836D0882024
:1062F00020600220794628608820C9F8001056E600
:1063000000E076E00F2095E60E2093E610F0C4F949
:10631000012010F087FC5E2019F039F90CF066FAC4
:10632000000664D4FE4D0121FD4810F004FD000676
:106330000AD5FDF78BFF0BF0E5FC000657D4FDF7FF
:106340009AFF2078000652D40CF08CFA00064ED446
:1063500095F800010028E6D1182019E09DF84C00BE
:1063600080B18DF800B0684604F096FB00063ED47C
:10637000422019F00CF9B8F8001041F00201A8F819
:10638000001092E79DF8480008B1012000E00220CB
:106390008DF80000684604F07FFB000627D4B8F8AB
:1063A000001041F00201A8F8001019E7FFF7DCFC2B
:1063B0009DF84C0000289DF848000DD010B10C202D
:1063C00001E014E00D208DF80000684604F064FB45
:1063D00000060CD4402040E708B1012000E0022074
:1063E0008DF80000684604F057FB000601D52068D0
:1063F000DDE5C4F800A07946C5F800A00020C9F882
:106400000010D4E510B5C748C74C86B0007820B15D
:106410000420FFF71AFA40B123E00620FFF715FA2F
:10642000F8B90420FFF711FAD8B90120FFF70DFAE7
:10643000B8B9372019F0ABF802A9532019F052FA75
:10644000000639D49DF8080010F002008DF808000D
:1064500007D0B648018841F002010180012010F008
:10646000E1FB012004A9CDE90001024603AB0421B0
:1064700009201AF0ACF900061ED49DF80C0005287E
:106480001DD1AB480079C00704D00720FFF7DDF924
:1064900068B114E066200BE0682019F078F8000677
:1064A0000AD4012010F0BEFB000605D407E06520E9
:1064B00019F06DF80006EFD5206806B010BD9D49B3
:1064C00000202060086078469B4908600020F4E7BF
:1064D00038B5684604F0EAFA934C000629D4974D83
:1064E0002878752827D00220FFF724FA70B17B2086
:1064F0002870684604F0E1FA00061AD41C208DF8D2
:106500000000684604F0C8FA000612D40120FFF724
:1065100011FA80B151202870684604F0CEFA0006C6
:1065200007D417208DF80000684604F0B5FA00067D
:1065300001D5206838BD9DF800000F2801D17E20CC
:1065400028707C4900202060086078467A490860FD
:10655000002038BD2DE9FC418046032024F091F94C
:10656000744E754F704C002530B9B8F1000F03D050
:106570000420FFF7DFF9E8B36946532019F0B2F9B8
:106580009DF8000010F002008DF8000002D00120FC
:1065900010F048FB3D2018F0FAFF9DF8000010B104
:1065A000012010F03FFB654975200870684604F033
:1065B0007DFA00061BD4684604F090FA000616D453
:1065C00001A804F062FA000611D49DF8040008B195
:1065D000192000E01A208DF80000684604F05CFAEB
:1065E000000604D40420FFF7AEF9000603D52068A6
:1065F000BDE8FC8106E08220206078463560386086
:106600008220F5E725607846356038600020EFE7A6
:106610002DE9F0438BB000273E4607A804F046FA68
:10662000414C00067AD49DF81C00DFF80881DFF8A1
:1066300008910025022803D0192801D01A286ED10C
:1066400003A9352019F04EF9000667D49DF80E0015
:1066500000F00F01000900EB800001EB400000F5A5
:10666000FA60ADF814009DF80D0000F00F0100096C
:1066700000EB800001EB40008DF816009DF80C0047
:1066800000F00F01000900EB800001EB40008DF8E5
:10669000170009A905A8FEF719FA03A9362019F071
:1066A00021F900063AD49DF80E0000F00F01000910
:1066B00000EB800001EB400000F5FA60ADF814003B
:1066C0009DF80D0000F00F01000900EB800001EBC8
:1066D00040008DF816009DF80C0000F00F01000935
:1066E00000EB800001EB40008DF8170008A905A819
:1066F000FEF7ECF968460AF03EFC00067AD404A8DE
:1067000024F0FBF8000675D4BDF8240020B3BDF8D2
:106710000010814220D39DF8100011E06AE06DE086
:106720006CC507200844000008C0072002000010C4
:1067300060DA07200CC0072010C007206C02001090
:10674000172809D2012703AB3522394602200395C9
:106750001AF083F800064DD4BDF8200088B1BDF8CA
:10676000001081420DD39DF8100050B1012603ABFB
:1067700036223146022003951AF06FF8000639D40C
:10678000E7BB56EA070045D006A9342019F0AAF85D
:1067900000062FD49DF81800012826D0022804D026
:1067A000032837D14D497D20087006A9532019F0E0
:1067B00099F800061ED49DF8180010F002008DF81C
:1067C000180004D0012010F02DFA000612D40EB1EA
:1067D000482000E0472018F0DAFE9DF8180020B1AC
:1067E000012010F01FFA000604D404A824F085F854
:1067F000000604D520680BB0BDE8F0830AE09DF8E0
:1068000010000EB1401E00E0401C8DF8100004A8DE
:1068100024F0D8F825607946C8F800500020C9F85F
:106820000010E8E738B50546684604F03FF92C4CFF
:10683000000604D4284604F028F9000601D5206893
:1068400038BD9DF8001006290FD008DC01290CD0B6
:1068500003290AD0042908D0052908D105E0072911
:1068600003D0132901D0152901D1012028701D4919
:1068700000202060086078461B490860002038BD71
:1068800038B50546684604F022F9154C000618D4C0
:106890009DF80010072916D006DC0DD2DFE801F0C4
:1068A0000C130C13131313000E290CD013290AD048
:1068B000152908D01B2906D0284604F0E6F8000662
:1068C00003D5206838BD01202870064900202060CB
:1068D0000860784604490860002038BD6C0200104A
:1068E00008C007200CC0072010C0072010B58AB0D0
:1068F00005A82DF078FFD24C000637D468462DF05D
:1069000072FF000632D40220ADF80A00ADF8020092
:10691000ADF804000A20ADF80600002168462DF00D
:10692000B9FC000622D40021C6A02DF021FE0006ED
:106930001CD40021C6A02DF01BFE000616D4012198
:1069400008462DF03DFC000610D40021C1A02DF01A
:106950000FFE00060AD4002105A82DF09BFC0006BE
:1069600004D401202DF096FB000602D520680AB061
:1069700010BD2DF0C9FFFAE72DE9F04F834699B01D
:106980000D4608462DF0B2FBAD4C00067DD45846AE
:106990002DF04DFC00067DD42B465A46B4A1684626
:1069A0003AF08EFC002168462DF0E2FD000671D41D
:1069B000B5482A22C589684629463BF005F90A20D0
:1069C0000DF805000DF101014FF0000905F80190E7
:1069D000494668462DF0CCFD00065BD42EF0AFF89A
:1069E000DFF8A8A20646DFF8A8829AF8000002287D
:1069F00005D000EB400108EBC10040688047A54F7F
:106A0000BD680021A4482DF0B3FD000642D400214A
:106A1000A1482DF0ADFD00063CD400218CA02DF046
:106A2000A7FD2EF08CF8861BB868411B4FF47A70D6
:106A3000B1FBF0F59AF80000022805D000EB400108
:106A400008EBC1004068804706EB4600C0EBC6106B
:106A500005EBC000401EB0FBF5F7ABF101002EF0D6
:106A600072F84FF47A714E436843B6FBF0F2FF1DA3
:106A7000FB088AA168463AF023FC68462DF05AFFCD
:106A8000000607D400218DA000E003E02DF070FD8A
:106A9000000603D5206819B0BDE8F08F8849C4F816
:106AA00000907846C1F80090864908600020F2E71F
:106AB00070B58AB0064605A82DF095FE604D00061B
:106AC0003CD468462DF08FFE000637D40121ADF886
:106AD0000210ADF80060BDF81400ADF80410ADF878
:106AE0000A10ADF80610401E2EF034F8BDF8221042
:106AF00000FB01F4BDF80000401E2EF02BF894FBC3
:106B0000F0F0ADF80E00012168462DF0C3FB000641
:106B100014D40424032E02D10D2C00D10E242146BE
:106B20003046FFF729FF000608D4E41C0F2CF1D3F0
:106B3000002105A82DF0AEFB000602D528680AB09A
:106B400070BD5F4900202860086078465D49086094
:106B50000020F4E710B500202DF069FB384C00064A
:106B60003AD406202DF0C2FA000635D400213FA009
:106B70002DF0FEFC00062FD4012108462DF020FB4D
:106B8000000629D4002150A02DF0F2FC000623D4E9
:106B9000022101202DF014FB00061DD400214AA083
:106BA0002DF0E6FC000617D4012102202DF008FB91
:106BB000000611D4002144A02DF0DAFC00060BD40D
:106BC000022108462DF0FCFA000605D400213EA063
:106BD0002DF0CEFC000601D5206810BD38490020FC
:106BE00020600860784637490860002010BD10B565
:106BF00001202DF04FFA124C000619D4012108464D
:106C00002DF0DEFA000613D405202DF06FFA0006F1
:106C10000ED4214B1822A533642100202DF06CFCEA
:106C2000000605D400212BA02DF0A2FC000601D502
:106C3000206810BDBDE8104001202DF0A6BB00006B
:106C400008C00720465072696E742D313100000073
:106C50000A00000084A5ACAEADE1E2E0A0E6A8AE7B
:106C6000ADADA0EF20AFA5E7A0E2EC0A200A00003E
:106C7000200A98908894922025752C209F908A8EC7
:106C800091929C2025750A005CE207207602001094
:106C9000A8C107200080004038390400D1EAEEF096
:106CA000EEF1F2FC3A20257520D1D2D02FD1202848
:106CB000257520CCCC2FD1290A0000000A200A001B
:106CC0000CC0072010C007203132352054454354F2
:106CD0000A00000020342036303232343220303086
:106CE000313733370A200A200A00000070B5ACB0F3
:106CF00002202DF0CFF9A44D00067BD402210846D6
:106D00002DF05EFA0006F8D4A0A2A3A102A83AF0E2
:106D1000D7FA002102A82DF02BFC012108462DF006
:106D20004FFA0006E9D49DA02DF004FE01202DF0BD
:106D3000B1F996A298A102A83AF0C2FA002102A8DD
:106D40002DF016FC02A801F021FC02A801F057F872
:106D5000002102A800F095FF02A800F0D5FF02A8CC
:106D600001F015FC02A801F095FC20221DA9904815
:106D700029F05AFB02AA8DA18EA000F00AFF02A8FA
:106D80002DF0D8FD8EA125A81E9A3AF099FA02AAF4
:106D900025A98DA000F0FDFE02A82DF0CBFD88A155
:106DA00025A81F9A3AF08CFA02AA25A98BA000F018
:106DB000F0FE02A82DF0BEFD81A125A8229A3AF08E
:106DC0007FFA02AA25A989A000F0E3FE02A82DF00F
:106DD000B1FD7BA125A8239A3AF072FA02AA25A94F
:106DE00087A000F0D6FE02A82DF0A4FD68462CF086
:106DF0000AFF00E0BCE086A125A8009A3AF060FAFC
:106E000002AA25A984A000F0C4FE02A82DF092FDDC
:106E100002A801F03FF885A02DF08CFD29A829F0EB
:106E2000FCFD2998012832D0032834D0042830D022
:106E3000072832D080A102AA81A000F0AAFE02A8F1
:106E40002DF078FD824C202202A8E1893AF0BCFEA8
:106E50000E2280A102A83AF048FE2AA90120CDE91D
:106E6000000101461BAB0222092019F0B0FC00060C
:106E70007ED49DF86C3001A80A22411E0A2B52D202
:106E8000DFE803F0510D1151181C20282C4D75A17D
:106E9000D1E776A1CFE776A1CDE778A1CBE7E1896D
:106EA000084478A102E0E189084478A109680160FA
:106EB00002711DE0E189084476A1F7E7E089084402
:106EC00076A102E0E089084476A10A680260898818
:106ED00081800DE0E089084474A1F6E7E1890DF1B5
:106EE0000200084473A10B68036089888180827165
:106EF00002A82DF01FFD02AA70A172A000F049FEA9
:106F000002A82DF017FD744800788DF86C0070B160
:106F100001280FD0022802AA30D024A10CE0E08979
:106F200008446EA1D1E7E18908446EA1BEE702AA38
:106F30006EA101E002AA6FA170A000F02AFE02A8D3
:106F40002DF0F8FC29F0BFFA01202DF01EFA552093
:106F500018F01DFB1CA803F001FE00060BD41CA8B2
:106F600003F0C4F9000606D41CA803F0EDFD00E010
:106F700001E0000604D528682CB070BD64A1DBE7F1
:106F800001200FF04FFEF7E708C007204650726956
:106F90006E742D313100000025730A00C8CDD4CEA7
:106FA000D0CCC0D6C8DF20CE20CFC40A000000005D
:106FB00008000020CDC0D0C0C1CED2CAC0000000A1
:106FC0002531306C7500000020C4C2C8C3C0D2C5D2
:106FD000CBDC2CC2D1C5C3CE0000000020C3CECB79
:106FE000CEC2CAC02CC2D1C5C3CE000020C4C2C804
:106FF000C3C0D2C5CBDC2CD1C1D0CED100000000A3
:1070000020C3CECBCEC2CAC02CD1C1D0CED10000BD
:107010002532644300000000D2C5CCCFC5D0C0D219
:10702000D3D0C020C3CECBCEC2CAC800D1C2DFC726
:10703000DC20D120CFCA0A00556E6B6E6F776E00D0
:1070400020CAC0CDC0CB20CEC1CCC5CDC000000071
:107050005CE2072020D1CACED0CED1D2DC20C1DB69
:10706000CBC0000052532D32333200005553420042
:10707000424C5545544F4F5448000000574946492B
:1070800000000000313230300A000000323430306D
:107090000A000000393630300A0000003134343044
:1070A000300A000033383430300A000035373630CB
:1070B000300A00003131353230300A003438303097
:1070C0000000000020D1CACED0CED1D2DC20C2D068
:1070D000C5CCC5CDCDCE000076020010313932309E
:1070E000300A0000343830300A000000C0D2CECB65
:1070F00000000000D8D2D0C8D500000020CFD0CEEC
:10710000D2CECACECB20CEC1CCC5CDC000000000AF
:10711000C0D2CECB20CDCEC2DBC900002DE9F843D2
:10712000F34DF44FDFF8D083002440B969460120C5
:1071300022F070FE000617D40098C0071DD0EF4E55
:107140003088800506D50122002110460AF060FB38
:10715000000609D43078000609D501221146002026
:107160000AF056FB000602D52868BDE8F88330888F
:1071700010F4207F08D1800406D42C6079463C604E
:107180000020C8F80010F0E74FF4FA74FA21204606
:1071900022F037F92146002022F033F9F6E72DE9F5
:1071A000F04F95B04FF00009D14FDFF854A3CDF860
:1071B0004890DFF840B33B68CAF80030DBF80000C5
:1071C000CE49DFF83483CAF804007F26CD4C098805
:1071D000D8F800204D46892B10D010DC812BFBD035
:1071E00006DC062B77D2DFE803F0F7F776F7F7F740
:1071F000822B71D0862BEFD0872B6CD1ECE0932BB8
:1072000014D00ADCA3F18A010929EBD2DFE801F0EE
:10721000E463636363FBE4E43E00962B70D0A12B30
:10722000ECD0A22BFAD0A32BE7D12CE10A2819D05D
:1072300008DC052816D00628E0D0082812D0092836
:1072400006D10FE00B280DD0802819D0812817D047
:107250000090AD4901A83AF033F8002101A82DF0C3
:1072600087F903E009B9A9A00DE00425AF4926700C
:10727000022008704B2018F08AF9FF2D3CD1EAE07B
:107280000029F2D1AAA00FF04AF8EEE7FCF7DEFFE2
:1072900013A804F0AFFBFCF7EEFF9DF84C000028AC
:1072A0007DD0DBF8000008282BD00ADC19D2DFE8FB
:1072B00000F018282828282828283860CBF8000053
:1072C0003FE02A2819D008DC09281AD0202814D039
:1072D000282806D111E0A8E040E0302838D0312835
:1072E00036D000219CA02DF043F926708F49022052
:1072F00008704B2018F04BF9A6E00EF0D2FF2AE000
:10730000BFE00EF0CEFF8949CAF800900220CAF80B
:10731000049008704C4612A9532018F0E3FA0006B6
:107320006FD4129810F00200129007D09148018893
:1073300041F00201018001200FF074FC3C60CBF8A9
:10734000004079460020C8F8001015B0BDE8F08F65
:1073500003202DF010FB7E202070C7E7252864D283
:10736000DFE800F0631E1E2B2B25631329634032D8
:107370003A6340636336633A3A6363631E2B343483
:10738000633A63633A5C5C3A2B0031B96749022087
:10739000087000215DA02DF0EBF8042553E06EE0AD
:1073A00019B9002174A02DF0E3F802254BE000216B
:1073B0007AA02DF0DDF8012545E019B9002180A063
:1073C0002DF0D6F803253EE00A253CE009253AE0F9
:1073D000834800780228F5D0CAF800904846CAF8D9
:1073E00004906AE714A9622018F07CFA000608D419
:1073F0009DF850000007EFD5684603F0CEFC00066C
:1074000002D53868A1E71AE09DF800000028E3D013
:107410005848018841F080010180DDE719B9002159
:1074200070A02DF0A5F808250DE00090364901A8C0
:1074300039F046FF002101A82DF09AF803E0032857
:107440001DD007281BD026706D00FF2D03D012A978
:10745000284600F01DF80020FFF760FE694C6A4ED8
:10746000207800EB400006EBC000406880472078A1
:1074700000EB400006EBC00080688047E5E7484627
:107480001BE70428FBD079461846C8F800105CE7D3
:1074900070B5040008680D4605D0611E88420FD102
:1074A0004FF4FA6110E05949584A363A31F9101050
:1074B00032F9100021F057FF002818D11B240CE0EE
:1074C000C00703D04FF4FA71002002E0C8214FF446
:1074D000167021F048FF002809D1012022F0F7FCA6
:1074E0002868401C2860A04201D10020286070BD9F
:1074F00008C007200CC0072010C0072000C00720CC
:1075000018C007206C020010D02205008EE8A8A148
:10751000AAA020AFA0ACEFE2A8208F84200A0A0A1C
:107520000A0A0A0A0A0A0A0A0A0A000000000010E7
:1075300091A1AEA920AEA1ACA5ADA020E120AFA045
:10754000ACEFE2ECEE208F84200A0A0A0A0A0A0A4B
:107550000A0A0A0A0A0A00008EE8A8A1AAA0209D29
:107560008A8B870A0A0A0A0A0A0A0A0A0A0A0A0AFD
:10757000000000000200001091A1AEA920AEA1AC55
:10758000A5ADA020E1209D918F87930A0A0A0A0ADF
:107590000A0A0A0A0A0A0A0A000000008220E7A072
:1075A000E1A0E520ADA5A2A5E0ADAEA520A2E0A595
:1075B000ACEF0A0A0A0A0A0A0A0A0A0A0A0A0A00AE
:1075C00091A1AEA920AEA1ACA5ADA020E1208E87EF
:1075D000930A0A0A0A0A0A0A0A0A0A0A0A0A000096
:1075E00008C2072091A1AEA920AEA1ACA5ADA020F4
:1075F000E1208F8F87930A0A0A0A0A0A0A0A0A0AEE
:107600000A0A0A0076020010A8C107202C3A0400DA
:1076100070B5F04C0546616819B101F8010B616065
:1076200070BD0A2D02D10D20FFF7F2FF216800295D
:10763000F6D02846BDE87040084710B5044602E081
:10764000641CFFF7E5FF20780028F9D110BD70B564
:10765000E04D0C462E68286002E0641CFFF7D8FF5E
:1076600020780028F9D12E6070BD2DE9FF5F8A4691
:107670000546E94615F8010B00286FD0252802D0F1
:10768000FFF7C6FFF6E715F8010B4FF000083028AA
:1076900002D02D2802D005E0012000E00220804623
:1076A00015F8010B002606E006EB860100EB41060B
:1076B00015F8010B303EA0F130010929F4D96C28EE
:1076C00001D04C2803D115F8010B48F0040800281C
:1076D00044D00246612801D3203AD2B24F2A3ED08C
:1076E00006DC422A38D0432A33D0442AC8D138E0B5
:1076F000532A0FD0552A34D0582AC1D15FF0100335
:107700005FEA487101D4442A2DD05AF8041B442A58
:107710002BD02FE05AF8047B002400E0641C385D75
:107720000028FBD102E02020FFF772FF5FEA88709B
:1077300003D42046641CB042F5D33846FFF77DFFE2
:1077400002E02020FFF764FF2046641CB04291D283
:10775000F7E71AF8040B93E70223D1E74EE008237A
:10776000CEE70A23CCE75AF8041B002902DA494283
:1077700048F0080800244F46B1FBF3F203FB121255
:10778000B1FBF3F1D2B2092A05D9782816D04FF00F
:10779000070C6244D2B230323A55641C09B1102C45
:1077A000EAD35FEA087003D52D2009F80400641CB1
:1077B00027465FEAC87004D0302003E04FF0270C62
:1077C000E7E72020834602E05846FFF721FF5FEA03
:1077D000887003D438467F1CB042F5D3641E19F874
:1077E0000400FFF715FF002CF8D102E02020FFF77E
:1077F0000FFF38467F1CB042A9D2F7E7BDE8FF9FD4
:107800000FB410B503A90298FFF72FFF10BC5DF865
:1078100014FB7049486070476E480021426811703F
:10782000416070470FB470B56A4C054606A96060A8
:107830000598FFF71AFF606800210170401B616026
:1078400070BC5DF814FB0FB470B5624C06A92568D6
:1078500020600598FFF709FF2560F1E770B5044641
:107860001E4615465CA0FFF7CBFF012E04D0022E6A
:107870001DD0042E29D122E02646002404E0315DEB
:1078800057A0FFF7BDFF641CAC42F8DB2020FFF7D8
:10789000BFFE002408E0305DA0F120015E2900D980
:1078A0002E20FFF7B5FE641CAC42F4DB0DE034F88B
:1078B000021B4DA0FFF7A4FF6D1EF8D105E002CC1E
:1078C0004BA0FFF79DFF6D1EF9D1BDE870400A2067
:1078D0009EE62DE9F0413F4E0746B068002817D0DC
:1078E00000244D1EB0688047002811D00D280CD010
:1078F000082806D02028F5DBAC42F3DA3855641CA2
:10790000F0E7002CEED0641EECE700203855012093
:10791000BDE8F08170B52F4C0B461146A568A060FC
:107920001846FFF7D6FFA56070BD30B500250D6085
:10793000036801E05B1C03601A78202AFAD02D2A24
:1079400003D101255A1C02605A78302A06D0A2F1D0
:1079500030030A2B29D20A2300242EE00468641C79
:1079600004602278622A07D0782A03D0202A08D817
:10797000012030BD102300E00223641C0460227843
:10798000EAE7A2F130030A2B0FD20823E4E7612AC9
:1079900001D3203AD2B2303AD2B2112A03D3D21F45
:1079A000D2B2092A01D99A4201D3002030BD04FB8A
:1079B00003240268521C02601278202AE7D805B11D
:1079C00064420C60D4E72038DF2801D801207047DA
:1079D00000207047340000102530386C583A000001
:1079E0002025303258000000202530345800000097
:1079F000202530384C58000030B502464FF6FF7352
:107A000018464B4C08E000BF12F8015B85EA1025D0
:107A1000655D85EA002080B2491E89B2F4D25840E3
:107A200030BD10B541F221033CE000BF11F8014B1D
:107A300080EA0420040402D583EA400000E040000C
:107A400080B2040402D583EA400000E0400080B226
:107A5000040402D583EA400000E0400080B2040440
:107A600002D583EA400000E0400080B2040402D561
:107A700083EA400000E0400080B2040402D583EABB
:107A8000400000E0400080B2040402D583EA4000D8
:107A900000E0400080B2040402D583EA400000E028
:107AA000400080B2521E92B2C0D210BD30B5034623
:107AB000002002461F4C0AE013F8015B521C85EAC5
:107AC000102592B234F8155085EA002080B28A421F
:107AD000F2D330BD41400020CA0700D05E208A07A3
:107AE00001D580F0BC004A0701D580F061000A078B
:107AF00001D580F0C200CA0601D580F09D008A063B
:107B000001D580F023004A0601D580F04600090621
:107B100001D580F08C007047024610B5FF20002987
:107B200005D0054B545C4440491E185DFAD110BD88
:107B3000623A0400623B0400400000102DE9F0416D
:107B400080462CF0F7FE002821D04FF496764FF4B3
:107B5000FA77FE4CFE4D012022F0B9F93146384645
:107B600021F04FFC012022F0B2F9A068A168091AA7
:107B7000A942FBD32CF0C8FE0028ECD10021F5A0CF
:107B80002CF0F6FC4046BDE8F0412CF0D3BEBDE839
:107B9000F0812DE9F05F14468B46824639F0A4FE51
:107BA0008146584639F0A0FEEB4D064609EB06002B
:107BB000E9890A274FF00008884217D22022204680
:107BC0003AF002F84A465146204639F003FFE88968
:107BD0003246801B2044594639F0FCFEE889275480
:107BE000E989641C01F80480BDE8F09F012000EBE6
:107BF00041012022204639F0E7FF4A4651462046FF
:107C000039F0E8FEE889324659462754E889C6EB40
:107C100040002044401C39F0DDFEE88904EB4000C0
:107C20004770E98904EB410181F80280DCE710B577
:107C3000044686B001202CF02DFA05A904A80BF00B
:107C400060FBC6A0FFF77AFF0498642148430599BA
:107C500090FBF1F2C6A1684639F032FB2246694634
:107C6000C5A0FFF796FF2046FFF768FFC649002032
:107C70000860C64908607846C549086006B000201B
:107C800010BD30B585B00546002004900C4604A810
:107C900021F027FDFCF7DAFA0499642091FBF0F259
:107CA00000FB12120A2392FBF3F391FBF0F2B9A14D
:107CB000684639F005FB2A466946B9A0FFF769FF17
:107CC0002846FFF73BFFFCF7D6FAB048006814B12E
:107CD00011280ED010E011282A4608D0B7A1A5A07F
:107CE000FFF757FF2846FFF729FF05B030BDB5A1C4
:107CF000F5E72068401C2060B4A16846226839F08E
:107D0000DFFA2A466946EAE77FB506462BF091FF7F
:107D10000028FBD18D4988688D4A8B681B1A9342D5
:107D2000FBD3032021F0B7FC044621F0FAFC02004B
:107D3000A94D4FF47A704FF0640132D041F2707364
:107D40009C4203DA3246A5A1A5A052E094FBF0F2D2
:107D500000FB124292FBF1F394FBF0F28DA1684616
:107D600039F0AEFA324669469DA0FFF712FF304661
:107D7000FFF7E4FE984A00200A212C3A01E0401C5B
:107D8000491E52F82030A34201DB0A28F7DB55F8E0
:107D9000212077A1684639F093FA3246694696A0C9
:107DA00027E094FBF0F200FB124292FBF1F394FB0C
:107DB000F0F278A1684639F083FA3246694688A025
:107DC000FFF7E7FE3046FFF7B9FE83490020583938
:107DD00000E0401C51F82020A24201DC0A28F8DB18
:107DE00055F8202062A1684639F06AFA32466946A1
:107DF00085A0FFF7CEFE3046FFF7A0FE7FBD70B531
:107E0000044688B001202CF045F9534E0125284640
:107E1000FDF75CFD002838D02A467DA1204639F0C8
:107E20004FFA2046FFF78AFEF1892022204639F0DA
:107E3000CBFE07A91420CDE9000102AB012229469F
:107E40000A2018F0C4FC2846FDF7FFFC50B1079A41
:107E5000611C530002A8FCF797FEF189201F08441B
:107E60006FA109E0079858224100601C39F0ACFE70
:107E7000F189A01F08446CA139F022FAF289601C34
:107E8000002111542046FFF759FE6D1C1E2DBEDB4C
:107E900008B070BD10B504468CB001202CF0FAF883
:107EA00063A0FFF74BFE65490A88A2F5194099388F
:107EB0002ED063A1684639F003FA2246694662A0D3
:107EC000FFF767FE2046FFF739FE09A90AA80CF064
:107ED000C2F9BDF824205AA1684639F0F1F92246CA
:107EE00069465AA0FFF755FE2046FFF727FE40F2ED
:107EF000044053A10288684639F0E2F922466946F7
:107F000053A0FFF746FE2046FFF718FE0CB010BD49
:107F100050A253A1684639F0D3F9224669464AA0D7
:107F2000FFF737FE2046FFF709FE4E4A4CA1684690
:107F300039F0C6F9224669464BA0FFF72AFE2046D3
:107F4000FFF7FCFD4A4A46A1684693E000800040E6
:107F500020A107000A0000005CE20720CFC0CCDFB0
:107F6000D2DC20C1D3D4C5D0C020CACB0A000000C7
:107F70002575252500000000C8D1CFCECBDCC7CEAB
:107F8000C2C0CDCE0000000008C007200CC00720F2
:107F900010C0072025752E25303175C20000000065
:107FA000C1C0D2C0D0C5DF20D7C0D1CEC228322EAA
:107FB00032202D20332E332900000000CDCED0CC2E
:107FC00000000000CDC5CDCED0CC000025303464FB
:107FD00020CED8C8C1CECA0098010010CDC5D200AD
:107FE000C0CACAD3CCD3CBDFD2CED028362E3620CF
:107FF0002D20382E3429000020C7C0D0DFC6C0C5D0
:10800000D2D1DF2E2E2E000020C7C0D0DFC400004A
:10801000CACEC420C7C0D9C8D2DB2025750A00004B
:10802000CDCED0CC0A000000CDC5CDCED0CC0A003C
:10803000494420D1C5D0C8C83A0A00000444000011
:10804000253034750000000020310000203200008F
:1080500020330000CED2CBC0C4CED7CDC0DF0000CD
:10806000257300001044000020C4E0F2E03A000054
:108070002044000039F024F922466946FEA01FE79B
:1080800010B50420FDF75FFC0106FD4801D500682E
:1080900010BD00210160FB4801607846FA49086084
:1080A000002010BDF948002100F8081FFF210176CB
:1080B000017780F820107047F0B5074687B00C466E
:1080C0000026032022F0DDFBD0B101263046FFF769
:1080D000D7FF002845D18DF800008DF801008DF8FC
:1080E000020040F2DA70ADF8140001208DF816009D
:1080F0008DF8170005A822F086FC684622F062FC85
:10810000684622F0FAFBE2499DF802508868E14A8D
:108110008B681B1A9342FBD3684622F0EEFB0EB12C
:10812000FFF7C0FF9DF802006CB1A84202D12068A1
:10813000401C2060AFF26C1101A8226839F0C0F831
:108140003A4601A907E0A8423A4602D0AFF294119C
:1081500001E0AFF29011D0A0FFF71BFD3846FFF70A
:10816000EDFC07B0F0BD30B50C00CEA187B00546E0
:10817000D1E90001CDE900010ED022F087FC10B159
:108180002068401C2060AFF2BC1102A8226839F0C0
:1081900097F82A4602A908E022F078FC2A4610B196
:1081A000AFF2E01101E0AFF2EC116846FFF7F1FC2D
:1081B0002846FFF7C3FC07B030BD30B5BBA30C4663
:1081C00005460FCB89B08DE80F0008A908460CF0D2
:1081D00042F8AC480068D8B109282A4621D0AFF24D
:1081E00004216846FFF7D5FC6CB12068401C206074
:1081F000AFF2282104A8226839F062F82A4604A9BF
:108200006846FFF7C6FC2846FFF798FC09B030BD6A
:108210002A46AFF258216846FFF7BBFC002CE7D195
:10822000F1E7AFF260216846FFF7B3FC002CEAD01B
:108230002168491C2160DBE77FB50C46054618F034
:1082400064FB88B18F482A460068012809D0AFF244
:108250008C219AA0FFF79DFCC4B12068401C2060CF
:1082600009E0AFF28821F4E72A46AFF2B02193A0EB
:10827000FFF78FFC54B1AFF2AC216846226839F0A9
:108280001FF82A4669468DA0FFF783FC2846FFF7B2
:1082900055FC7FBD7FB50C46054625F069FD38B11C
:1082A0002A46AFF2C8210FE02068401C206018E089
:1082B0000AF017FF70B17348016803290AD0042936
:1082C00008D02A46AFF204317EA0FFF762FC002CF2
:1082D000EAD111E02A46AFF21C317AA0FFF759FC2F
:1082E00054B1AFF218316846226838F0E9FF2A46E7
:1082F000694674A0FFF74DFC2846FFF71FFC7FBDC1
:1083000030B5054671A085B000680C46049003F0B6
:10831000BCFA000607D42A46AFF2603104A8FFF782
:1083200038FC74B918E057482A460068192817D055
:10833000AFF2583104A8FFF72CFC6CB12068401C48
:108340002060AFF278316846226838F0B9FF2A46DB
:10835000694604A8FFF71DFC2846FFF7EFFBC4E4BD
:10836000AFF2A031E6E72DE9F043814658A00C4674
:108370008BB007C801AB002683E8070001202BF073
:1083800089FE08A80BF063FC3E4D932803D12868B2
:10839000062800D00126002108460BF0A8FC002783
:1083A00012E02868082815D117B94CA0FFF7C6FBC2
:1083B000BDF8002050A14846521C38F081FF4846C5
:1083C000FFF7BCFB01267F1C694600200BF068FF0D
:1083D0000028E6D1DFF8A880D8F80000932800D163
:1083E0000126002101200BF082FC002712E0286802
:1083F000082815D117B942A0FFF7A0FBBDF800204F
:108400003DA14846521C38F05BFF4846FFF796FBFB
:1084100001267F1C694601200BF042FF0028E6D1AF
:10842000D8F80000932800D10126002102200BF08B
:108430005EFC002712E02868082815D117B937A07C
:10844000FFF77CFBBDF800202BA14846521C38F0FA
:1084500037FF4846FFF772FB01267F1C6946022062
:108460000BF01EFF0028E6D1D8F8000093286CD04E
:1084700006B15FE072E068E020C2F0E5ECFF3A0090
:1084800008C007200CC0072010C007200040024091
:1084900000800040E0C81000D5CEC420D7C0D1CEA7
:1084A000C2000000CFCE20CFC4000000CFCE20CF2E
:1084B000C0CCDFD2C820CFC400000000DDD1CFCFB8
:1084C000C7D30000CFCFC7D300000000CEC7D30072
:1084D000CFE0ECFFF2FC20CFC4000000CFCEC2D032
:1084E000C5C6C4C5CDCDDBC520D4C8D1CAC0CBC894
:1084F000C7C0D6C8C83A0A0023253034750A000020
:10850000CFCEC2D0C5C6C4C5CDCDDBC520C0CAD272
:10851000C8C2C8C7C0D6C8C83A0A0000CFCEC2D0A9
:10852000C5C6C4C5CDCDDBC520D1CCC5CDDB3A0A8F
:10853000000000004A46AFF2745101A8FFF729FB82
:10854000F4B12068401C20600FE02868802801D02A
:1085500081288ED14A46AFF27C51EEE74A46AFF20F
:10856000A45101A8FFF715FB54B1AFF2A05104A824
:10857000226838F0A5FE4A4604A901A8FFF709FBC6
:108580004846FFF7DBFA0BB0BDE8F083704770B5E3
:108590008AB0064605A80BF05AFB20B13F220C21F9
:1085A00005A839F011FB00258DF820502022052167
:1085B00005A839F009FB324605A9FEA0FFF7E9FA44
:1085C0003046FFF7BBFA00200BF0A7FBFD4C20B9AB
:1085D000694600200BF065FB28B13F22142105A855
:1085E00039F0F2FA08E00A23052205A90DF10B0083
:1085F000FCF7CAFA00063AD48DF81E50324605A997
:10860000F1A0FFF7C6FA3046FFF798FA9DF814007C
:108610003F2816D0BDF8000005A9FCF747FB00066F
:1086200025D4324605A9EEA0FFF7B3FA3046FFF78E
:1086300085FAF048007828B301200BF06EFB50B9A2
:1086400004E0EDA105A839F02BF9EAE7694601201D
:108650000BF027FB20B1E8A105A839F021F909E0CA
:10866000BDF8000005A9FCF721FB000602D5206833
:108670000AB070BD324605A9E2A0FFF78AFA30467B
:10868000FFF75CFAE448256005607846E349086036
:108690000020EDE710B58CB004461822E0A105A833
:1086A00039F023FA0BA803F0A5F99DF82C0008B1C6
:1086B000E1A101E0AFF2DC61224605A8FFF769FA0B
:1086C0002046FFF73BFA9DF82C00002879D0694638
:1086D00000200BF084FA002873D1BDF80020D7A148
:1086E00001A8521E38F0ECFD224601A9D5A0FFF7E3
:1086F00050FA2046FFF722FABDF80000CFA1C0F1E2
:10870000190201A838F0DCFD224601A9D2A0FFF72A
:1087100040FA2046FFF712FA694602200BF05FFA92
:1087200000284ED1BDF80020AFF2EC6101A838F06E
:10873000C7FD224601A9CBA0FFF72BFA2046FFF781
:10874000FDF904A902200BF01BFA002839D1BDF86D
:108750001000BDF80010421AAFF21C7101A838F0E9
:10876000AFFD224601A9BCA0FFF713FA2046FFF790
:10877000E5F9A0480078002823D0694601200BF0D5
:108780002EFA00281DD1BDF80020ACA101A838F0B8
:1087900097FD224601A9B5A0FFF7FBF92046FFF798
:1087A000CDF9BDF80000A5A1C0F1400201A838F044
:1087B00087FD224601A9A8A0FFF7EBF92046FFF7A5
:1087C000BDF90CB010BDF0B5074695B00C460025BC
:1087D000032009F063FD7B4E000602D5306815B01A
:1087E000F0BD09F074FD000605D411A9052009F0BB
:1087F000BAFC00060AD514B12068401C206001258F
:108800003F220A21684639F0DFF914E00A230522E5
:10881000694611A8FCF7B8F913A9002009F0A3FCD8
:10882000000608D49DF84C00000604D514B1206859
:10883000401C2060012500208DF80A006A4690A1A6
:1088400005A838F03DFD44B1AFF680010DA82268BF
:1088500038F036FD3A460DA906E015B1AFF69C0199
:1088600001E0AFF6A8013A4605A8FFF792F9FBF739
:10887000EDFC3846FFF762F9FBF7FDFCAEE770B59B
:10888000064688B0032009F009FD4E4C000602D5CB
:10889000206808B070BD09F01AFD28B1FBF7D6FCBE
:1088A0003246AFF6C80109E005A9052009F05BFCD6
:1088B00030B1FBF7CBFC3246AFF6F80154A04BE0E9
:1088C0000A230522694605A8FCF75EF900258DF804
:1088D0000A50324669464EA0FFF75BF93046FFF773
:1088E0002DF904A9002009F03EFC9DF810000007B6
:1088F00001D551A101E0AFF61C11324663A0FFF78C
:1089000048F93046FFF71AF99DF81000400701D5E5
:1089100049A101E0AFF63C11324660A0FFF739F9FA
:108920003046FFF70BF99DF81000000601D542A173
:1089300001E0AFF6581132465CA0FFF72AF9304645
:10894000FFF7FCF868460AF0AFFA68B1FBF77EFC67
:108950003246AFF690115BA0FFF71BF93046FFF7E8
:10896000EDF8FBF788FC93E73246694655A0FFF720
:1089700010F93046FFF7E2F8274825600560784691
:1089800026490860002084E770B5504C0546B222A5
:10899000E18939F019F9E1890A20685403214CA0D2
:1089A0002CF0A0F80024002128462BF0E1FD641CE7
:1089B0000A2C8FE0D1C5D0C8C9CDDBC920CDCECC23
:1089C000C5D0000008C00720D0C5C3C8D1D2D0C0D0
:1089D000D6C8CECDCDDBC920CDCECCC5D0000000D1
:1089E000C4C0D2C020D0C5C3C8D1D2D0C0D6C8C898
:1089F00000000000084400003F3F2D3F3F2D3F3F57
:108A000000000000C4C0D2C020C7C0CCC5CDDB2050
:108A1000DDCACBC7000000000CC0072010C0072033
:108A2000CFC0CCDFD2DC20CFC420C0CAD2C8C2C8DD
:108A3000C7C8D02E00000000C4C000002530327529
:108A40000000000020CFC5D0C5D0C5C3C8D1D2D04A
:108A5000C0D6C8C9000000002020D1C2CEC1CEC4FB
:108A6000CDCE000020D1CCC5CD00000020C0CAD2A0
:108A7000C8C2C8C7C0D6C8C920DDCACBC70000005D
:108A8000DDCACBC7202825732900000020C0CAD228
:108A9000C8C2C8C7C8D0CEC2C0CDC00020C0D0D5C3
:108AA000C8C220CED2CAD0DBD200000020CDC5C8BB
:108AB000D1CFD0C0C2C8CCC0DF20CED8C8C1CAC0B8
:108AC0000000000020C2C5D0D1C8DF005CE2072052
:108AD0001B330000FFF467AF2BF016FFBDE87040BA
:108AE00008202BF035BB10B588B00446202168461D
:108AF00039F094F8FDA00068009022F030FD78B1C4
:108B00001C28FCA1684605D038F058FF2246AFF675
:108B10004C310BE038F052FF2246AFF6603105E0F1
:108B2000F4A1684638F04AFF2246F7A1FFF731F872
:108B30002046FFF703F8F84900200860F74908606D
:108B40007846F749086008B0002010BD2DE9F14FC4
:108B500090B029F078F9F04EF04FDFF8C49300247C
:108B600088B132F0CDFE109A88B1AFF69031EDA009
:108B7000FFF70FF81098FEF7E1FF1098FFF7B3FF2B
:108B800034603C60C1E0AFF6AC31109A5BE0D8A134
:108B9000E4A0FEF7FEFF1098FEF7D0FF28F06AFF72
:108BA000DFF8948300282CD103202BF073FA98F877
:108BB0000C0008F10D05012808D0022808D0032870
:108BC00038D0DEA1109838F07BFB17E0284616E07D
:108BD000DFA1284638F026FE0246E0A1109838F0C2
:108BE0006FFB1098FEF7AAFFD348E2A1713038F06E
:108BF00019FE821CE0A1109838F062FB1098FEF775
:108C00009DFF29F0C7F901202BF044FADDA0FEF703
:108C100095FF002021F022F9B8B102202BF03AFA9A
:108C2000E0A1E3A0DDF84020FEF7B3FF1098FEF7C7
:108C300085FFA5E76421284635F023F90028C5D033
:108C4000AFF68041109AB7A0EEE729F0BBFC98F888
:108C500008000328DDD100254FF0220B4FF02E0A2B
:108C60002BE06A1CD6A1684638F02AFBC5EBC5008C
:108C700000EB400008EB40018DF801401E2208A8DF
:108C800001F2E12138F0A6FE08A838F02DFE1D28DB
:108C900009D98DF83E408DF83DB08DF83BA08DF898
:108CA0003CA08DF83AA008A96846109AFEF771FF1B
:108CB0001098FEF743FF6D1CEDB298F8D402A8425D
:108CC000CFD8C2B2BEA1684638F0FAFA6946BDA054
:108CD000109AFEF75EFF1098FEF730FF98F8D40266
:108CE00010B1AFF6285101E0AFF628518DA0109ACF
:108CF000FEF74FFF1098FEF721FF98F8D00200F022
:108D0000010028F039FE34603C607946C9F8001053
:108D100011B00020BDE8F08F70B5044601202BF0A3
:108D2000B9F920F0FEFC002831D0ABA0FEF706FF19
:108D300018E0002021F092F8A0B102202BF0AAF94F
:108D4000224698A1ACA0FEF724FF2046FEF7F6FECF
:108D500071490020086071490860784670490860D0
:108D6000002070BD20F0DDFC0028E2D12046FFF796
:108D70000BFEA5A0FEF7E2FEAB4DAC68AB4E00BF0C
:108D800020F0CFFC18B9A868001BB042F8D3BDE8AA
:108D9000704002202BF07EB910B50446012027F068
:108DA00075FB22F059F9A0F55960B0F5C04F224685
:108DB00002D0AFF6F05101E0AFF600619CA0FEF7E3
:108DC000E8FE2046BDE81040FEF7B8BE70B5054687
:108DD0000C4646A0FEF7B2FE96A0FEF7AFFE04F0EA
:108DE0000F0003282ED097A0FEF7A8FEE00708D0BA
:108DF0002A46AFF6306199A0FEF7CBFE2846FEF773
:108E00009DFEA00708D52A46AFF6486195A0FEF75B
:108E1000C0FE2846FEF792FE600708D52A46AFF648
:108E20005C6192A0FEF7B5FE2846FEF787FE20079C
:108E300008D52A46AFF674618EA0FEF7AAFE284632
:108E4000FEF77CFEC4F303100C2818D08BA0FEF7AD
:108E500075FE600608D42A46AFF6986183A0FEF737
:108E600098FE2846FEF76AFE200608D42A46AFF68A
:108E7000AC6180A0FEF78DFE2846FEF75FFEC4F3CE
:108E800003200A2818D082A0FEF758FE600508D5F6
:108E90002A46AFF6D06175A0FEF77BFE2846FEF7A6
:108EA0004DFE200508D42A46AFF6E86171A0FEF712
:108EB00070FE2846FEF742FEC4F30330052814D0A6
:108EC00079A0FEF73BFE600408D42A46AFF60C7189
:108ED00066A0FEF75EFE2846FEF730FE200404D5AD
:108EE0002A46AFF6207163A0EAE0EEE05850322047
:108EF0000000000020424C5545544F4F544820D7A5
:108F0000C0D1D2DC00000000CDC5D220C7C0C3CB89
:108F1000D3D8CAC80000000008C007200CC0072032
:108F200010C00720CCCEC4D3CBDC20424C554554D6
:108F30004F4F54480000000060DA0720CDE5E8E715
:108F4000E2E5F1F2EDFBE920ECEEE4F3EBFC0000EE
:108F500056657273696F6E20000000005379732E9E
:108F600020436F6E6669672E2053657473202D2031
:108F7000257300003D2000004275696C643A20258D
:108F800073000000C8C4C5D220CFCEC8D1CA20D338
:108F9000D1D2D0CEC9D1D2C22E2E2E0A0A0A0A0AA6
:108FA00000000000CFD0CECFD3D9C5CD0000000047
:108FB000D2C5D1D220424C5545544F4F54480000A1
:108FC00025640000D3D1D2D0CEC9D1D2C220CDC029
:108FD000C9C4C5CDCE000000CED2CACBDED7C8D220
:108FE000C520C2CDC5D8CDC5C520CFC8D2C0CDC83B
:108FF000C50A0A0A0A0A0A00D2C5D1D220C1C0D2C3
:10900000C0D0C5C9000000000AC2CACBDED7C8D292
:10901000C520C2CDC5D8CDC5C520CFC8D2C0CDC80A
:10902000C50A0A0A0A0A0A000080004080C3C90172
:1090300055534200205749464920D7C0D1D2DC0AB7
:109040000000000020C2D1C520D1C8C3CDC0CBDBF9
:1090500020CDC020C2D5CEC40A0000002020CFC839
:10906000CD2037002020CFC8CD2038002020CFC809
:10907000CD2036002020CFC8CD20350020CFC8CD50
:10908000203720C820CFC8CD203820C220300A0089
:1090900020CFC8CD203720C220302C20CFC8CD20F3
:1090A0003820C220310A000020CFC8CD203720C28E
:1090B00020312C20CFC8CD203820C220300A00001B
:1090C000FEF767FD2846FEF739FDC4F30340032889
:1090D0001AD0F4A0FEF732FD600308D5F7492A46FE
:1090E000AFF27800FEF755FD2846FEF727FD200376
:1090F0000AD5F2492A46AFF28400FEF74AFD284617
:10910000BDE87040FEF71ABD70BD70B50C4605464F
:10911000AFF22820FEF712FDE9A0FEF70FFD04F0E4
:109120000700042821D0AFF2E400FEF707FDE007B6
:1091300007D02A46E149E8A0FEF72BFD2846FEF7B6
:10914000FDFCA00707D52A46DC49E5A0FEF721FD76
:109150002846FEF7F3FC600707D42A46D749E2A069
:10916000FEF717FD2846FEF7E9FCC4F3C20003280A
:1091700018D0DFA0FEF7E2FC200707D42A46CF492B
:10918000D5A0FEF706FD2846FEF7D8FCE00609D478
:109190002A46CA49D2A0FEF7FCFC2846BDE870402A
:1091A000FEF7CCBC70BD10B586B00446AFF2C42348
:1091B000D2A21421684638F099F822F09CF8D349DD
:1091C000401821D0A0F6C300B0F5804018D0D04997
:1091D0002246C84212D1AFF2D0216846FEF7D9FC30
:1091E0002046FEF7ABFCCB4900200860CA49086066
:1091F0007846CA49086006B0002010BDAF49ECE7C8
:10920000AE4922460839E8E72246C5A1E5E72DE93F
:10921000F0478046C54800268568DFF814A3374626
:109220008146404688F80070002137F029FA04464C
:10923000404638F059FB68B136B9012630462AF06D
:1092400029FFBCA0FEF77AFC03202AF023FF40464A
:10925000FEF774FC012C04D0BCB1022C19D0032CF5
:1092600020D0D9F80800411B5145DAD3D9F80800BD
:10927000411B51451AD3914942461831ADA0FEF722
:1092800088FC4046FEF75AFC12E08C4942460839F9
:1092900001E08A494246A7A0FEF77BFC4046FEF764
:1092A0004DFCE3E7854942461831F4E7032C02D12F
:1092B0004046FFF778FF9748076097480760784671
:1092C000964908600020BDE8F0872DE9F041B6B06E
:1092D00000262D962E962F963096319632963396FE
:1092E000349626A835962BF07EFA8A4C000617D4C1
:1092F0002020ADF8A6000220ADF8A2000120ADF8B4
:109300009A00ADF89C00ADF898000820ADF89E00DA
:10931000ADF8A460012126A82AF0BCFF000603D501
:10932000206836B0BDE8F08102202BF03EFB84A01F
:10933000FEF704FC01202AF0ADFE88A0FEF7FEFB3C
:1093400003202BF018FB8D4C0027002020F086FD19
:1093500048B102202AF09EFE89A0FEF7EFFB012013
:109360002AF098FE08E02BF06AFB20880743BFB282
:109370007807EAD5B807E8D52BF061FB20880028EC
:10938000FAD16A4CA068814DA168091AA942FBD3A1
:109390007FA0FEF7D3FB01202AF07CFE1DA80AF077
:1093A00056FC20B13F220C211DA838F00DFCB04620
:1093B0008DF88060202205211DA838F005FC03AA45
:1093C0001DA978A0FEF7E5FB03A8FEF7B7FB1CA8D4
:1093D00021F0C4FA18B924A821F08FFA20B172A1A3
:1093E00003A838F05DFA12E0BDF870209DF89110E6
:1093F000A2F5FA629DF890000092CDE901019DF876
:1094000072309DF873206DA103A837F059FF032037
:109410002AF040FE03A8FEF791FB01202AF03AFE55
:1094200003A8FEF7ECFC6CA26EA103A837F048FF7E
:10943000002103A82BF09CF86BA0FEF77FFB2BF01C
:10944000FEFAB80703AA02D51C49083900E01B49F7
:1094500068A0FEF79EFB03A8FEF770FB780703AA3F
:1094600002D51649083900E0144964A0FEF791FBC3
:1094700003A8FEF763FB63A0FEF760FB002108462C
:1094800028F0D7F80121002028F0D3F840B90221B4
:10949000002028F0CEF818B1084903AA0839BBE02B
:1094A000B8E0000020CFC8CD203720C220312C20CA
:1094B000CFC8CD203820C220310A0000C47F000070
:1094C0002047534D2F424C5545544F4F544820D7B9
:1094D000C0D1D2DC0A0000002020CFC8CD2033004C
:1094E0002020CFC8CD2032002020CFC8CD20310091
:1094F00020CFC8CD203120C220300A00257320574C
:1095000049464920D7C0D1D2DC00000000EEFCFF64
:10951000F77BF3FF08C007200CC0072010C007200E
:10952000CDC5D2202B332E335600000000800040E2
:10953000404B4C00CCCEC4D3CBDC2057494649002D
:109540003D20D2C5D5CDCECBCEC3C8D7C5D1CAC894
:10955000C920CFD0CEC3CECD203D0A00D2C5D1D2B6
:1095600020C4C0D2D7C8CACEC220CAD0DBD8CAC88D
:1095700020C820C1D3CCC0C3C80A0000AE0300106D
:10958000CFD0CECFD3D9C5CD0A00000020A107008F
:109590003D3D3D2020CFD0CEC3CECD203120203D3B
:1095A0003D3D0A00CFC4000058582D58582D58583A
:1095B00058582058583A58580A000000253032753B
:1095C0002D253032752D2530327520253032753AF3
:1095D000253032750A000000465072696E742D31D4
:1095E0003100000025730A00C4C0D2D7C8CAC80A17
:1095F0000000000020CAD0DBD8CAC80020C1D3CCEC
:10960000C0C3C80052533233322D310A200A200A17
:1096100000000000FA4903AAFAA0FEF7BAFA03A86C
:10962000FEF78CFAFAA0FEF789FA03202BF0A3F9D3
:10963000002020F013FC08B1012700E000270121E1
:10964000002027F0F6FF30B10221002027F0F1FFC3
:1096500008B1012600E000263743E9D003202AF0B4
:1096600019FD0EB1EDA000E0EFA0FEF767FA0120B2
:109670002AF010FD0321002027F0DBFF002020F05E
:10968000EDFB0028FAD1EBA0FEF758FA00210220EA
:1096900027F0CFFF0121022027F0CBFF40B90221A4
:1096A000084627F0C6FF18B1D54903AA083901E0DA
:1096B000D34903AAD3A0FEF76CFA03A8FEF73EFA3B
:1096C000D3A0FEF73BFA03202BF055F9002020F041
:1096D000C5FB08B1012700E000270121022027F087
:1096E000A8FF30B10221084627F0A3FF08B10126E8
:1096F00000E000263743E9D003202AF0CBFC0EB16E
:10970000C6A000E0C8A0FEF719FA01202AF0C2FCAA
:109710000321022027F08DFFA068A168091AA94241
:10972000FBD3002020F09AFB0028FAD103A8FFF712
:1097300033FB03A8FFF76BFD03A8FFF707FA00212F
:1097400003A8FEF7B9FC002103A8FEF79AFA00214E
:1097500003A8FEF708FD002103A8FEF72EFD002157
:1097600003A8FEF7CDFD002103A8FEF765FD00214B
:1097700003A8FEF78FFD002103A8FEF7F4FD03A860
:10978000FEF788FF002103A8FFF71DF847462CA924
:109790001320CDF8B08016F070F908B164202C9039
:1097A000A8A11DA82C9A37F08BFD03AA1DA9A6A07D
:1097B000FEF7EFF903A8FEF7C1F92BF0A5F803A80F
:1097C000FFF7E2F8AFF2F420FEF7B8F903A8FFF7CD
:1097D000A3FA01202AF05EFC9EA0FEF7AFF9032059
:1097E0002BF0C9F8A668002020F038FB00B1A6686D
:1097F000A068801BA842F6D3814903AA083997A024
:10980000FEF7C7F903A8FEF799F997A0FEF796F9B6
:1098100003202BF0B0F8A668002020F01FFB00B951
:10982000A668A068801BA842F6D303202AF032FC69
:1098300073485C30FEF782F901202AF02BFC0020EF
:1098400020F00CFB0028FAD18AA0FEF777F903205C
:109850002BF091F88A4E06E020F039FBA068A16851
:10986000091AB142FBD3002020F0F8FA00284FF08B
:109870000300F1D020F00DFB022020F0FDFA03AA36
:1098800080A168A0FEF785F903A8FEF757F97FA02D
:10989000FEF754F903202BF06EF84FF4FA76C82146
:1098A00030461FF0AEFDA068A168091AA942FBD39B
:1098B000002020F0D3FA0028F1D003AA71A159A00A
:1098C000FEF767F903A8FEF739F9002020F0C6FA81
:1098D0000028FAD101202AF0DDFB1FF022FF00282A
:1098E0007ED06DA0FEF72AF903202AF0D3FB2BF0DF
:1098F000A6F86F4D2878400702D441485C3001E05B
:109900003F486430FEF71AF901202AF0C3FB69A032
:10991000FEF714F903202BF02EF8694E2AF0CFFA47
:10992000A068A168091AB142FBD3002020F096FA82
:109930000028F3D002202AF0ADFB62A0FEF7FEF86B
:1099400001202AF0A7FB62A0FEF7F8F803202BF015
:1099500012F82BF074F803202AF09CFB28784007BB
:1099600002D527485C3001E025486430FEF7E6F870
:1099700003A8FEF78FFA2AF0C7FFADF8947025A967
:10998000392016F07AF8ADF8887022A93A2016F03E
:1099900074F81B49BDF888207C311DA837F090FC75
:1099A00003AA1DA94DA0FEF7F4F803A8FEF7C6F818
:1099B000BDF894204DA11DA837F082FC03AA1DA973
:1099C0004DA0FEF7E6F803A8FEF7B8F8542015F00E
:1099D000DEFD2BA801F0C2F82BA800F087FC00E008
:1099E00005E02BA801F0B0F80125464E12E103AACC
:1099F000AFF6502144A0FEF7CCF803A8B6E700006C
:109A0000C47F000020D0C0C7CCDBCAC0CDC8C50011
:109A100020C7C0CCDBCAC0CDC8C5000020CDCED089
:109A2000CC0A0A0A0000000020CDC5CDCED0CC0A59
:109A30000A0A000052533233322D320A200A200A19
:109A40000000000025750000DFD0CACED1D2DC2096
:109A5000D7CB0000CACDCECFCAC00A00D0C0C7CC79
:109A6000DBCAC0CDC8C50000C7C0CCDBCAC0CDC8EA
:109A7000C50A0A00C8CDC4C8CAC0D2CED0DB000017
:109A8000400D0300CFD0CEC9C4C5CD00C4C8CDC0E1
:109A9000CCC8CA0A00000000C4C5CDC5C6CDDBC90C
:109AA00020DFD9C8CA0A20C7C0CAD0DBD20A00004A
:109AB000AC030010D2C5D1D220C7C0CCCAC00A00A6
:109AC00000350C00CFD0CEC9C4C5CD0A00000000BF
:109AD00020CED2CAD0DBD20A00000000D7C8D1CB3A
:109AE000CE20D6C8CACBCEC20000000025303475C7
:109AF00020D1C5CA00000000C7C0C4C5D0C6CAC0B6
:109B00000000000002000010C4C5CDC5C6CDDBC9F1
:109B100020DFD9C8CA000000308840F00200308041
:109B200001200DF07FF801202AF0B4FABDF888304A
:109B30002A465DA103A837F0C3FB03A8FDF7FEFF8B
:109B40001CA820F00BFF18B924A820F0D6FE28B1DD
:109B5000AFF2AC5103A837F0A3FE13E0BDF87020BC
:109B60009DF89100A2F5FA629DF890100092CDE95F
:109B700001109DF872309DF87320AFF2C05103A818
:109B800037F09EFB03202AF085FA03A8FDF7D6FFE5
:109B900001202AF07FFA2AF0B7FE03A8FEF7F4FEB0
:109BA000AFF2D060FDF7CAFF2DA903A8FEF784FA33
:109BB0002EA903A8FEF765F82FA903A8FEF7D3FA8C
:109BC00030A903A8FEF7F9FA32A903A8FEF798FB1B
:109BD00033A903A8FEF730FB34A903A8FEF75AFB0C
:109BE00031A903A8FEF7BFFB35A903A8FEF7EBFDDB
:109BF000A76803E0002020F031F980B9A06843F69F
:109C00000951C21BBDF894004843B2EB801FF1D349
:109C10006D1CADB2BDF8880085427FF67DAF552042
:109C200015F0B5FC2BA800F099FF2BA800F05EFB07
:109C30002BA800F089FF308840F00200308001201E
:109C40000CF0F0FF1DA0FDF779FF03202AF022FAA7
:109C500023A0FDF773FF308840F002003080012020
:109C60000CF0E0FFFEE710B586B0044605A9012020
:109C700015F038FE9DF814201CA1684637F020FB33
:109C8000224669461BA0FDF784FF2046FDF756FFDC
:109C90001E49002008601E49086078461D4908607A
:109CA00006B0002010BD0000D6C8CACB2025303435
:109CB0007520C8C720253034750A00003DD2C5D5AF
:109CC000CDCECBCEC3C8D7C5D1CAC8C920D2C5D185
:109CD000D220C7C0C2C5D0D8C5CD3D0A0A0A0A00E5
:109CE00028CFCEC4CFC8D1DC290A0A00253032647F
:109CF00000000000CDCECCC5D020CACACC20C220E6
:109D0000CCC0C3C0C7C8CDC50000000008C0072034
:109D10000CC0072010C00720F0B5036802790D6859
:109D2000002462F30704EB18002242EB0401FE4D0D
:109D3000FE4EDFF8FCC30C0A04D1FE4FE824FF1AE4
:109D40008C4108D289202860012030607846CCF808
:109D500000008920F0BD036001712A6078463260FE
:109D6000CCF800000020F0BDF0B500230C681A46C6
:109D70000979057961F30702016865F30703611842
:109D80005A41E94CE94DEA4E130A04D1E94FE82360
:109D90007F1A934107D289202060012028607846ED
:109DA00030608920F0BD01600271002020602860D1
:109DB000784630600020F0BDF0B500220C681346F4
:109DC0000979057961F30703016865F30702D64D48
:109DD000D64EDFF85CC30F1B72EB030708D2892055
:109DE0002860022030607846CCF800008920F0BD61
:109DF000091B62EB030201600271002028603060E1
:109E00007846CCF800000020F0BDF0B50368096882
:109E10000022CB18C44CC54DC54E52EB020106D1F1
:109E2000DFF810C3E827BCEB030C8F4107D2892071
:109E3000206001202860784630608920F0BD0360F2
:109E4000226078462A6030600020F0BDF0B50368DB
:109E500009680022CB18B44CB44DB54E52EB020148
:109E600006D1DFF8D4C20227BCEB030C8F4107D226
:109E70008920206001202860784630608920F0BD6C
:109E80000360226078462A6030600020F0BD30B563
:109E900002680968A44BA54CA54D8A4207D28920C7
:109EA00018600220206078462860892030BD511A51
:109EB000016000201860206078462860002030BDD6
:109EC000F0B5036809680022CB18974C974D984E5F
:109ED00052EB020106D1DFF860C20227BCEB030C93
:109EE0008F4107D2892020600120286078463060A9
:109EF0008920F0BD0360226078462A60306000202F
:109F0000F0BD30B502680968874B884C884D8A429D
:109F100007D28920186002202060784628608920B6
:109F200030BD511A0160002018602060784628601A
:109F3000002030BD10B5028809887C4B11447A4A54
:109F40007B4CB1F5803F07D3892010600120186059
:109F500078462060892010BD0180002010601860C4
:109F600078462060002010BD0021016001716E481C
:109F700001606E48016078466D49086000207047B6
:109F8000002101608180817167480160674801603C
:109F9000784667490860002070471CB50023CDE96A
:109FA0000033036800938388ADF8043080798DF81E
:109FB000060000201060DDE900340968CB1A70EB60
:109FC000040301D2411E05E0DDE90043611A83412B
:109FD00001D2012111605449086054490860784653
:109FE0005349086000201CBD2DE9FC410022CDE949
:109FF0000022026800928288ADF8042082798DF8F0
:10A000000620DDE900430A680021141941EB030230
:10A01000CDE90042150E444A444B454C08D1DDE9D8
:10A020000067DFF818C1464DBCEB0606BD4108D2FB
:10A030008920106001201860784620608920BDE8E2
:10A04000FC81009D0560BDF8045085809DF8065098
:10A05000857111607846196020600020EFE72DE9D6
:10A06000FC410022CDE90022026800928288ADF80E
:10A07000042082798DF80620DDE900730A6800214A
:10A08000294C2A4D2A4EBF1A8B4107D289202060C5
:10A0900001202860784630608920D0E7DDE9007330
:10A0A000BA1A63EB0103CDE900230260BDF8042076
:10A0B00082809DF806208271216078462960306098
:10A0C0000020BCE72DE9FF410022CDE90222CDE9C5
:10A0D00000220A6802928A88ADF80C2089798DF8EE
:10A0E0000E10016800918188ADF8041081798DF817
:10A0F0000610DDE90031DDE902421B195141CDE9CD
:10A1000000310C0E0849094A094B06D1DDE9005619
:10A110000A4F0B4C7D1BB44118D2892008600120E6
:10A120001060784618600DE008C007200CC00720BA
:10A1300010C00720FF0FA5D4FFE30B54FFFF63A758
:10A14000B3B6E00D892004B0BDE8F081009C046046
:10A15000BDF8044084809DF80640847100200860AA
:10A160001060784618600020EDE72DE9FC410022E0
:10A17000CDE900220B68097961F3070201680091BB
:10A180008188ADF8041081798DF80610DDE900149E
:10A190005B186241CDE90032140E8849884A894B28
:10A1A00006D1DDE90056884F884C7D1BB44107D2AB
:10A1B00089200860012010607846186089203EE7F9
:10A1C000009C0460BDF8044084809DF806408471C2
:10A1D0000020086010607846186000202FE72DE905
:10A1E000F0410546006809680024A1FB002304FB38
:10A1F000003001FB04014FF4FA70101841F1000126
:10A200004FF47A72234636F0BFFF6C4A6C4B6D4EAA
:10A2100031B9DFF8BCC10227BCEB000C8F4107D27B
:10A2200089201060032018607846306089208BE711
:10A230002860146078461C603060002084E72DE9B7
:10A24000F0410546006809880024A1FB002304FBB7
:10A25000003001FB040141F28830101841F1000187
:10A2600042F21072234636F08FFF544A544B554E3B
:10A2700031B9DFF85CC10227BCEB000C8F4107D27B
:10A2800089201060032018607846306089205BE7E1
:10A290002860146078461C603060002054E7018814
:10A2A00042F20F72491C89B20180914201D9012109
:10A2B00001804249002008604149086078464149D0
:10A2C000086000207047018842F20F72491E89B26F
:10A2D0000180914200D90280384900200860384945
:10A2E0000860784637490860002070470168394A9D
:10A2F000491C0160914201D9012101602F490020D0
:10A3000008602F49086078462E4908600020704791
:10A310000168304A491E0160914200D90260274914
:10A320000020086026490860784626490860002019
:10A3300070472DE9F0410446D1E90001D4E900233A
:10A34000A0FB025601FB026100FB031168194941A1
:10A350008018594142F21075401941F1000152191B
:10A3600043F1000392185B4136F00EFF134B144D7E
:10A37000144E0A0A04D1184FE8223F1A8A4107D224
:10A380008920186003202860784630608920DBE649
:10A39000C4E9000100201860286078463060002081
:10A3A000D2E66422B0FBF2F102FB1101B0FBF2F045
:10A3B0003229114600D3401C4843704708C007208B
:10A3C0000CC0072010C00720FFFF63A7B3B6E00D45
:10A3D000FFE30B54FFE0F505FF0FA5D42DE9FF4780
:10A3E00017F0F0FD6E4C000615D401F0FFFFDFF80A
:10A3F000B481DFF8B4916D4F002668B1012820D0F8
:10A4000087281DD0684601F0A2F8000603D49DF805
:10A4100000000E287ED0AEE0684601F098F80006F5
:10A4200079D403A801F0BAF8000674D49DF80000AE
:10A430000E2805D1BDF80C00402801D171203870DC
:10A4400089E0684601F083F8000664D49DF80000B6
:10A450001D2827D2DFE800F0260F22222222141422
:10A460001414141414140F12121212120F24242490
:10A470002426121212001BF087FE03E0202000E0C9
:10A480006020387002F060F8000674D49DF8000077
:10A49000474D0E2811D0172812D014E05020F0E7B5
:10A4A0003020EEE7882009212060C8F800107946A6
:10A4B000C9F8001004B0BDE8F0870CF07FFC05E09F
:10A4C0002878022844D001200CF0ACFB000652D4BE
:10A4D0009DF80000172806D12878012835D11BF0F7
:10A4E000C3FE000647D49DF800000E2825D1287829
:10A4F000022826D108F04DFFD8B901A806F03BFD8F
:10A50000000638D40DF1060006F019FD000632D41D
:10A51000284801E027E02EE000788DF80800172099
:10A520008DF8090001A801F017FF000623D432209E
:10A5300038709DF800000E2803D0C0B2172804D050
:10A5400009E02878032803D005E02878022802D102
:10A5500002F0EFF92E7026607946C8F800600020FE
:10A56000C9F80010A6E7F9F771FE1BF00DFEF9F728
:10A5700082FE01F0E9FF20689CE708B5684600F01C
:10A5800095FA58B99DF80000082807D0092805D089
:10A590000A2803D008480088002800D0012008BD00
:10A5A00008C007200CC0072010C007206C02001054
:10A5B000CC0100106D02001098C107202DE9F8436E
:10A5C000CD4ECE4FCE4C05464FF08808B0F1004F2F
:10A5D00006D0B5F1104F03D00220C4F800800AE085
:10A5E000684601F04BF9000628D49DF8000040B100
:10A5F0000A20C4F800803060784638608820BDE8C2
:10A60000F88301226946284625F00EFF000615D47E
:10A610009DF80000FF2809D0FF208DF800000122DE
:10A620006946284625F00BFF000607D4280F8DF851
:10A630000000684601F018F9000601D52068DEE741
:10A64000B0490120087000204860206030607846E2
:10A6500038600020D3E7AB4900200870A8490860A3
:10A66000A54908607846A549086000207047A549BB
:10A6700001200870A249002008609F4908607846C0
:10A680009E49086000207047F8B5684601F0F6F86A
:10A690009B4D000618D49DF80000974E974FA8B127
:10A6A0009849002400070C70FF218DF8001001224A
:10A6B000694625F0C4FE000606D48DF800406846C1
:10A6C00001F0D2F8000609D52868F8BD8820286076
:10A6D0000A203060784638608820F8BD2C607846C3
:10A6E000346038600020F8BD2DE9F74F92B0144671
:10A6F00010A801F0C3F8824D000649D49DF840002F
:10A70000DFF8F481DFF8F4918827B0B1060730460E
:10A7100025F0A1FE7B4A401E4FF0000A51680B193C
:10A720005B1D98420ED22F60C8F800A079468820A1
:10A73000C9F8001015B0BDE8F08F0A212F60C8F8E5
:10A740000010F3E746EA01078DF800401298ADF8D3
:10A75000010093466E462246F01C139937F03AF9F1
:10A760003019FF21C4700171221D711C781C25F065
:10A7700066FE00060CD40920B0EB177F01D1621DE4
:10A7800000E001226946384625F059FE000601D551
:10A790002868CFE7DBF804102144091DCBF804102A
:10A7A000C5F800A07946C8F800A00020C9F800103C
:10A7B000C0E72DE9F04F524D4F4F99B0D5F80090BA
:10A7C00016A8D7F800A001F059F8000664D49DF847
:10A7D0005800DFF82881040700264FF0010B012202
:10A7E00001A9204625F020FE000655D49DF804005E
:10A7F000F0B3FF284AD00444241D04F0704025F033
:10A800002AFE24F07041401E884211D39DF80400B6
:10A8100040280DD8761CE2E7641E012201A92046DB
:10A8200025F002FE000637D49DF80400402808D920
:10A83000882028607946C7F800B0C8F8001019B021
:10A8400079E7241AA41E022215A9204625F0ECFD62
:10A85000000621D4A41C9DF8042002A9204625F05E
:10A86000E3FD000618D4BDF8540040F0005000E0AD
:10A870000CE09DF8042002A925F0E1FD00060BD4B0
:10A880009DF8040021180C1AE41E761E002EC3D178
:10A89000FFF7FAFE000601D52868D0E7C5F800905A
:10A8A0007946C7F800A04846C8F80010C7E708B5C1
:10A8B000684600F0E3FF08B1002008BD9DF80000E5
:10A8C0000028FAD000070122694625F0ADFD0006F8
:10A8D00005D50B4800680028EFD0012008BD9DF881
:10A8E000000008B1FF28F8D100208DF8000068466C
:10A8F00000F0BAFFE0E700000CC0072010C00720FE
:10A9000008C00720C40100102DE9F0418046FB4833
:10A9100016461D4600780F4680B11A46404625F07F
:10A9200083FDF74C000606D42A4639464046FFF719
:10A93000DBFE000602D52068BDE8F0812A463146DC
:10A940004046BDE8F04125F07ABD38B5022269469F
:10A950004FF0704025F068FDE94C000602D52088D4
:10A9600085B201E0BDF8005001F0B4F8E549E64ACF
:10A97000854206D1002020600860784610600020E3
:10A9800038BD88202060112008607846106088203B
:10A9900038BD2DE9FF4FDA4CDA4EDB4F81B09946D6
:10A9A00092468B4600254FF070484A465146019822
:10A9B00025F045FD000611D401F08CF8ADF800003B
:10A9C00002226946404625F03AFD000606D44A4672
:10A9D0005946019825F028FD000603D5206805B0EA
:10A9E000BDE8F08F4A465146584636F02DFF10B963
:10A9F000FFF7ABFF58B16D1CADB2032DD5D382204C
:10AA0000206022203060784638608220E7E700200E
:10AA100020603060784638600020E0E71CB5C0EB6D
:10AA2000C000401F0A4640F0704007236946FFF708
:10AA3000B0FF1CBD00B587B00246B4481C23694670
:10AA4000FFF7A7FF07B000BDC0EBC000401F40F0FC
:10AA50007040072225F0E8BC38B5AD4C0246012312
:10AA600069462046FFF750FF38BDA94B0146012239
:10AA7000184625F0D9BC38B5A54C0246641C012304
:10AA800069462046FFF740FF38BDA14B01465B1CDD
:10AA90000122184625F0C8BC38B59D4C0246A41CBE
:10AAA000012369462046FFF72FFF38BD984B01462A
:10AAB0009B1C0122184625F0B7BC38B5944C0246C1
:10AAC000E41C012369462046FFF71EFF38BD904B6A
:10AAD0000146DB1C0122184625F0A6BC38B58C4C7B
:10AAE0000246241D012369462046FFF70DFF38BDAD
:10AAF000874B01461B1D0122184625F095BC1CB54D
:10AB0000C0EBC00026300A4640F0005007236946DB
:10AB1000FFF7FAFE1CBDC0EBC000263040F000502D
:10AB2000072225F081BC38B5794C02464B3401230D
:10AB300069462046FFF7E8FE38BD754B01464B33AA
:10AB40000122184625F070BC38B5714C02464C34D1
:10AB5000042369462046FFF7D7FE38BD6C4B0146FB
:10AB60004C330422184625F05FBC38B5684C0246C9
:10AB70005034022369462046FFF7C6FE38BD644BB9
:10AB8000014650330222184625F04EBC38B5604CC1
:10AB900002465234042369462046FFF7B5FE38BD0D
:10ABA0005B4B014652330422184625F03DBC38B5B4
:10ABB000574C02465634022369462046FFF7A4FE4E
:10ABC00038BD534B014656330222184625F02CBCA3
:10ABD00038B54F4C02465834022369462046FFF7E9
:10ABE00093FE38BD4A4B014658330222184625F0E1
:10ABF0001BBC38B5464C02465A34012369462046F0
:10AC0000FFF782FE38BD424B01465A3301221846F7
:10AC100025F00ABC38B53E4C02465B340423694635
:10AC20002046FFF771FE38BD394B01465B330422E5
:10AC3000184625F0F9BB832208B502EB80000A46CE
:10AC400040F0005004236946FFF75EFE08BD8322F2
:10AC500002EB800040F00050042225F0E5BB38B53F
:10AC60002B4C02468734042369462046FFF74CFEEE
:10AC700038BD274B014687330422184625F0D4BB44
:10AC800038B5234C02468B34022369462046FFF731
:10AC90003BFE38BD1E4B01468B330222184625F081
:10ACA000C3BB38B51A4C02468D340423694620468E
:10ACB000FFF72AFE38BD164B01468D330422184695
:10ACC00025F0B2BB38B5124C0246913402236946D6
:10ACD0002046FFF719FE38BD0D4B01469133022285
:10ACE000184625F0A1BB38B5094C02469334012320
:10ACF00069462046FFF708FE38BD0000C401001079
:10AD000008C007200CC0072010C00720020000F078
:10AD100028000020F94B01460122184625F084BB8B
:10AD200038B5F64C0246641C042369462046FFF7FA
:10AD3000EBFDE1E7F14B01465B1C0422184625F0D0
:10AD400073BB38B5ED4C0246641D042369462046AA
:10AD5000FFF7DAFDD0E7E94B01465B1D04221846F8
:10AD600025F062BB38B5E54C024609340423694638
:10AD70002046FFF7C9FDBFE7E04B01460933042237
:10AD8000184625F051BB38B5DC4C02460D34012382
:10AD900069462046FFF7B8FDAEE7D84B01460D33B4
:10ADA0000122184625F040BB38B5D44C02460E347B
:10ADB000042369462046FFF7A7FD9DE7CF4B0146D8
:10ADC0000E330422184625F02FBB38B5CB4C024673
:10ADD0001234022369462046FFF796FD8CE7C74BE5
:10ADE000014612330222184625F01EBB38B5C34C6B
:10ADF00002461434022369462046FFF785FD7BE7AF
:10AE0000BE4B014614330222184625F00DBBCD225D
:10AE100008B502EB80000A4640F000500423694662
:10AE2000FFF772FD08BDCD2202EB800040F000501C
:10AE3000042225F0F9BA40F20D1208B502EB8000A9
:10AE40000A4640F0005004236946FFF75DFD08BD47
:10AE500040F20D1202EB800040F00050042225F079
:10AE6000E3BA38B5A54C0246963404236946204619
:10AE7000FFF74AFD40E7A14B0146963304221846EE
:10AE800025F0D2BA38B59D4C02469A34042369465F
:10AE90002046FFF739FD2FE7984B01469A330422ED
:10AEA000184625F0C1BA38B5944C02469E340123A9
:10AEB00069462046FFF728FD1EE7904B01469E336A
:10AEC0000122184625F0B0BA38B58C4C02469F34A2
:10AED000042369462046FFF717FD0DE7874B01461F
:10AEE0009F330422184625F09FBA38B5834C02469A
:10AEF000A334042369462046FFF706FDFCE67F4B9A
:10AF00000146A3330422184625F08EBA38B57B4C8F
:10AF10000246A734042369462046FFF7F5FCEBE61A
:10AF2000764B0146A7330422184625F07DBA38B582
:10AF3000724C0246AB34012369462046FFF7E4FC1D
:10AF4000DAE66E4B0146AB330122184625F06CBAA7
:10AF500038B56A4C0246AC34022369462046FFF7F6
:10AF6000D3FCC9E6654B0146AC330222184625F0F6
:10AF70005BBA38B5614C0246AE34042369462046BC
:10AF8000FFF7C2FCB8E65D4B0146AE33042218461B
:10AF900025F04ABA38B5594C0246B2340123694605
:10AFA0002046FFF7B1FCA7E6544B0146B23301221D
:10AFB000184625F039BA38B5504C0246B33401234F
:10AFC00069462046FFF7A0FC96E64C4B0146B3339A
:10AFD0000122184625F028BA38B5484C0246B43448
:10AFE000022369462046FFF78FFC85E6434B014666
:10AFF000B4330222184625F017BA38B53F4C024642
:10B00000B634042369462046FFF77EFC74E63B4BCA
:10B010000146B6330422184625F006BA38B5374C37
:10B020000246BA34042369462046FFF76DFC63E606
:10B03000324B0146BA330422184625F0F5B938B52B
:10B040002E4C0246BE34042369462046FFF75CFCC2
:10B0500052E62A4B0146BE330422184625F0E4B9D5
:10B0600038B5264C0246C234042369462046FFF711
:10B070004BFC41E6214B0146C2330422184625F021
:10B08000D3B938B51D4C0246C63401236946204663
:10B09000FFF73AFC30E6194B0146C6330122184649
:10B0A00025F0C2B91CB500EB800000F27D100A4605
:10B0B00040F0005005236946FFF726FC1CBD00EB5D
:10B0C000800000F27D1040F00050052225F0ACB960
:10B0D0004FF4CA7208B502EB40000A4640F0005037
:10B0E00002236946FFF710FC08BD4FF4CA7202EB59
:10B0F000400040F00050022225F096B9BB0000202D
:10B100004FF4CE7208B502EB40000A4640F0005002
:10B1100002236946FFF7F8FB08BD4FF4CE7202EB3D
:10B12000400040F00050022225F07EB91CB500EB33
:10B13000800001EB810100EB810000F28D1040F0F6
:10B14000005005236946FFF7DFFB1CBD00EB8000C4
:10B1500001EB810100EB8100134600F28D1040F0FD
:10B1600000500522194625F05FB9090108B501EB29
:10B17000800000F2D22040F0005004236946FFF71F
:10B18000C3FB08BD090101EB8000134600F2D22089
:10B1900040F000500422194625F046B91CB500EBDA
:10B1A000800001EB810100EB810000F2CD3040F026
:10B1B000005005236946FFF7A7FB1CBD00EB80008C
:10B1C00001EB810100EB8100134600F2CD3040F02D
:10B1D00000500522194625F027B938B5F84C02462B
:10B1E000042369462046FFF78FFB85E5F44B0146B3
:10B1F0000422184625F018B91CB500EB800000F2B7
:10B2000025500A4640F0005005236946FFF77CFBB5
:10B210001CBD00EB800000F2255040F000500522DC
:10B2200025F002B938B5E64C0246183404236946C5
:10B230002046FFF769FB5FE5E14B01461833042226
:10B24000184625F0F1B81CB500EB800000F23D5027
:10B250000A4640F0005005236946FFF755FB1CBD28
:10B2600000EB800000F23D5040F00050052225F038
:10B27000DBB81CB500EB800000F251500A4640F0EC
:10B28000005005236946FFF73FFB1CBD00EB800023
:10B2900000F2515040F00050052225F0C5B81CB511
:10B2A00000EB800000F265500A4640F00050052394
:10B2B0006946FFF729FB1CBD00EB800000F26550DA
:10B2C00040F00050052225F0AFB81CB500EB80001F
:10B2D00001EB810100EB810000F2655040F000506D
:10B2E00005236946FFF710FB1CBD00EB800001EB56
:10B2F000810100EB8100134600F2655040F00050E0
:10B300000522194625F090B81CB500EB800001EB32
:10B31000810100EB810000F22D6040F00050052318
:10B320006946FFF7F1FA1CBD00EB800001EB8101DB
:10B3300000EB8100134600F22D6040F00050052222
:10B34000194625F071B81CB500EB800001EB8101B6
:10B3500000EB810000F60D0040F000500523694627
:10B36000FFF7D2FA1CBD00EB800001EB810100EB7E
:10B370008100134600F60D0040F0005005221946EA
:10B3800025F052B81CB500EB800000F679200A4683
:10B3900040F0005005236946FFF7B6FA1CBD00EBEC
:10B3A000800000F6792040F00050052225F03CB8DE
:10B3B00040F6862208B502EB40000A4640F00050F5
:10B3C00002236946FFF7A0FA08BD40F6862202EB89
:10B3D000400040F00050022225F026B81CB500EBDA
:10B3E000800001EB810100EB410000F67D2040F080
:10B3F000005005236946FFF787FA1CBD00EB80006B
:10B4000001EB810100EB4100134600F67D2040F086
:10B4100000500522194625F007B840F6EE2208B57F
:10B4200002EB40000A4640F0005002236946FFF755
:10B430006BFA08BD40F6EE2202EB400040F00050EF
:10B44000022224F0F1BF40F6F62208B502EB4000DC
:10B450000A4640F0005002236946FFF755FA08BD3E
:10B4600040F6F62202EB400040F00050022224F0A9
:10B47000DBBF38B5534C0246022369462046FFF72E
:10B4800043FA39E44F4B01460222184624F0CCBF60
:10B4900038B54C4C0246A41C022369462046FFF7EF
:10B4A00033FA29E4474B01469B1C0222184624F03C
:10B4B000BBBF38B5434C0246241D012369462046D4
:10B4C000FFF722FA18E43F4B01461B1D01221846E4
:10B4D00024F0AABF38B53B4C0246641D02236946DE
:10B4E0002046FFF711FA07E4364B01465B1D0222A6
:10B4F000184624F099BF38B5324C0246E41D0223A9
:10B5000069462046FFF700FA13E42E4B0146DB1D87
:10B510000222184624F088BF38B52A4C0246093466
:10B52000012369462046FFF7EFF913E4254B014656
:10B5300009330122184624F077BF38B5214C024662
:10B540000A34012369462046FFF7DEF913E41D4B58
:10B5500001460A330122184624F066BF40F609323C
:10B5600008B502EB40000A4640F00050022369464D
:10B57000FFF7CAF908BD40F6093202EB400040F07F
:10B580000050022224F050BF38B50E4C0246413420
:10B59000022369462046FFF7B7F90EE4094B01463E
:10B5A00041330222184624F03FBF38B5054C02460D
:10B5B0004334022369462046FFF7A6F90EE4000053
:10B5C00026050020000B0020FE4B014602221846F3
:10B5D00024F02ABF38B5FB4C0246A41C042369465C
:10B5E0002046FFF791F90AE4F64B01469B1C042222
:10B5F000184624F019BF38B5F24C0246A41D0423A6
:10B6000069462046FFF780F934E4EE4B01469B1D66
:10B610000422184624F008BF38B5EA4C02460A3422
:10B62000042369462046FFF76FF923E4E54B014602
:10B630000A330422184624F0F7BE1CB500EB800044
:10B6400000F64C300A4640F0005005236946FFF7EB
:10B650005BF91CBD00EB800000F64C3040F0005060
:10B66000052224F0E1BE38B5D64C0246223404232C
:10B6700069462046FFF748F90DE4D24B01462233D4
:10B680000422184624F0D0BE38B5CE4C02462634EB
:10B69000012369462046FFF737F90DE4C94B0146FF
:10B6A00026330122184624F0BFBE40F6663208B5A4
:10B6B00002EB80000A4640F0005004236946FFF781
:10B6C00023F908BD40F6663202EB800040F00050DE
:10B6D000042224F0A9BE1CB500EB800001EB81011F
:10B6E00000EB810000F6653040F00050052369460C
:10B6F000FFF70AF91CBD00EB800001EB810100EBB4
:10B700008100134600F6653040F0005005221946CE
:10B7100024F08ABE1CB500EB800001EB810100EB38
:10B72000810000F6C93040F0005005236946FFF75C
:10B73000EBF81CBD00EB800001EB810100EB810008
:10B74000134600F6C93040F000500522194624F097
:10B750006BBE40F61E5208B502EB80000A4640F070
:10B76000005004236946FFF7CFF808BD40F61E528B
:10B7700002EB800040F00050042224F055BE38B5A2
:10B78000914C0246012369462046FFF7BDF80AE4C2
:10B790008D4B01460122184624F046BE38B58A4C2E
:10B7A0000246641C042369462046FFF7ADF80BE40B
:10B7B000854B01465B1C0422184624F035BE38B583
:10B7C000814C0246641D042369462046FFF79CF81D
:10B7D0000BE47D4B01465B1D0422184624F024BE79
:10B7E00038B5794C02460934042369462046FFF7F0
:10B7F0008BF80BE4744B014609330422184624F0FD
:10B8000013BE38B5704C02460D34042369462046F9
:10B81000FFF77AF80BE46C4B01460D33042218460F
:10B8200024F002BE38B5684C024611340223694642
:10B830002046FFF769F80BE4634B014611330222FF
:10B84000184624F0F1BD38B55F4C0246133402238C
:10B8500069462046FFF758F80BE45B4B014613336B
:10B860000222184624F0E0BD38B5574C0246153484
:10B87000012369462046FFF747F80BE4524B014687
:10B8800015330122184624F0CFBD2DE9F8430422D8
:10B890006946002020F036FE4C4C00060FD44C497F
:10B8A000009882274B4D4C4E4FF0190888420DD11D
:10B8B00004226946104620F025FE000602D52068C5
:10B8C000BDE8F88345490098884206D0276078464D
:10B8D000C5F8008030608220F2E7002020602860F8
:10B8E000784630600020EBE72DE9F043374EDFF873
:10B8F000E480DFF8E49091B000254FF40057002475
:10B900006119684600F0FAF820226946204620F0C6
:10B910000FFF00060ED42034BC42F1D3002461197D
:10B92000684600F0EBF8202208A9204620F0EAFD46
:10B93000000603D5306811B0BDE8F083202208A9C5
:10B94000684635F081FF40B1822019213060C8F887
:10B9500000107946C9F80010EDE72034BC42DED370
:10B96000ED1DFF2DCBD9002030607946C8F80000CE
:10B97000C9F80010DFE770B58CB000208DF8240006
:10B9800013480A9024226946042020F0BBFD0F4D85
:10B99000000626D4FFF7A8FF000622D400244FF4A7
:10B9A0000056012209A9204620F0C2FE000618D444
:10B9B000641CB442F5D324226946042020F0B8FE6A
:10B9C00000060DE0430B0020620D002008C0072098
:10B9D0009CE634960CC0072010C00720CEFAADDEDE
:10B9E00002D528680CB070BD04220AA9002020F0FE
:10B9F0009FFEF7E738B504466946002008F0EFF8E7
:10BA00000106434801D5006815E4BDF8001001B1F6
:10BA100001212170002101603E48016078463E49C5
:10BA20000860002007E4FF2008F013BA10B588B0C2
:10BA30006846C11D06F088F8354C00060BD40DF1A0
:10BA40000E00FEF79DFA000605D40DF11500FEF775
:10BA500097FA000602D5206808B010BD6846FEF7C8
:10BA6000E9FFF9E738B5FEF770FF294C48B368469F
:10BA7000FFF7C0FF00061FD49DF80000F0B1702052
:10BA800013F085FD000617D4712013F080FD000629
:10BA900012D46F2013F07BFD00060DD4FFF7C6FF14
:10BAA000000609D4722013F072FD000604D46F2042
:10BAB00013F06DFD000604D52068E2E4FFF7B6FF41
:10BAC000F8E71449002020600860784612490860B1
:10BAD0000020D6E400B589B01E226946D00624F0C5
:10BAE000A3FC000604D50A48008880B209B000BD56
:10BAF0001C210DF10200FBF77FFFF7E75FF000026A
:10BB000000F8011B491C521C202AF9D37047000081
:10BB100008C007200CC0072010C007207FB50546CD
:10BB200003A8FEF7C3FF264C000640D49DF80C0086
:10BB3000012832D00026022809D087202060214821
:10BB40000660784620490860872004B070BD002058
:10BB500005F048FA00062AD42888ADF80400688861
:10BB6000ADF8060028798DF808008DF8096001A865
:10BB700004F078F900061AD469462B2013F0B2FEBF
:10BB8000000614D411489DF800100078C90704D0AD
:10BB9000012802D001208DF80C0003A8FEF78DFFCC
:10BBA000000604D4284601F0FDFC000601D52068FB
:10BBB000CBE703208DF80C0003A8FEF76DFFC4E768
:10BBC00008C007200CC0072010C007207602001014
:10BBD00038B504466846FEF769FF01060A4801D5F4
:10BBE000006838BD9DF80010032909D08721016045
:10BBF000064900200860784605490860872038BD5E
:10BC0000204601F009FF38BD08C007200CC00720FE
:10BC100010C0072038B504466846FEF747FF010606
:10BC20000A4801D5006838BD9DF80010032909D0E5
:10BC300087210160064900200860784605490860B0
:10BC4000872038BD204601F0DDFF38BD08C0072041
:10BC50000CC0072010C0072038B504466846FEF720
:10BC600025FF01060A4801D5006838BD9DF800107F
:10BC7000032909D087210160064900200860784621
:10BC800005490860872038BD204602F06FF838BDAE
:10BC900008C007200CC0072010C0072038B5044694
:10BCA0006846FEF703FF01060A4801D5006838BD63
:10BCB0009DF80010032909D0872101600649002062
:10BCC0000860784605490860872038BD204602F0A4
:10BCD0002BF938BD08C007200CC0072010C0072072
:10BCE00038B504466846FEF7E1FE01060A4801D56C
:10BCF000006838BD9DF80010032909D08721016034
:10BD0000064900200860784605490860872038BD4C
:10BD1000204602F0BDF938BD08C007200CC007203E
:10BD200010C0072038B504466846FEF7BFFE01067E
:10BD30000A4801D5006838BD9DF80010032909D0D4
:10BD4000872101600649002008607846054908609F
:10BD5000872038BD204602F077FA38BD08C007209A
:10BD60000CC0072010C0072038B504466846FEF70F
:10BD70009DFE01060A4801D5006838BD9DF80010F7
:10BD8000032909D087210160064900200860784610
:10BD900005490860872038BD204602F0E9FA38BD21
:10BDA00008C007200CC0072010C0072038B5044683
:10BDB0006846FEF77BFE01060A4801D5006838BDDB
:10BDC0009DF80010032909D0872101600649002051
:10BDD0000860784605490860872038BD204602F093
:10BDE0007FFB38BD08C007200CC0072010C007200B
:10BDF00038B504466846FEF759FE01060A4801D5E3
:10BE0000006838BD9DF80010032909D08721016022
:10BE1000064900200860784605490860872038BD3B
:10BE2000204602F0F1FB38BD08C007200CC00720F7
:10BE300010C0072038B56846FEF738FE0E4C0006E5
:10BE400011D49DF80000032809D087200B492060F9
:10BE50000020086078460A490860872038BD02F053
:10BE60008BFC000601D5206838BD04208DF8000049
:10BE70006846FEF711FE38BD08C007200CC0072039
:10BE800010C007202DE9FE43294C00262068822897
:10BE900000D001266846FEF709FE00063AD49DF858
:10BEA00000001D280DD101A800F04AF8000631D489
:10BEB0002048018821F00201018000F0A5FE000663
:10BEC00028D49DF8000000251B4FDFF87080032860
:10BED0000DD004280BD00E2809D01B2807D08720AE
:10BEE000206079463D60C8F80010BDE8FE83002060
:10BEF00002F084FC00060DD49DF800001B280BD036
:10BF00006846FEF7E4FD000604D46846FEF7C4FD6B
:10BF1000000601D52068E8E716B101200AF082FE8C
:10BF2000256079463D600020C8F80010DDE700007C
:10BF300008C00720020000100CC0072010C0072016
:10BF40002DE9F04796B0824613A8FEF7AFFD504C9E
:10BF5000000654D49DF84C10002505264D4FDFF8FF
:10BF600038810DF13C0904290AD01D2948D08720C9
:10BF7000206079463D60C8F8001016B0BDE8F08733
:10BF800014A9504602F085FD20B192282AD09328AA
:10BF900075D123E09DF85000002873D03F48007809
:10BFA00000286FD01D208DF84C0013A8FEF774FDFB
:10BFB000000664D44846FFF74CF800065FD412A888
:10BFC000FFF758F800065AD40AF015FB60B3256055
:10BFD00079463D600020C8F80010CEE7F8F736F942
:10BFE0000E2005E03868312849D1F8F72FF91620DE
:10BFF0008DF84C0013A8FEF74FFDF8F73CF93EE032
:10C000000DA806F018F8000639D412A90F9806F00A
:10C0100069FA000633D44846FFF711F800062ED41B
:10C0200012A8FFF71DF8CDE70C208DF801000F983E
:10C03000CDF802001298CDF80600684607F0ECF93A
:10C0400000061CD4684608F069FB000617D4FEF70A
:10C050002EFC18B1FEF7FFFA000610D4684607F070
:10C0600006FA00060BD4684608F090FB000606D4DA
:10C07000FEF71DFC28B1FEF7FAFA000602D520688B
:10C080007BE7FFE78DF84C6013A8FEF705FD74E72A
:10C0900008C007200CC0072010C00720084400007B
:10C0A00070B586B005460E4603A8FEF7FFFC2D4C82
:10C0B00000064ED49DF80C001D280DD104A8FFF7F2
:10C0C0003FFF000645D42848018821F00201018085
:10C0D00000F09AFD00063CD49DF80C1001292DD0EB
:10C0E0000020022909D08721216020490860784674
:10C0F0001F490860872006B070BD2988ADF804107C
:10C100006988ADF8061029798DF808108DF80900B6
:10C1100001A803F0A7FE00061BD469462B2013F0EC
:10C12000E1FB000615D413489DF800100078C907FC
:10C1300004D0012802D001208DF80C0003A8FEF7DE
:10C14000BCFC000605D43146284603F023F900065E
:10C1500001D52068CFE706208DF80C0003A8FEF774
:10C160009BFCC8E708C00720020000100CC0072095
:10C1700010C007207602001038B56846FEF796FC1E
:10C180000F4C000616D49DF80000062809D0872021
:10C190000C4920600020086078460B490860872021
:10C1A00038BD03F079F9000604D46846FEF78FFC29
:10C1B000000601D5206838BD6846FEF76DFC38BD25
:10C1C00008C007200CC0072010C0072038B505465E
:10C1D0006846FEF76BFC0F4C000612D49DF8000079
:10C1E000062809D087200C49206000200860784686
:10C1F0000A490860872038BD284603F085F9000603
:10C2000001D5206838BD07208DF800006846FEF78C
:10C2100043FC38BD08C007200CC0072010C0072011
:10C2200038B504466846FEF741FC01060B4801D5C7
:10C23000006838BD9DF8001004290BD0062909D0EC
:10C24000872101600649002008607846054908609A
:10C25000872038BD204603F099FA38BD08C0072072
:10C260000CC0072010C0072038B504466846FEF70A
:10C270001DFC01060B4801D5006838BD9DF8001073
:10C2800004290BD0062909D0872101600649002026
:10C290000860784605490860872038BD204603F0CD
:10C2A00037FB38BD08C007200CC0072010C007208E
:10C2B00038B504466846FEF7F9FB01060B4801D580
:10C2C000006838BD9DF8001004290BD0062909D05C
:10C2D000872101600649002008607846054908600A
:10C2E000872038BD204603F0C5FB38BD08C00720B5
:10C2F0000CC0072010C0072038B505466846FEF779
:10C30000D5FB124C000617D49DF80000022809D076
:10C3100087200F4920600020086078460D4908609A
:10C32000872038BD002004F05DFE000604D42846B6
:10C3300003F098FD000601D5206838BD01208DF876
:10C3400000006846FEF7A8FB38BD000008C00720C3
:10C350000CC0072010C0072038B505466846FEF718
:10C36000A5FB1F4C000632D49DF8000010281FD0FA
:10C370000CDC0C281CD004DC012819D002280DD1BB
:10C3800016E00D2814D00E2808D111E013280FD084
:10C3900014280DD015280BD0182809D08720114952
:10C3A00020600020086078460F490860872038BD6B
:10C3B0006846FEF782FB000609D46846FEF78EFB4E
:10C3C000000604D4284608F087FB000601D5206843
:10C3D00038BD08208DF800006846FEF75DFB38BDCB
:10C3E00008C007200CC0072010C007202DE9F0412D
:10C3F00086B002A8FEF75AFB504C00067ED49DF88A
:10C40000080001274E4E0025082807D0092805D02E
:10C410000A2874D0872006B0BDE8F08108F006FC39
:10C42000009031684FF00A080191042821D005DC02
:10C4300048B1012809D0032829D118E0052802D0E5
:10C44000822824D11FE0009560E06846FFF7C2F81B
:10C45000000670D401A8FFF7CEF800066BD48DF863
:10C46000088002A8FEF718FB000664D44EE00820FE
:10C4700000E009208DF8080002A8FEF70DFB0090EF
:10C480003068019042E003290DD004290BD009F057
:10C490007FFF03A8FFF75BF800064CD49DF80C0063
:10C4A0000E2803D011E005F02DFC2FE004A9622036
:10C4B00013F018FA00063ED49DF81000C00704D00F
:10C4C0000120F8F7EDFD000635D40098822801D050
:10C4D000922801D105F016FC6846FFF77BF80006AC
:10C4E00029D401A8FFF787F8000624D49DF8080096
:10C4F00009280BD08DF8088002A801E01BE00DE0B0
:10C50000FEF7CAFA15E000BFCDE90075009820607B
:10C510000199316079460B4A11607CE78120CDE9B1
:10C5200000056846FFF756F8000604D401A8FFF797
:10C5300062F80006E8D520686DE7000008C0072013
:10C540000CC0072010C007202DE9F04186B003A8D9
:10C55000FEF7FDFF364C000660D402A8FEF7A6FAEF
:10C5600000065BD401A8FFF73FF8000656D404A8E4
:10C57000FFF74BF8000651D49DF8080087272D4D92
:10C580002D4E4FF000080A2801D0092835D109F0B6
:10C59000C7FA000642D401980128684608D0FEF781
:10C5A00096FA00063AD49DF80800092805D013E051
:10C5B000FEF79EFA000631D414E00198922801D0CB
:10C5C000822802D113208DF800009DF80C00142859
:10C5D00002D10C208DF800000198932802D10E2082
:10C5E0008DF800006846FEF757FA000616D49DF84D
:10C5F0000800092814D00A2808D027607846C5F812
:10C6000000803060872006B0BDE8F0819DF80C0006
:10C610000E2805D1F9F7FCFF000601D52068F2E7E6
:10C62000019820600499296079463160EBE70000A9
:10C6300008C007200CC0072010C0072038B50546E9
:10C640006846FEF733FA164C00061FD49DF800002A
:10C650000C2809D087201349206000200860784604
:10C6600011490860872038BD6846FEF726FA0006A3
:10C670000CD40D208DF800006846FEF72FFA000656
:10C6800004D4284603F0B4FC000601D5206838BD68
:10C6900008208DF800006846FEF7FEF938BD00005E
:10C6A00008C007200CC0072010C00720F0B585B0D7
:10C6B00001A807F0CCFA344C000655D46846FEF7C2
:10C6C000F5F9000650D49DF8000002252F4E304F9A
:10C6D00013281ED00CDC0D281BD004DC012818D038
:10C6E00002280DD115E00E2813D0102808D143E000
:10C6F00014280ED015280CD018280AD01B283BD09F
:10C70000872020600020306078463860872005B0A0
:10C71000F0BD012004F066FC000625D404A804F056
:10C7200001F9000622D59DF81000E8B1012809D0D2
:10C73000022810D0882020600920306078463860B8
:10C740008820E4E7F7F782FD18208DF8000006E066
:10C75000F7F791FD08E0F7F779FD8DF8005068468E
:10C76000FEF79AF90006F3D52068D0E78DF800505F
:10C770006846FEF791F9CAE7922020607846356056
:10C7800038609220C3E7000008C007200CC00720D3
:10C7900010C007202DE9F04385B0814602A807F0BC
:10C7A00056FA2C4C000645D40620F9F74EF82A4DCF
:10C7B0002A4E38B90420F9F748F818B90120F9F7DA
:10C7C00044F880B16846FEF771F9000632D49DF84E
:10C7D000000000274FF0870802280ED00D2817D040
:10C7E000182829D114E091202060B12028607846D3
:10C7F0003060912005B0BDE8F08301A8FFF7FAF89A
:10C80000000617D416499DF804000978084213D190
:10C8100001A9484603F024FEA8B19DF8040048B1E0
:10C82000F7F714FD18208DF800006846FEF734F97C
:10C83000F7F721FD2068DDE7C4F8008078462F6017
:10C8400030608720D6E702208DF800006846FEF7AA
:10C8500023F9CFE708C007200CC0072010C007202D
:10C8600008440000F8B506466846FEF71FF9504C2C
:10C87000000650D49DF800004E4D132812D004DC61
:10C8800001280FD00E2804D10CE015280AD01B284F
:10C8900008D087202060002028607846464908603C
:10C8A0008720F8BDF9F7A5FA93281ED06846FEF751
:10C8B00004F900062FD49DF800001B2819D002208F
:10C8C0008DF800006846FEF709F9000623D4012020
:10C8D00004F088FB00061ED4304609F07FF950B101
:10C8E0008F280FD0922816D117E0F7F7AFFC0E2053
:10C8F00019E01020E4E708208DF800006846FEF7F4
:10C90000CBF8F8BDF7F7A2FC2868072801D114205E
:10C9100009E0F7F7B0FC2068F8BDF7F797FC286846
:10C920003128F6D116208DF800006846FEF7B4F8DD
:10C93000EFE72DE9FC4101A8F8F72BFB1C4C0006A2
:10C940000BD4BDF804001B4E1B4F002540B16946B7
:10C95000622012F0C7FF000609D52068BDE8FC81FF
:10C96000812020607846356038608120F6E79DF8A8
:10C970000000800703D5002110A027F0F9FDF8F78B
:10C980000DFB30B1F7F762FC09F002FDF7F773FC1D
:10C99000E3E70F48018841F00201018001200AF01D
:10C9A00041F925607846356038600020D6E7000000
:10C9B00008C007200CC0072010C007208493818B7B
:10C9C000888A809220848E8A938C858D92800A003A
:10C9D00002000010F8B506460D466846FEF766F8F8
:10C9E0001C4C00062DD49DF80020132A19D008DC19
:10C9F000012A16D0022A14D00E2A12D0102A06D1EB
:10CA00000FE0142A0DD0152A0BD0182A09D0872040
:10CA1000114920600020086078461049086087208E
:10CA2000F8BD6846FEF749F800060AD46846FEF7E6
:10CA300055F8000605D42946304609F099FA000653
:10CA400001D52068F8BD08208DF800006846FEF783
:10CA500023F8F8BD08C007200CC0072010C007202D
:10CA6000F8B506460D466846FEF720F81D4C000650
:10CA700027D49DF800101C4A1C48102911D004DC52
:10CA800002290ED00D2904D10BE0112922D014293E
:10CA900007D087212160002111607946016087203D
:10CAA000F8BD6846FEF709F800060AD46846FEF7A6
:10CAB00015F8000605D42946304609F015FB000696
:10CAC00001D52068F8BD08208DF800006846FDF704
:10CAD000E3FFF8BD91212160A92111607946016031
:10CAE0009120F8BD08C007200CC0072010C0072007
:10CAF0003EB501A8FDF7C9FF214C00063ED46846AB
:10CB0000FDF7D4FF000639D402A901201DF082F9F7
:10CB1000000633D49DF800001A4D022806D00E28D6
:10CB200004D0102802D00298C00705D004F08CF879
:10CB300080B1922822D114E09DF804208721124868
:10CB400021600AB1042100E00021296079460160DA
:10CB500087203EBD10208DF800006846FDF79CFF41
:10CB60003EBD2868312809D1F7F770FB16208DF8F3
:10CB700000006846FDF790FFF7F77DFB20683EBD9B
:10CB800008C007200CC0072010C0072038B5054694
:10CB90006846FDF78BFF184C00061DD49DF8000079
:10CBA000112809D0872015492060002008607846A8
:10CBB00013490860872038BD1248296801606968F8
:10CBC0004160A9688160342012F0E1FC000603D4C2
:10CBD00027F09AFE000601D5206838BD284607F0E8
:10CBE00071FB10B109F0D4FBF6E702208DF80000CC
:10CBF0006846FDF751FF38BD08C007200CC007206C
:10CC000010C0072092C707202DE9FC416846FDF7B8
:10CC10004DFF194C000622D49DF800000025174E48
:10CC2000174F052809D01D2820D08720206078467E
:10CC3000356038608720BDE8FC8101A90120FEF73E
:10CC400006F800060BD404F0C1F8000607D4012052
:10CC50008DF800006846FDF71FFF000601D520682B
:10CC6000E9E7019800B1012009F052FC25607846FF
:10CC7000356038600020DEE708C007200CC00720C0
:10CC800010C0072038B56846FDF710FF0E4C0006AF
:10CC900011D49DF80000072809D087200B49206097
:10CCA0000020086078460A490860872038BD04F0F3
:10CCB000B5F8000601D5206838BD01208DF80000C8
:10CCC0006846FDF7E9FE38BD08C007200CC0072004
:10CCD00010C0072038B504466846FDF7E7FE010698
:10CCE0000A4801D5006838BD9DF80010032909D015
:10CCF00087210160064900200860784605490860E0
:10CD0000872038BD204604F00FFA38BD08C0072040
:10CD10000CC0072010C0072038B504466846FDF750
:10CD2000C5FE01060A4801D5006838BD9DF800100F
:10CD3000032909D087210160064900200860784650
:10CD400005490860872038BD204604F065FA38BDE3
:10CD500008C007200CC0072010C0072038B50446C3
:10CD60006846FDF7A3FE01060A4801D5006838BDF4
:10CD70009DF80010032909D0872101600649002091
:10CD80000860784605490860872038BD204604F0D1
:10CD9000BBFA38BD08C007200CC0072010C0072010
:10CDA00038B504466846FDF781FE0106204801D5E6
:10CDB000006838BD9DF8001001290BD0022909D068
:10CDC000872101601B490020086078461A490860E5
:10CDD000872038BD204604F015FC38BD38B5044620
:10CDE0006846FDF763FE0106114801D5006838BDAD
:10CDF0009DF8001001290FD0032910D004290ED06E
:10CE000005290CD0872101600A4900200860784676
:10CE100009490860872038BD0121204605E009F056
:10CE200011FB27F071FD0021084604F065FC38BDB8
:10CE300008C007200CC0072010C007202DE9F843C8
:10CE40008046694601201CF0E5FF104C00060DD419
:10CE500000980F4E0F4FC0074FF0000509D0002279
:10CE60000121404604F0D4FC000609D52068BDE845
:10CE7000F883872020607846356038608720F6E7A1
:10CE800025607846356038600020F0E708C007204C
:10CE90000CC0072010C0072038B504464FF00040F2
:10CEA000FDF78CFB000602D51648006838BD204609
:10CEB000FDF77DFE00061FD4A01CFDF789FE0006CD
:10CEC0001AD4201DFDF795FE000615D409F066FF63
:10CED000000602D509F05CFA0EE06846FDF73EFE5A
:10CEE000000609D46846FDF701FA000604D4684636
:10CEF000FDF72AFE000602D5FDF75BFC38BDFDF705
:10CF0000C3FB38BD08C007202DE9F04188B001A857
:10CF1000FDF7BBFD384C00065ED49DF80400374F8A
:10CF2000374E48B1912020609C20306078463860B0
:10CF3000912008B0BDE8F08106A901201CF06AFF2D
:10CF4000000649D406984FF00005C00746D0684651
:10CF5000FDF7ACFD00063FD46846FDF7AEFD0006C8
:10CF60003AD46846FDF7BAFD000635D408208DF89E
:10CF700000006846FDF790FD00062DD44FF0010833
:10CF80008DF8088002A8FEF7D8FA000624D4032002
:10CF90008DF80C0003A8FDF7C6FD00061CD4194946
:10CFA0000220087014482560FEF714FB000613D415
:10CFB00013483560FEF71FFB00060DD4ADF8108056
:10CFC00004A8FEF7E1FA000606D4ADF8145005A84F
:10CFD000FEF7EBFA000608D52068AAE78720206054
:10CFE0007846356038608720A3E72560784635604D
:10CFF000386000209DE7000008C0072010C007200F
:10D000000CC00720000000102DE9FF4706466846C7
:10D0100003F0B1FFA24C000665D4BDF800004FF448
:10D02000B46148433178C1EB011100EB81007178A4
:10D03000451802A8FEF7DEFC000654D403A8F9F751
:10D04000F1FB00064FD49DF80C00E8B395499DF81C
:10D050000800DFF854920978DFF850A208424FF038
:10D0600086074FF0170817D06946022005F07BF8B5
:10D07000000638D401A9032005F075F8000632D463
:10D08000BDF80000BDF80410C0EB001000EB40003C
:10D0900001EB4010854215D36846FEF7F3F9000610
:10D0A00021D401A8FEF7FEF900061CD4BDF800004B
:10D0B000BDF80410C0EB001000EB400001EB401085
:10D0C00085420BD2276000E008E07946C9F800806D
:10D0D0008620CAF8001004B0BDE8F08730461DF085
:10D0E00071FC000601D52068F5E703F0F3FFF2E7D5
:10D0F0002DE9FF4781466946532012F0F3FB684C47
:10D10000000629D49DF8000000F004008DF800000E
:10D1100001A8FDF7CBFC00061ED49DF80400624D6B
:10D12000624E0027DFF88881102817D009DC02281A
:10D1300014D00D2819D091210E287DD00F2806D1AA
:10D140009AE011280AD0192815D01A2813D003A85C
:10D15000F9F768FB000670D52068BCE74846FFF782
:10D1600053FF05E088F800700FE048461DF02AFCE8
:10D170000006F1D4F6E74846FFF746FF0028EBD15A
:10D1800098F80000C246022805D0276078462F6034
:10D19000306000209FE79DF8000020B14D2012F084
:10D1A000F6F90006D8D448461DF0A7FB0006D3D4F4
:10D1B000404999F8028088683F4A8B681B1A93425D
:10D1C000FBD348461DF099FB0006C5D499F8021020
:10D1D000414507D1822020600520286078463060D4
:10D1E000822078E703218AF8001034494FF00108C3
:10D1F00001A881F80080FDF77BFC0006ACD401A8F3
:10D20000FDF74AFC0006A7D40420F8F7AFFB0006A0
:10D21000A2D49DF8000020B1012009F003FD000612
:10D220009AD402A9532012F05DFB000694D49DF815
:10D23000080010F0010001E01BE024E08DF8080078
:10D2400008D0012009F0EEFC000685D408F0F6FFB6
:10D25000000681D49DF8080020B1012009F0E2FC0D
:10D26000000686D4C4F8008078462F603060012024
:10D2700031E7A020216001E0D220216028607846BB
:10D280003060912027E79DF80C108720206011B1B5
:10D290000420286000E02F607846306087201AE77D
:10D2A00008C00720084400000CC0072010C0072059
:10D2B000CE01001000800040E0C8100020C0072010
:10D2C0002DE9FE43054601A8FEF794FBAB4C000692
:10D2D0002BD49DF80400AA4EAA4F4FF086084FF0B9
:10D2E0001A09A8B1A848007848B16946022004F09C
:10D2F0003AFF000619D4BDF8000085421CD36846E9
:10D30000F8F78AFC000610D4BDF80000854213D35C
:10D3100002A8F9F787FA000607D49DF8080098B12B
:10D320006846FEF7AFF8000602D52068BDE8FE8328
:10D33000BDF80000854207D2C4F800807846C6F8E0
:10D34000009038608620F1E7002020603060784649
:10D3500038600020EAE72DE9F14F88B000278DF80A
:10D36000047003A90898F7F7B1FBBDF80C0048F268
:10D370006901834D834E814C401E4FF086094FF06A
:10D38000140A884205D300BFC4F80090C5F800A075
:10D390005EE001A9532012F0A5FA00067ED49DF8A4
:10D3A000040000F004008DF804006846FDF77EFBE1
:10D3B0000006F3D49DF80000102820D009DC0228D4
:10D3C0001DD00D281BD091210E2868D00F2808D120
:10D3D00098E0112813D0192811D01A280FD01C2832
:10D3E0000DD006A8F9F71EFA000657D49DF81810BC
:10D3F0008720002920607CD0042028608AE0BDF8C6
:10D400000C00FFF75DFFDFF8848138B3862845D133
:10D4100088F800709DF800001C2810D01A283DD014
:10D4200019283BD06846FDF748FB000636D41C207F
:10D430008DF800006846FDF72FFB00062ED4022071
:10D44000F8F781FA000629D41A20C4F80090286061
:10D4500078463060862009B0BDE8F08F02A81DF044
:10D460007DFA00064FF0010B07D54FF4FA60ADF8D6
:10D4700008008DF80AB08DF80BB005A902A8F7F7DF
:10D4800025FBBDF80C10BDF8140098F8002081426F
:10D49000404610D9012A08D0418001E05EE02EE02C
:10D4A00088F800B0C4F800B062E042888A4204D034
:10D4B00088F8007068E7012AF7D008981DF0A3FAF1
:10D4C00000064BD44FF0020988F800909DF8040044
:10D4D00048B13A2012F05BF800063FD4012009F071
:10D4E000A1FB00063AD40220F8F740FA000635D432
:10D4F00000E00EE09DF800001C280FD018E0A020EE
:10D50000216001E0D22021602860784630609120BF
:10D51000A1E72F607846306087209CE76846FDF7DA
:10D52000D6FA00061AD46846FDF7B6FA000615D4F6
:10D5300003F0D0FD9DF80000192807D01A2805D067
:10D54000276078462F603060002084E79DF8040053
:10D5500050B13E2012F01BF8000601D520687AE792
:10D5600000210BA027F004F888F80090C4F800B060
:10D5700078462F60306001206DE7000008C007206A
:10D580000CC0072010C0072008440000CE01001086
:10D59000200A200A200A200A200A200A200A200A3B
:10D5A00000000000F0B5054641799E4C9E4F9F4E0D
:10D5B0008DB0862009B1042902D92060062005E03B
:10D5C000297909B11E2907D92060052038607846DD
:10D5D000306086200DB0F0BD6988288803F062FCB9
:10D5E00000067DD468796946FDF797FD000677D47B
:10D5F000BDF800100020A1F57F42FF3A71D0064629
:10D6000000906846FDF7D0FB000669D46846FEF737
:10D6100003F8000664D4012769463846FDF7F7FB96
:10D6200000065DD47F1CFFB2112FF5D36846FDF7CD
:10D6300018FC00067ED46846FDF724FC000679D469
:10D64000012769463846FDF7F6FA000672D47F1CBA
:10D65000FFB20B2FF5D3012769463846FEF779F85C
:10D66000000667D47F1CFFB2112FF5D36846FDF783
:10D67000B4FD00065ED46846FDF7D4FD000659D41B
:10D680006846FDF7ECFA000654D46846FDF709FB3E
:10D6900000064FD46846FDF7BDFA00064AD40127BC
:10D6A000009669463846FEF700F8000642D47F1C13
:10D6B000FFB2052FF5D9ADF800606846FDF785FB90
:10D6C000000637D46846FDF791FB000632D4684661
:10D6D000FDF7D6FA00062DD46846FDF7F3FA01E00F
:10D6E00028E029E0000625D4009601266946304648
:10D6F000FDF7A1FB00061DD4761CF6B2112EF5D362
:10D700002846FDF754FA000614D4A81CFDF760FA69
:10D7100000060FD4281DFDF76CFA00060AD401207C
:10D7200009F080FA000605D44FF00040FCF746FFF0
:10D73000000608D520684DE78B21216038607846C7
:10D740003060084646E701248DF800406846FDF742
:10D75000EAF9000633D436480470681DFDF713FB60
:10D7600000062CD46846FDF7F9F9000627D4684670
:10D77000FCF7BCFD000622D46846FDF7E5F900067B
:10D780001DD46846FDF7FBF9000618D46846FCF77F
:10D7900086FD000613D46846FDF7E7F900060ED4AF
:10D7A0006846FDF7FDF9000609D46846FCF79EFDC2
:10D7B000000604D46846FDF7E9F9000602D5FCF737
:10D7C000F8FF07E708F084FE000624D48DF8014036
:10D7D00068798DF8020006F0E9FE00061BD4684661
:10D7E00005F01AFE000616D4684606F097FF0006FC
:10D7F00011D4FCF730FF00060DD4684605F037FE63
:10D80000000608D4684606F0C1FF000603D4FCF702
:10D810002EFF000602D508F0BBFDD0E7FCF734FF71
:10D82000D8E6000008C007200CC0072010C0072061
:10D830000000001070B5057A724E94B00446102DA9
:10D840000AD98620704930600320086078466F4905
:10D850000860862014B070BD0DB90125257260687E
:10D860000E9021460EA8FCF7BAFC000605D44FF036
:10D870000040FCF7A3FE000601D53068EAE76846E1
:10D88000FDF79CFA000652D40EA96846FCF7DEFAB2
:10D8900000064CD46846FDF787FA000647D4684670
:10D8A000FDF79DFA000642D4BDF80000401CADF81B
:10D8B00000006846FDF789FA000638D46946284614
:10D8C000FDF7B1FA000632D40EA96846FCF7BEFA9D
:10D8D00000062CD469462846FDF799FA000626D49E
:10D8E00069462846FDF7B4FA000620D4214668466A
:10D8F000FCF7E6FA00061AD469462846FDF79BFABB
:10D90000000614D404F10800FDF7CDFA00060ED489
:10D910002046FDF7D9FA000609D4201DFDF7E5FAE7
:10D92000000604D40EA8FDF7F1FA000602D5FCF7B4
:10D9300040FF8FE7012026F0ADFB000658D409F028
:10D94000ABF8000654D40D208DF80500207A8DF830
:10D9500013006068CDF807002068CDF80B000E9822
:10D96000CDF80F002A4905A833F09AFF0DF1060003
:10D97000FDF713FA00063BD401A805F04DFD0006A3
:10D9800036D401A806F0CAFE000631D4012006F004
:10D9900060FA00062CD46846FEF72CF8000627D45F
:10D9A0009DF8000090B11B48007878B110A8FDF7F1
:10D9B000F4F900061CD48DF84C50206811900E9894
:10D9C000129010A804F088FF000611D4FCF743FE63
:10D9D00000060DD401A805F04AFD000608D401A8F0
:10D9E00006F0D4FE000603D4FCF741FE000602D583
:10D9F00008F0CEFC9BE7064900200870FCF744FEC7
:10DA000028E7000008C007200CC0072010C007202E
:10DA1000D0C707200844000070B5057A744E94B052
:10DA20000446102D0AD98620724930600320086010
:10DA3000784671490860862014B070BD05B901258B
:10DA400060680E9021460EA8FCF7C9FB000605D4BD
:10DA50004FF00040FCF7B2FD000601D53068EBE75F
:10DA60006846FDF7ABF9000662D40EA96846FCF7DC
:10DA70000EFA00065CD46846FDF796F9000657D406
:10DA80006846FDF7BDF9000652D4BDF80000401C01
:10DA9000ADF800006846FDF7A9F9000648D46846CD
:10DAA000FDF7C4FD000643D40EA96846FCF7CEF985
:10DAB00000063DD46846FDF7AFFD000638D4694640
:10DAC0002846FDF7B0F9000632D40EA96846FCF7E7
:10DAD000DEF900062CD469462846FDF798F90006C1
:10DAE00026D469462846FDF7B3F9000620D421461E
:10DAF0006846FCF706FA00061AD469462846FDF780
:10DB00009AF9000614D404F10800FDF7CCF90006D8
:10DB10000ED42046FDF7D8F9000609D4201DFDF7E4
:10DB2000E4F9000604D40EA8FDF7F0F9000602D5CA
:10DB3000FCF73FFE80E708F08FFF00064FD40E2071
:10DB40008DF80500207A8DF813006068CDF8070085
:10DB50002068CDF80B000E98CDF80F00274905A8D6
:10DB600033F09EFE0DF10600FDF717F9000636D4DE
:10DB700001A805F051FC000631D401A806F0CEFD45
:10DB800000062CD46846FDF735FF000627D49DF823
:10DB9000000090B11A48007878B110A8FDF7FDF8A0
:10DBA00000061CD48DF84C50206811900E981290ED
:10DBB00010A804F0E1FE000611D4FCF74CFD0006AD
:10DBC0000DD401A805F053FC000608D401A806F006
:10DBD000DDFD000603D4FCF74AFD000602D508F07F
:10DBE000D7FBA5E7054900200870FCF74DFD23E7AA
:10DBF00008C007200CC0072010C00720D0C707208E
:10DC00000844000030B504460079544D8FB008B187
:10DC100010280AD9862052492860032008607846D7
:10DC20005049086086200FB030BD4FF00040FCF72F
:10DC3000C5FC000601D52868F5E76846FDF7BEF883
:10DC4000000636D421466846FCF721F9000630D498
:10DC50006846FDF7A9F800062BD420796946FDF740
:10DC6000E2F8000625D421466846FCF710F90006C4
:10DC70001FD420796946FDF7CAF8000619D4201D83
:10DC8000FDF788F9000614D42046FDF772F9000666
:10DC90000FD46846FDF7AAFA00060AD42146684662
:10DCA000FCF7D4F8000604D46846FDF796FA00069F
:10DCB00002D5FCF77EFDB6E708F0AEFE000647D4BD
:10DCC00008208DF805000025CDF806500DF10B0059
:10DCD000FDF737F900063BD46846FDF743F9000627
:10DCE00036D4BDF80000ADF80C008DF80A5020685D
:10DCF000CDF80E0001A805F08FFB000628D401A87E
:10DD000006F00CFD000623D46846FDF773FE0006FE
:10DD10001ED49DF8000048B11348007830B1206847
:10DD20000E900EA804F07BFE000611D4FCF793FCC5
:10DD300000060DD401A805F09AFB000608D401A83E
:10DD400006F024FD000603D4FCF791FC000602D582
:10DD500008F01EFBADE7FCF797FC64E708C007205E
:10DD60000CC0072010C007200844000030B504464E
:10DD70000079694D91B008B110280AD98620674909
:10DD8000286003200860784665490860862011B045
:10DD900030BD4FF00040FCF711FC000601D52868AB
:10DDA000F5E70DA8FDF70AF8000650D421460DA8A6
:10DDB000FCF74CF800064AD40DA8FCF7F5FF000666
:10DDC00045D420790DA9FDF72EF800063FD4214651
:10DDD0000DA8FCF73BF8000639D420790DA9FDF712
:10DDE00016F8000633D40EA8FDF7D2FC00062ED498
:10DDF0009DF8380088B10DA9FDF7B8FC000626D4BF
:10DE000021460DA8FCF743F8000620D40DA99DF883
:10DE10003800FDF79EFC000619D40DA8FDF7E6F9C1
:10DE2000000614D421460DA8FCF731F800060ED4E4
:10DE30000DA8FDF7D2F9000609D4201DFDF7AAF8B8
:10DE4000000604D42046FDF794F8000602D5FCF73E
:10DE5000B0FC9CE708F0A0FD000656D404208DF825
:10DE600001000FA94C2011F03DFD00064DD49DF896
:10DE70003C00800702D49DF8380020B9684605F0C0
:10DE8000CBFA000641D49DF83C009DF8381000F014
:10DE90000100401E084204D1684606F03FFC00061F
:10DEA00033D40DA8FDF7A6FD00062ED49DF834004E
:10DEB00048B11C48007830B12068109010A804F0D8
:10DEC000D8FD000621D4FCF7C6FB00061DD49DF842
:10DED0003C00800702D49DF8380020B9684605F060
:10DEE000C6FA000611D49DF83C009DF8381000F0E9
:10DEF0000100401E084204D1684606F047FC0006B7
:10DF000003D4FCF7B4FB000602D508F041FA9EE703
:10DF1000FCF7BAFB3BE7000008C007200CC0072055
:10DF200010C007200844000030B504460079544D65
:10DF30008FB008B110280AD98620524928600320E2
:10DF4000086078465049086086200FB030BD4FF019
:10DF50000040FCF733FB000601D52868F5E768466A
:10DF6000FCF72CFF000636D421466846FBF76EFF0F
:10DF7000000630D46846FCF717FF00062BD4207942
:10DF80006946FCF750FF000625D421466846FBF79A
:10DF90005DFF00061FD420796946FCF738FF0006B4
:10DFA00019D4201DFCF7F6FF000614D42046FCF718
:10DFB000E0FF00060FD46846FDF73EF900060AD4DC
:10DFC00021466846FBF742FF000604D46846FDF789
:10DFD00029F9000602D5FCF7ECFBB6E708F0BCFC1B
:10DFE000000647D407208DF805000025CDF806501F
:10DFF0000DF10B00FCF7A5FF00063BD46846FCF7CB
:10E00000B1FF000636D4BDF80000ADF80C008DF865
:10E010000A502068CDF80E0001A805F0FDF90006B1
:10E0200028D401A806F07AFB000623D46846FDF741
:10E03000E1FC00061ED49DF8000048B113480078AA
:10E0400030B120680E900EA804F040FD000611D4F7
:10E05000FCF701FB00060DD401A805F008FA000644
:10E0600008D401A806F092FB000603D4FCF7FFFADF
:10E07000000602D508F08CF9ADE7FCF705FB64E774
:10E0800008C007200CC0072010C00720084400006B
:10E0900070B504460079684E92B0032508B1102887
:10E0A00009D9862030606548056078466449086073
:10E0B000862012B070BD4FF00040FCF77FFA0006DA
:10E0C00001D53068F5E70DA8FCF778FE000650D4BE
:10E0D00021460DA8FBF7DBFE00064AD40DA8FCF78D
:10E0E00063FE000645D420790DA9FCF79CFE0006CE
:10E0F0003FD421460DA8FBF7CAFE000639D420798B
:10E100000DA9FCF784FE000633D40EA8FDF740FBF2
:10E1100000062ED49DF8380088B10DA9FDF726FB26
:10E12000000626D421460DA8FBF7B1FE000620D438
:10E130000DA99DF83800FDF70CFB000619D40DA8B9
:10E14000FDF77AF8000614D421460DA8FBF79FFED0
:10E1500000060ED40DA8FDF765F8000609D4201DB1
:10E16000FCF718FF000604D42046FCF702FF000667
:10E1700002D5FCF71EFB9CE708F0AEFB000655D469
:10E180008DF801500FA94C2011F0ACFB00064DD4C6
:10E190009DF83C00800702D49DF8380020B96846FD
:10E1A00005F03AF9000641D49DF83C009DF838107E
:10E1B00000F00100401E084204D1684606F0AEFAA5
:10E1C000000633D40DA8FDF715FC00062ED49DF8EB
:10E1D000340048B11B48007830B12068109010A876
:10E1E00004F09EFC000621D4FCF735FA00061DD48D
:10E1F0009DF83C00800702D49DF8380020B968469D
:10E2000005F035F9000611D49DF83C009DF8381052
:10E2100000F00100401E084204D1684606F0B6FA3C
:10E22000000603D4FCF723FA000602D508F0B0F884
:10E230009FE7FCF729FA3CE708C007200CC007203D
:10E2400010C007200844000010B5044690B04FF0FD
:10E250000040FCF7B3F9000603D54348006810B04E
:10E2600010BD0EA8FCF7AAFD000626D40EA8FCF7E8
:10E27000D5FE000621D40E980D9021460DA8FBF77F
:10E2800006FE000619D40DA8FCF78EFD000614D476
:10E290000DA8FCF7F0FD00060FD421460DA8FBF7F2
:10E2A000D5FD000609D40DA8FCF7DBFD000604D45B
:10E2B0002046FCF7A2FE000602D5FCF77AFACEE76C
:10E2C00008F0DFFA000648D408208DF801000E9807
:10E2D000CDF802000DF10700FCF777FE00063CD4F4
:10E2E0000DA8FCF783FE000637D4BDF83400ADF866
:10E2F000080000208DF806002068CDF80A00684666
:10E3000005F08AF8000628D4684606F007FA0006E9
:10E3100023D40DA8FDF76EFB00061ED49DF8340033
:10E3200048B11248007830B120680F900FA804F06F
:10E3300076FB000611D4FCF78EF900060DD4684672
:10E3400005F095F8000608D4684606F01FFA0006A6
:10E3500003D4FCF78CF9000602D508F019F8ACE7F5
:10E36000FCF792F97BE7000008C007200844000092
:10E3700030B5044691B04FF00040FCF71FF9564D00
:10E38000000619D40DA8FCF719FD000631D40DA81C
:10E39000FCF744FE00062CD421460DA8FBF756FDE1
:10E3A000000626D40DA8FCF7FFFC000621D40EA819
:10E3B000FDF7EEF9000602D5286811B030BD9DF8D2
:10E3C0003800C8B10DA9FDF7D1F9000611D42146D6
:10E3D0000DA8FBF75CFD00060BD40DA99DF83800D5
:10E3E000FDF7B7F9000604D42046FCF706FE000648
:10E3F00011D5FCF7DEF9E0E70DA8FCF73CFD0006BF
:10E40000F7D421460DA8FBF742FD0006F1D40DA874
:10E41000FCF727FDE6E708F014FA000656D40420BE
:10E420008DF801000FA94C2011F05CFA00064DD4C4
:10E430009DF83C00800702D49DF8380020B968465A
:10E4400004F0EAFF000641D49DF83C009DF8381026
:10E4500000F00100401E084204D1684606F05EF953
:10E46000000633D40DA8FDF7C5FA00062ED49DF89A
:10E47000340048B11948007830B12068109010A8D5
:10E4800004F0F7FA000621D4FCF7E5F800061DD4E5
:10E490009DF83C00800702D49DF8380020B96846FA
:10E4A00004F0E5FF000611D49DF83C009DF83810FB
:10E4B00000F00100401E084204D1684606F066F9EB
:10E4C000000603D4FCF7D3F8000602D507F060FF7E
:10E4D0008FE7FCF7D9F870E708C007200844000070
:10E4E00030B5044691B04FF00040FCF767F8444D5A
:10E4F000000656D40EA8FCF761FC000626D40EA830
:10E50000FCF78CFD000621D40E980D9021460DA835
:10E51000FBF79CFC000619D40DA8FCF745FC00068F
:10E5200014D40DA8FCF7B8FC00060FD421460DA8A2
:10E53000FBF78CFC000609D40DA8FCF7A3FC000631
:10E5400004D42046FCF759FD000603D5FCF731F949
:10E5500011B030BD08F015F900064AD40DA8FDF73A
:10E5600049FA000645D49DF8340048B125480078A2
:10E5700030B120680F900FA804F0A8FA000638D434
:10E5800007208DF801000E98CDF802000DF107006C
:10E59000FCF71BFD000604D40DA8FCF727FD0006C0
:10E5A00001D52868D4E7BDF83400ADF80800002094
:10E5B0008DF806002068CDF80A00684604F02CFFAC
:10E5C000000616D4684606F0A9F8000611D4FCF738
:10E5D00042F800060DD4684604F049FF000608D44E
:10E5E000684606F0D3F8000603D4FCF740F80006AE
:10E5F00002D507F0CDFEA9E7FCF746F8A8E7000032
:10E6000008C007200844000010B5044692B04FF03F
:10E610000040FBF7D3FF000603D55548006812B051
:10E6200010BD0DA8FCF7CAFB00062ED40DA8FCF700
:10E63000F5FC000629D421460DA8FBF728FC0006AE
:10E6400023D40DA8FCF7B0FB00061ED40EA8FDF7DE
:10E650009FF8000619D49DF83800C8B10DA9FDF740
:10E6600085F8000611D421460DA8FBF710FC000622
:10E670000BD40DA99DF83800FDF76BF8000604D403
:10E680002046FCF7BAFC000611D5FCF792F8C6E765
:10E690000DA8FCF701FC0006F7D421460DA8FBF7F6
:10E6A000F6FB0006F1D40DA8FCF7ECFBE6E708F05A
:10E6B00048F8000656D403208DF801000FA94C201D
:10E6C00011F010F900064DD49DF83C00800702D4EB
:10E6D0009DF8380020B9684604F09EFE000641D43B
:10E6E0009DF83C009DF8381000F00100401E0842E3
:10E6F00004D1684606F012F8000633D40DA8FDF7E1
:10E7000079F900062ED49DF8340048B119480078F4
:10E7100030B12068109010A804F002FA000621D44D
:10E72000FBF799FF00061DD49DF83C00800702D43A
:10E730009DF8380020B9684604F099FE000611D40F
:10E740009DF83C009DF8381000F00100401E084282
:10E7500004D1684606F01AF8000603D4FBF787FFD9
:10E76000000602D507F014FE8FE7FBF78DFF56E792
:10E7700008C007200844000000B58FB04FF00040EB
:10E78000FBF71CFF000603D51B4800680FB000BD57
:10E7900007F0B7FF000626D410208DF801000DA861
:10E7A000FCF70CFB00061ED40D98CDF8020068465D
:10E7B00004F032FE000616D4684605F0AFFF0006EE
:10E7C00011D4FBF748FF00060DD4684604F04FFE55
:10E7D000000608D4684605F0D9FF000603D4FBF70D
:10E7E00046FF000604D507F0D3FDFBF7E2FFCDE7B7
:10E7F000FBF74AFFCAE7000008C00720F0B5734DD9
:10E80000070091B0288802D040F0200001E040F0DD
:10E81000100028804FF00040FBF7D0FE6C4E000641
:10E8200071D40EA8FCF7B9FA000668D469469DF8C1
:10E830003800FCF772FC000661D4BDF800006946A0
:10E84000401CADF800009DF83800FCF759FC0006AC
:10E8500055D46846FCF782F9000650D46846FBF7A9
:10E8600057FD00064BD46846FCF76EF9000646D407
:10E870006846FCF784F9000641D46846FBF723FD9F
:10E8800000063CD46846FCF770F9000637D46846A9
:10E89000FCF786F9000632D46846FBF739FD00061E
:10E8A0002DD46846FCF772F9000628D40024684687
:10E8B0000094FCF779FA00067AD46846FDF79AF8D6
:10E8C000000602D507F064FD19E0022025F0E2FB06
:10E8D000000614D438003F4F0DD09DF8000028B139
:10E8E000387818B103F00EFA000608D407F0D4FE09
:10E8F000000604D411E007F0CFFE000604D5FBF7B4
:10E9000058FF11B0F0BD53E09DF8000028B13878F1
:10E9100018B103F0F7F90006D4D40FA96A2011F05A
:10E92000ACF8000644D49DF83C0010F002008DF8CD
:10E930003C0002D0742010F02AFE8DF8004068469A
:10E94000FCF721FA0006BDD48DF800406846FCF7BC
:10E95000EAF80006B6D46846FCF7B9F80006B1D468
:10E960009DF80000022806D18DF800406846FCF7AB
:10E9700082F80006A6D402208DF8050005F016FEE8
:10E9800000069FD401A804F047FD00069AD4FBF7C7
:10E9900062FE000696D401A804F069FD000691D439
:10E9A000FBF765FE00068DD4FBF76EFE000601D571
:10E9B0003068A6E7288820F0B00028800648346038
:10E9C000046078460549086000209AE702000010BC
:10E9D00008C00720084400000CC0072010C0072012
:10E9E000FE49008808807047FC490988018070470B
:10E9F000FA49008848807047F84949880180704783
:10EA000030B58FB005460B208DF801000DA8FCF73E
:10EA1000B6F8F34C000630D4BDF83400ADF80A0067
:10EA20000DA8FCF79BF8000627D40D98CDF806003A
:10EA300028798DF80C002888ADF802006888ADF8B8
:10EA40000400684604F0E8FC000616D4684605F0A9
:10EA500065FE000611D4FBF7FEFD00060DD46846E6
:10EA600004F005FD000608D4684605F08FFE000698
:10EA700003D4FBF7FCFD000602D520680FB030BDC3
:10EA8000D8490020206008607846D74908600020F7
:10EA9000F4E72DE9F34F9BB007461C990020119035
:10EAA0000870CE493888DFF83CB308807888488001
:10EAB0003879CB4D862408B11E2804D905212C6055
:10EAC000CBF8001012E0388848F6AD611426884271
:10EAD0001DD878884FF01708B0F5B46F0DD32C60AF
:10EAE0007846C149CBF80080086002E07946BE480C
:10EAF000016086201DB0BDE8F08F05A8FCF761F825
:10EB000000067CD43888BDF81410884203D22C60EB
:10EB1000CBF80060EAE70DD105A8FCF763F8000622
:10EB2000EFD47888BDF81410884203D22C60CBF85B
:10EB30000080DBE702A8FCF777F80006E1D405A81F
:10EB4000FCF73CF90006DCD405990298814209D013
:10EB50008C20286000207946CBF80000A248016094
:10EB60008C20C7E7022005F074F90006C9D4012003
:10EB700003F094FB0006C4D44FF00040FBF71EFDE9
:10EB80000006BED46846FCF708F900067DD405A847
:10EB9000FCF714F90006F9D4059898B102A99DF87C
:10EBA0000000FCF78CFA0006F0D405A902A8FBF7D8
:10EBB000B3F80006EAD402A99DF80000FCF772FA47
:10EBC0000006E3D405A8FCF731FD0006DED4059865
:10EBD00098B102A99DF80000FCF73CFD0006D5D4D1
:10EBE00005A902A8FBF798F80006CFD402A99DF862
:10EBF0000000FCF722FD0006C8D402A900E0D9E01D
:10EC00009DF80000FCF771FA0006BFD4BDF80800BB
:10EC100002A9401CADF808009DF80000FCF758FA66
:10EC20000006B3D405A8FCF7DAF80006AED4BDF8A8
:10EC3000140098B102A99DF80000FCF7FBFB000648
:10EC4000A4D405A902A8FBF775F900069ED402A971
:10EC50009DF80000FCF7E1FB000697D405A8FCF73F
:10EC6000CFF8000692D4BDF81400A8B102A99DF80F
:10EC70000000FCF7F5FB000688D405A902A8FBF705
:10EC800059F9000687D402A900E08AE29DF8000045
:10EC9000FCF7D9FB000687D401208DF80400C0B230
:10ECA00005A9FCF7C0F8000684D40598B8B19DF812
:10ECB000041002AA9DF80000FCF748FA000685D46B
:10ECC00005A902A8FBF728F8000688D49DF80410CF
:10ECD00002AA9DF80000FCF729FA000685D49DF8E9
:10ECE000040005A9FCF7B4F8000685D40598B8B16E
:10ECF0009DF8041002AA9DF80000FCF743FA0006F4
:10ED00008FD405A902A8FBF780F8000689D49DF8E6
:10ED1000041002AA9DF80000FCF727FA000685D42B
:10ED20009DF80400401CC0B28DF804001028B6D92C
:10ED300005A8FCF7A0F8000688D4059E4FF000084F
:10ED40009EB102A99DF80000FCF7A0FA000684D449
:10ED500005A902A8FAF7E0FF00068DD402A99DF8E4
:10ED60000000FCF786FA000686D405A8FCF794F8A4
:10ED7000000687D405984FF00009B0F1000A13D0BF
:10ED800002A99DF80000FCF797FA00068CD405A9AB
:10ED900002A8FAF7C1FF000686D402A99DF8000078
:10EDA000FCF77DFA00068AD401A90B2010F09AFD29
:10EDB000000601D528689DE69DF80400012801D0D1
:10EDC000032823D105A8FBF7F9FF000686D402AA81
:10EDD00001219DF80000FCF7F1F907E0D2010010D5
:10EDE00008C007200CC0072010C00720000687D4E9
:10EDF00005A902A8FAF790FF000687D402AA01210C
:10EE00009DF80000FCF7CAF9000688D49DF80400BC
:10EE1000022803D0042801D0062873D146EA0A004C
:10EE200048EA090108436ED086EA0A0188EA090027
:10EE3000014368D000200990BAEB060179EB080085
:10EE400005D2B6EB0A0A68EB0904012004E0BAEB2C
:10EE5000060A69EB080400201A90002081468046CB
:10EE6000064601208DF80400C0B205A9FBF7DBFFC0
:10EE700000068BD405999DF8040019EB010948EBB5
:10EE8000060805A9FBF7E4FF000685D4059810B134
:10EE90000998401C09909DF80400401CC0B28DF8F0
:10EEA00004001028E0D9002610208DF80400C0B21C
:10EEB00005A9FBF7B8FF000688D4059804903043F5
:10EEC0004BD00498AAFB003204FB00200AFB060189
:10EED0005FEA58024FEA3900181851414A46434642
:10EEE00032F052F9BAEB000A049A64EB0104B9EB70
:10EEF00002091A9A68EB060832B1049A101A66EBF6
:10EF0000010604E082E056E0049A10184E41099987
:10EF10000590491E09919DF8041002AA9DF8000071
:10EF2000FCF74CF90006A4D405A902A8FAF7F4FEF0
:10EF300000069ED49DF8041002AA9DF80000FCF77C
:10EF40002DF9000695D400BF9DF80400401E10F076
:10EF5000FF008DF80400AAD158E05AEA0400F3D06B
:10EF600059EA0800F0D19DF8040005A9FBF770FFED
:10EF700000068AD405980028E6D01A9848B10920DE
:10EF800028600020CBF800007846FE490860092080
:10EF9000B0E5099800EBD070421012EB0A0044EB88
:10EFA000E271099A4FEAE27332F0EEF8BAEB000A26
:10EFB00064EB0104A8E701208DF80400C0B205A9A4
:10EFC000FBF731FF0006AED40598B8B19DF80410E8
:10EFD00002AA9DF80000FCF7F1F80006A3D405A9E9
:10EFE00002A8FAF799FE00069DD49DF8041002AA23
:10EFF0009DF80000FCF7D2F8000694D49DF80400B8
:10F00000401CC0B28DF804001028D7D901248DF817
:10F01000044000BF9DF8040005A9FCF7A7FB00060B
:10F0200087D40598B8B19DF8041002AA9DF8000095
:10F03000FCF780FB000685D405A902A8FAF76CFE50
:10F04000000696D49DF8041002AA9DF80000FCF773
:10F0500061FB00068DD49DF80400401CC0B28DF801
:10F0600004001128D6D305A8FCF7C0F80006AAD4DE
:10F07000059898B102A99DF80000FCF7CAF80006AF
:10F08000A1D405A902A8FAF747FE00069BD402A95D
:10F090009DF80000FCF7B0F8000694D405A8FCF732
:10F0A000CBF800067DD4059898B102A99DF8000020
:10F0B000FCF7D6F8000674D405A902A8FAF72CFECE
:10F0C00000066ED402A99DF80000FCF7BCF800060B
:10F0D00067D48DF8044000BF9DF8040005A9FBF734
:10F0E000B6FD00065DD40598B8B19DF8041002AADB
:10F0F0009DF80000FCF7F9F8000652D405A902A813
:10F10000FAF70AFE00064CD49DF8041002AA9DF8F6
:10F110000000FCF7DAF8000643D49DF80400401C18
:10F12000C0B28DF804000B28D6D305A8FBF746FE25
:10F13000000636D4059898B378883C21B0FBF1F0EE
:10F14000401CC1B28DF8041002AA9DF80000FCF723
:10F15000EBF8000625D405A902A8FAF7DDFD0006A4
:10F160001FD49DF8041002AA9DF80000FCF7CCF80B
:10F17000000616D4397902AA9DF80000FCF7F3F8CE
:10F1800000060ED405A902A8FAF7C6FD000608D4A9
:10F19000397902AA9DF80000FCF7D5F8000600D4E2
:10F1A00000E087E08DF804409DF8040005A9FCF715
:10F1B00089FA00067ED49DF8041002AA9DF800008A
:10F1C000FCF799FA000675D405A902A8FAF7A4FD80
:10F1D00000066FD49DF8041002AA9DF80000FCF709
:10F1E0007AFA000666D49DF80400401CC0B28DF87F
:10F1F00004000528D8D902A90120FBF78CFC0006E1
:10F2000058D405A90120FBF722FD000652D49DF831
:10F210000000012814D002280DD003280BD00428A8
:10F220000ED0882002212860CBF80010794655487E
:10F23000016088205EE405A902A8FAF710FF03E048
:10F2400005A902A8FAF7D0FE00067AD402A9012087
:10F25000FBF755FC000674D4012004F0FAFD00060B
:10F260006FD413A8FCF7C6FB00066AD446499DF884
:10F270004C004FF092060978084267D016A9032087
:10F2800004F06AFD00065CD418A9052002F06BFFAB
:10F29000000656D4052216A918A832F0D5FA88B16E
:10F2A000FBF787FA422010F072F9032025F063FB88
:10F2B000312000E01BE02E60CBF800007846314999
:10F2C00008605CE012A9002002F04DFF000638D46F
:10F2D0009DF8480080062FD507F0BEF9000604D43B
:10F2E0003846FFF78DFB000602D507F051F828E0FD
:10F2F0003888ADF828007888ADF82A0038798DF87C
:10F300002C0014A90AA803F038FCDBF80000282818
:10F310000FD028780006E8D414A8FBF790FE00066A
:10F32000E3D415A8FBF79CFE0006DED41C980470FD
:10F3300015E001201190EFE705A8FBF73FFD00065F
:10F3400002D5FBF736FA0CE4059840B907F084F9CA
:10F350000006CAD43846FFF753FB0006C5D48DF823
:10F36000044001A8FBF787FB0006BED4119868B1E2
:10F3700028212E60CBF800107946024801609220C7
:10F3800019E5000010C0072008440000FBF77CF9D5
:10F3900011E50000F8B5054646793B4C3B4A3C4B2D
:10F3A00086200EB1022E02D92060072005E02E79BA
:10F3B0000EB11E2E06D92060052010607846186018
:10F3C0008620F8BD29B16988288801F06BFD000608
:10F3D00041D400270126009769463046FBF72BFCF5
:10F3E000000638D4761CF6B20B2EF5D36846FBF730
:10F3F00036FC00062FD46846FBF753FC00062AD4DF
:10F400006846FBF707FC000625D4ADF80070684697
:10F41000FBF736FC00061ED46846FBF753FC0006DB
:10F4200019D42846FBF7C3FB000614D4A81CFBF72D
:10F43000CFFB00060FD4281DFBF7DBFB00060AD428
:10F44000012007F0EFFB000605D44FF00040FBF76A
:10F45000B5F8000601D52068F8BD02208DF800003F
:10F460006846FBF760FB000607D40A4901200870D4
:10F47000681DFBF706FE000602D5FBF79AF9F8BDFA
:10F48000FBF702F9F8BD000008C007200CC00720F8
:10F4900010C00720000000101CB54FF00040FBF723
:10F4A0008DF8000602D5174800681CBD07F00AFD5C
:10F4B00000061ED400248DF800406846FBF733FB9D
:10F4C000000616D48DF8044001A8FBF7DAFD00060B
:10F4D0000FD46846FBF7FBFA00060AD49DF800003B
:10F4E00002280BD18DF800406846FBF7C4FA0006ED
:10F4F00004D506F04DFFFBF75CF91CBDFBF7C4F823
:10F500001CBD000008C007202DE9F04F054600791A
:10F510009A4C9B4E9B4F93B04FF086084FF0050BD3
:10F5200008B11E2804D9C4F80080C6F800B017E05E
:10F53000288848F6AD614FF01409884205D900BF0C
:10F54000C4F80080C6F800900AE068884FF0170AF7
:10F55000B0F5B46F0AD300BFC4F80080C6F800A0AD
:10F5600078463860862013B0BDE8F08F02A8FBF71C
:10F5700028FB000615D42888BDF808108842DFD380
:10F5800009D102A8FBF72EFB00060AD46888BDF853
:10F5900008108842E0D34FF00040FBF70FF8000658
:10F5A00001D52068DFE76846FBF775FD00067CD4CF
:10F5B00002A8FBF739FB000677D4029898B103A99B
:10F5C0009DF80000FBF7EBFE00066ED402A903A82D
:10F5D000FAF7A2FB000668D403A99DF80000FBF728
:10F5E000D1FE000661D403A99DF80000FBF7EDFEF3
:10F5F00000065AD4BDF80C0003A9401CADF80C005D
:10F600009DF80000FBF7D4FE00064ED40120804692
:10F6100002A9FBF71CFB000647D40298A8B103AA75
:10F6200041469DF80000FBF7E9FE00063DD402A923
:10F6300003A8FAF771FB000637D403AA41469DF8E8
:10F640000000FBF7CBFE00062FD408F10100C0B28A
:10F6500080460A28DCD903A90120FBF75CFA0006E2
:10F6600023D402A90120FBF7F2FA00061DD49DF86D
:10F6700000004FF0880801280BD0022803D0022098
:10F68000C4F800801DE002A903A8FAF7E8FC04E032
:10F690000BE002A903A8FAF7A7FC000605D403A90A
:10F6A0000120FBF72CFA000602D5FBF782F85AE797
:10F6B0009DF80000012809D002280AD00920C4F8CA
:10F6C000008030607846386088204CE78DF815B0AF
:10F6D00002E006208DF8150002A8FBF750FA00069C
:10F6E00042D4BDF80800401CADF81E0002A8FBF78C
:10F6F00035FA000638D40298401CCDF81A0002A84A
:10F70000FBF73AFB00062FD4029808901E490DF132
:10F71000250032F0C5F828798DF824002888ADF846
:10F7200016006888ADF8180004F040FF00061BD4EE
:10F7300005A803F071FE000616D405A804F0EEFF3C
:10F74000000611D4FAF787FF00060DD405A803F0D0
:10F750008EFE000608D405A805F018F8000603D4AC
:10F76000FAF785FF000602D506F012FE9DE706496E
:10F7700000200870FAF788FFF5E6000008C00720AF
:10F780000CC0072010C00720D0C7072030B50446A2
:10F7900000785C4D91B008B10A280AD986205A49F0
:10F7A000286004200860784658490860862011B017
:10F7B00030BDA0680D90211D0DA8FAF710FD0006C0
:10F7C00005D44FF00040FAF7F9FE000601D528688D
:10F7D000EDE70EA8FBF74DFA000650D40DA90EA8D0
:10F7E000FAF734FB00064AD40EA8FBF738FA0006F5
:10F7F00045D40EA8FBF74EFA000640D4BDF83800F9
:10F80000401CADF838000EA8FBF73AFA000636D4D3
:10F8100020780EA9FBF71BFA000630D40DA90EA81C
:10F82000FAF714FB00062AD420780EA9FBF703FA96
:10F83000000624D40EA8FBF7F7F900061FD40DA983
:10F840000EA8FAF703FB000619D40EA8FBF7E2F99D
:10F85000000614D42046FBF746FA00060FD4201DFC
:10F86000FBF75EFA00060AD404F10800FBF769FA18
:10F87000000604D40DA8FBF775FA000602D5FAF7C6
:10F8800098FF94E707F028F9000635D40FA8FBF796
:10F8900054F9000630D49DF83C00022803D107F04B
:10F8A00025FB000628D49DF83C00012827D109201B
:10F8B0008DF8010020788DF802000D98CDF8030036
:10F8C000684603F0A9FD000616D4684604F026FF3A
:10F8D000000611D4FAF7BFFE00060DD4684603F007
:10F8E000C6FD000608D4684604F050FF000603D4A5
:10F8F000FAF7BDFE000602D506F04AFDBFE7FAF7AB
:10F90000C3FE54E708C007200CC0072010C0072022
:10F9100030B504460078544D8FB008B10A280AD992
:10F9200086205249286004200860784650490860C3
:10F9300086200FB030BDA0680D90211D0DA8FAF7EC
:10F940004EFC000605D44FF00040FAF737FE0006E3
:10F9500001D52868EDE70EA8FBF78BF9000650D417
:10F960000DA90EA8FAF793FA00064AD40EA8FBF7E1
:10F9700076F9000645D40EA8FBF78CF9000640D4B2
:10F98000BDF83800401CADF838000EA8FBF778F938
:10F99000000636D420780EA9FBF759F9000630D4BA
:10F9A0000DA90EA8FAF773FA00062AD420780EA93A
:10F9B000FBF741F9000624D40EA8FBF735F9000641
:10F9C0001FD40DA90EA8FAF762FA000619D40EA8E2
:10F9D000FBF720F9000614D42046FBF784F9000653
:10F9E0000FD4201DFBF79CF900060AD404F108008F
:10F9F000FBF7A7F9000604D40DA8FBF7B3F900063E
:10FA000002D5FAF7D6FE94E707F086F8000624D46C
:10FA10000A208DF8010020788DF802000D98CDF8AD
:10FA20000300684603F0F8FC000616D4684604F0AC
:10FA300075FE000611D4FAF70EFE00060DD46846D6
:10FA400003F015FD000608D4684604F09FFE00068A
:10FA500003D4FAF70CFE000602D506F099FCD0E7B5
:10FA6000FAF712FE65E7000008C007200CC0072067
:10FA700010C0072030B504460078564D8FB008B14D
:10FA80000A280AD98620544928600420086078464C
:10FA90005249086086200FB030BDA0680D90211D2E
:10FAA0000DA8FAF79CFB000605D44FF00040FAF7CA
:10FAB00085FD000601D52868EDE70EA8FBF7FBF8E9
:10FAC000000650D40DA90EA8FAF7C0F900064AD4D2
:10FAD0000EA8FBF7E6F8000645D40EA8FBF7FCF8E5
:10FAE000000640D4BDF83800401CADF838000EA820
:10FAF000FBF7E8F8000636D420780EA9FBF7A7F844
:10FB0000000630D40DA90EA8FAF7C1F900062AD4D0
:10FB100020780EA9FBF78FF8000624D40EA8FBF777
:10FB200083F800061FD40DA90EA8FAF7B0F9000655
:10FB300019D40EA8FBF76EF8000614D42046FBF784
:10FB4000D2F800060FD4201DFBF7EAF800060AD40D
:10FB500004F10800FBF7F5F8000604D40DA8FBF744
:10FB600001F9000602D5FAF724FE94E706F0F4FF47
:10FB7000000629D411208DF801000EA8FBF779F8B2
:10FB8000000621D40E98CDF802000D98CDF806009D
:10FB9000684603F041FC000616D4684604F0BEFD3A
:10FBA000000611D4FAF757FD00060DD4684603F09D
:10FBB0005EFC000608D4684604F0E8FD000603D4A5
:10FBC000FAF755FD000602D506F0E2FBCBE7FAF79F
:10FBD0005BFD60E708C007200CC0072010C00720AD
:10FBE0002DE9F04F85B06846FAF74FFFF84F000651
:10FBF0000ED49DF80000DFF8DC93DFF8DCA30024CE
:10FC0000012809D001A90120FBF759FA000607D500
:10FC1000386805B0BDE8F08F3C60C9F800401CE1D1
:10FC20008DF800400DF104029DF800009DF80410CD
:10FC3000135C401CC0B219448DF804108DF800000C
:10FC40000528F1D31046FAF78FF900067DD4A046B7
:10FC50000494ADF80C400124E04EDFF884B325464F
:10FC60003078022805D000EB40000BEBC000406864
:10FC70008047E8B2054601A9FBF714FA0006E5D46F
:10FC800001A92846FBF7D9FC0006DFD403A92846C2
:10FC9000FBF71EFA0006D9D403A92846FBF730FA71
:10FCA0000006D3D403A92846FBF7B7FB00064CD4C3
:10FCB00003A92846FBF7C7FB000646D48DF8004091
:10FCC0009DF8001001AA2846FBF730FA00063CD444
:10FCD0009DF8001004AA2846FBF747FA000634D422
:10FCE0009DF8001001AA2846FBF758FA00062CD40C
:10FCF0009DF80000401CC0B28DF800001028DFD92C
:10FD000001A92846FBF7B5FA00061ED401A928462A
:10FD1000FBF7C5FA000618D48DF800409DF80010D6
:10FD200001AA2846FBF7D1FA00060ED49DF8000080
:10FD3000401CC0B28DF800000A28EFD98DF80040B1
:10FD40009DF8001001AA284600E073E0FBF7DCFAFA
:10FD500000066FD49DF80000401CC0B28DF8000072
:10FD60001828EDD98DF800409DF8001001AA28460A
:10FD7000FBF7E9FA00065DD49DF80000401CC0B214
:10FD80008DF800001E28EFD98DF800409DF8001076
:10FD900001AA2846FBF79FFC00064BD49DF8000003
:10FDA000401CC0B28DF800000528EFD98DF8004046
:10FDB0009DF8001001AA2846FBF7ACFC000639D4D8
:10FDC0009DF80000401CC0B28DF800001028EFD94B
:10FDD00001A92846FBF710FA00062BD401A92846F2
:10FDE000FBF731FA000625D46D1CEDB2042D7FF629
:10FDF00037AF25463078022805D000EB40010BEBE9
:10FE0000C10040688047E0B2044601A9FBF7BAFA96
:10FE100000060FD403A92046FBF7CAFA000609D44E
:10FE200028468DF80050C1B201AA2046FBF7D6FA49
:10FE3000000602D5FAF7BDFCEBE69DF80000401C79
:10FE4000C0B28DF800000A28EDD9641CE4B2022C7F
:10FE5000D0D9C7F80080C9F8008079460020CAF8D8
:10FE60000010D6E6F0B504460179594D594E5A4F67
:10FE70008FB0862009B11E2902D9286005200DE027
:10FE8000218848F6AD62914202D92860142005E02D
:10FE90006188B1F5B46F07D32860172030607846C9
:10FEA000386086200FB0F0BD0EA9022004F0B3F92F
:10FEB000000615D4BDF83800A0B103F0B1F9000672
:10FEC0000ED446480678012E04D0012006F0AAFE82
:10FED000000605D44FF01040FAF770FB000609D574
:10FEE0002868DFE7912028608A20306078463860F3
:10FEF0009120D7E7FFF774FE000620D401F0EAF85E
:10FF000000061CD42046FBF7B4FA000617D4A01C48
:10FF1000FBF7BEFA000612D4201DFBF7CAFA000652
:10FF20000DD401208DF800006846FAF7A4FD000604
:10FF300005D469462B200FF0D5FC000602D5FAF750
:10FF400038FCAFE79DF80000C00701D16079E8B345
:10FF5000012E49D06846FAF701FE000633D4684600
:10FF6000FAF7C4F900062ED46846FAF7EDFD00064C
:10FF700029D406F089F9000625D41A490220087010
:10FF800012208DF805006946042003F0E5FE000606
:10FF900019D4BDF80000401CADF8060020798DF89A
:10FFA00010002088ADF808006088ADF80A006846A7
:10FFB000FAF7D4FD000606D40098039001A803F0D8
:10FFC00056FA000610D506F0E3F9B8E70CE0000099
:10FFD00008C007200CC0072010C0072076020010C0
:10FFE000A8C1072000000010FAF74EFB5AE70000F6
:10FFF000F8B505460379384C3849394A86200BB1A3
:020000040001F9
:100000001E2B02D9206005200EE02B8848F6AD6734
:100010001426BB4202D920600E6006E06B88B3F55F
:10002000B46F06D3206017200860784610608620E1
:10003000F8BD2C490120FBF742F8000640D42A49BC
:100040000220FBF73CF800063AD42846FAF7AFFD49
:10005000000635D4A81CFAF7BBFD000630D4281DD5
:10006000FAF7C7FD00062BD4002568460095FBF77C
:10007000B1FA000624D468460095FBF7BCFA0006E6
:100080001ED48DF800606846FBF757FA000617D4B7
:100090000120ADF800006846FBF776FA00060FD4A1
:1000A00069461C200FF01EFC000609D49DF80000D4
:1000B00040B1ADF800506846FAF757FD000601D58B
:1000C0002068F8BD032009498DF80000022008705F
:1000D0006846FAF728FDF8BD08C007200CC00720C5
:1000E00010C00720140200101902001000000010B8
:1000F0002DE9FC414FF00040FAF760FA4C4C000645
:100100007ED46846F9F73CFF00062AD401273E4614
:10011000F0B205466946FAF7F2FC000621D46D1CE0
:10012000EEB20B2EF4D3002568460095FAF70CFDCD
:10013000000616D4ADF800506846FAF716FD000622
:100140000FD468460095FAF721FD000609D4ADF8F2
:1001500000700220C0B206466946FBF7FFF90006B0
:1001600005D506F015F9FAF724FBBDE8FC81761CED
:10017000F0B21B28EED92F4F04226946384620F0F2
:1001800053F900064ED42C4E0098B04227D00422DA
:100190006946381D009520F052F9000642D42548E2
:1001A00004226946083020F04AF900063AD4214872
:1001B000042269460C3020F042F9000632D41D4872
:1001C00004226946103020F03AF900062AD40422AD
:1001D00069463846009620F032F9000622D41548C8
:1001E000042269461430009520F029F9000619D43C
:1001F000104804226946183020F021F9000600E07A
:1002000010E00FD40B48042269461C3020F017F987
:10021000000607D4074804226946203020F00FF971
:10022000000601D52068A0E7FAF72EFA9DE7000046
:1002300008C0072004000020CEFAADDEFEB56846F7
:10024000F9F792FE284C000640D400270125ADF8AE
:1002500008702E46F0B206466946FAF723FF0006FC
:1002600034D402A93046FAF733FF00062ED402A98F
:100270003046FAF745FF000628D402A93046FBF7BE
:10028000CCF8000622D402A93046FBF7DCF80006C1
:100290001CD469463046FAF7ECFF000616D46946CE
:1002A0003046FAF7FCFF000610D4761CF6B2042E96
:1002B000D0D9E8B205466946FBF764F8000605D4D4
:1002C00002A92846FBF774F8000601D52068FEBD98
:1002D0006D1CEDB2022DECD904482760076078460A
:1002E000034908600020FEBD08C007200CC007209D
:1002F00010C007207CB506466846F9F735FE0D4D5F
:10030000000607D401246A4631462046FAF7FCFF6E
:10031000000601D528687CBD641CE4B2052CF2D32C
:1003200005490020286008607846044908600020DC
:100330007CBD000008C007200CC0072010C00720AB
:100340007CB506466846F9F70FFE0D4D000607D44A
:1003500001246A4631462046FAF7F5FF000601D52A
:1003600028687CBD641CE4B2052CF2D3054900204A
:100370002860086078460449086000207CBD0000C1
:1003800008C007200CC0072010C00720FEB5074694
:100390006846F9F7E9FD144D000617D4002601243C
:1003A00002966A4639462046FAF7C0FE00060DD48A
:1003B00002AA39462046FAF7D8FE000606D46A4655
:1003C00039462046FAF7EAFE000601D52868FEBD48
:1003D000641CE4B2052CE4D304482E600660784621
:1003E000034908600020FEBD08C007200CC007209C
:1003F00010C007202DE9FC4107466846F9F7B4FD17
:10040000144E000615D401252C46E0B204466A4677
:100410003946FAF75AFF00060BD4641CE4B2052CE7
:10042000F3D3E8B204466A463946FAF7D7FF000626
:1004300002D53068BDE8FC81641CE5B2032DF0D321
:1004400005490020306008607846044908600020B3
:10045000F0E7000008C007200CC0072010C00720EC
:100460002DE9F04F97B080464FF000098A4681F899
:100470000090052001F012FFFC4C00067ED4FF2006
:1004800003F0E7FC0006F9D415A8FBF7B3FA000661
:10049000F4D46946002003F0A2FB0006EED4BDF8B8
:1004A00000009027F24DF34E192802D30120276057
:1004B000E1E06946022003F0AEFE0006DED4BDF89E
:1004C000000090B1EC480DF12C0B007800287CD096
:1004D0006946012003F083FB0006CFD4BDF800007D
:1004E000402805D303202760C5E00C202760C2E028
:1004F00014A9002001F037FE0006BFD49DF850007B
:10050000010902D004202760B5E001070BD54007A0
:1005100009D4872020607846C5F800903060872095
:1005200017B0BDE8F08F03A9052001F01CFE0006FE
:10053000A4D46946032003F00FFC00069ED4206873
:10054000052805D0052203A9684631F07DF9D0B110
:100550009DF8500000077DD56946002003F0FCFBA4
:1005600000068BD403A90B2001F0FDFD000685D405
:100570000C2203A9684631F067F900E08EE028B14B
:100580000520276077E00720276074E003A90C208E
:1005900001F0E9FD000691D4062208F1060103A846
:1005A00031F052F910B10620276064E003A9112050
:1005B00001F0D9FD000671D40622414603A831F0AE
:1005C00043F918B10820276055E0D4E069460E20B1
:1005D00001F0C9FD000661D403A800F0CCFC0006C0
:1005E0005CD4BDF80000BDF80C10884207D9632028
:1005F0000EF0CDFF000651D4092027603BE003A98F
:10060000F4F7C9F99DF80C00694600F5FA60ADF8F9
:100610002C009DF80D008DF82E009DF80E008DF831
:100620002F000F2001F09FFD000637D4BDF8001009
:100630003C20B1FBF0F28DF83020B1FBF0F200FB72
:1006400012108DF831008DF8329003A9102001F0BE
:100650008AFD00E023E0000620D46946042003F070
:100660007BFB00061AD4BDF80000BDF80C108842D0
:1006700006D00A20276028607846306090204FE737
:100680006946062001F06FFD000672D4BDF80C002B
:10069000BDF80010401C8142EBD110E069E001F090
:1006A00016FE00287FF46FAF0BF104001AF025F955
:1006B00000065ED40BA81AF051F9000659D402F0D6
:1006C000EFFD000655D40BF10701002003F044FBB9
:1006D00000064ED4D8F80610CDF83F10B8F80A003E
:1006E000ADF84300D8F80010CDF84510B8F8040074
:1006F000ADF8490013A9042003F02EFB000638D4FE
:10070000D8F806100791B8F80A00ADF82000D8F81C
:100710000010CDF82210B8F80400ADF82600D8F883
:100720000C000A9006A90BA8F4F7D0F9BDF84C000C
:10073000ADF81A0006A8FAF73AFA000619D49DF89F
:1007400030109DF83100C1EB011100EB8100ADF8D4
:1007500000006846FAF73CFA00060AD44748FAF760
:1007600048FA000605D44FF00040F9F727FF0006CD
:1007700004D52068D4E60BF1040097E706F098FA58
:1007800000066ED406A806F0A8FA000669D49DF803
:100790005000000707D43848007820B10BA801F0BA
:1007A000A4FD00065DD4344F4FF001088AF80080A4
:1007B0003878D8B102F01AF8000652D40121304836
:1007C00006F0B9FA00060AD5F3F740FD01F09AFAEF
:1007D000F3F751FD05F0DCFDF9F7EBFFC9E702F097
:1007E00041F800063DD420680028E7D0112003F02E
:1007F000C8FC000635D406A9002003F0D2FC000690
:100800002FD4387858B107A9052001F0ACFC0006B8
:1008100027D406A9012003F0C4FC000621D412202D
:1008200003F0AFFC00061CD49DF8540050B368469A
:10083000FAF794F9000614D46846F9F757FD000654
:100840000FD46846FAF780F900060AD4FBF7EEF8F1
:10085000000606D44F468AF80090F9F715FF000607
:100860005AD505F095FDF9F7A4FF59E608C0072011
:100870000CC0072010C00720084400006D020010C3
:100880006CC50720FFE747468DF800806846FBF7F8
:10089000CAF80006E5D4ADF81090CDF80C908DF8AC
:1008A0001290B84638468DF80070C0B203A9FAF726
:1008B00026F90006D5D49DF80000401CC0B28DF882
:1008C00000000A28F1D94F4603A8CDF80C90FAF79A
:1008D0003BF90006C5D403A80397FAF757F90006B9
:1008E000BFD4ADF80C7003A8FAF73FF90006B8D4EE
:1008F0004046ADF80C808DF80080C0B203A9FAF72D
:100900002DFE0006ADD49DF80000401CC0B28DF84D
:1009100000001B28F1D999E7276078462F603060E6
:100920000020FDE52DE9F04796B0002180460170DA
:10093000052001F0B3FCC04C00067DD4FF2003F07D
:1009400088FA0006F9D415A8FAF79FF80006F4D43F
:100950009DF85400B94EBA4D48B1912020609C20BA
:10096000286078463060912016B0BDE8F08769466F
:10097000012003F034F90006DFD4BDF80000902711
:10098000402802D30320276027E06946022003F0B5
:1009900042FC0006D1D4BDF80000E0B101F097FCA4
:1009A0000006CAD428684FF002094FF0920A2328A3
:1009B00009D00FA9002001F0D6FB0006BDD49DF898
:1009C0003C0000090BD0C4F800A07846C5F80090A0
:1009D00030609220C8E70C202760286061E003A9FE
:1009E000052001F0C0FB0006A7D46946032003F0F0
:1009F000B3F90006A1D420684FF0070A28B90522F0
:100A0000694603A830F020FF98B39DF83C0000072A
:100A10007DD56946002003F09FF900068DD403A917
:100A20000B2001F0A0FB000687D40C2203A9684626
:100A300030F00AFF20B100E0A6E005202760CCE7F7
:100A400069460E2001F08FFB000695D403A800F044
:100A500092FA000690D4BDF80000BDF80C10884250
:100A600008D063200EF093FD000685D4092027608E
:100A7000B3E713E06946042003F06EF9000689D459
:100A800003A9102001F06FFB00067DD4BDF8000023
:100A9000BDF80C104FF00A0A884206D02760C5F84E
:100AA00000A07846306090205EE76946062001F09D
:100AB0005AFB000668D4BDF80C00BDF80010401CBD
:100AC0008142EBD103A90C2001F04DFB00065BD461
:100AD0006946012003F040F9000655D40622694614
:100AE00003A830F0B1FE10B10620276075E703A916
:100AF000112001F038FB000646D46946022003F0BD
:100B00002BF9000640D4062203A9684600E005E060
:100B100030F09AFE30B1082027605EE701F0D7FB85
:100B20000028BBD106AD281D19F0E7FE00067BD4D6
:100B300006A819F013FF000676D4E91D002003F083
:100B40000BF9000670D40DF12B01012003F004F91C
:100B5000000669D40DF13101022003F0FDF8000612
:100B600062D40EA9042003F0F7F800065CD4BDF8A7
:100B70003800ADF8420010A906A8F3F7A7FF11A9A5
:100B8000052001F0F0FA00E04EE000064CD44FF0F2
:100B90000040F9F713FD000646D406F0B0F8000651
:100BA00039D49DF83C00000704D406A801F09DFB51
:100BB000000630D4012188F8001001F017FE00066D
:100BC00029D4204D01211F4806F0B5F800060AD5AA
:100BD000F3F73CFB01F096F800061CD4F3F74BFB4F
:100BE0002078000617D401F03DFE000613D495F8D6
:100BF00000010028E6D1112003F0C3FA00060AD450
:100C000010A9012003F0CDFA000604D4122003F04D
:100C1000B8FA000604D505F0BBFBF9F7CAFDA3E658
:100C2000F9F732FD000601D520689DE688F80090AE
:100C3000012005F0F7FF97E608C0072010C0072045
:100C40000CC007206CC507202DE9F0438BB007A925
:100C5000012019F0DFF8594C000645D4684601F030
:100C6000EAF9000640D408A9032003F075F8544DB2
:100C7000DFF85081000616D40027052208A903A832
:100C800030F0E2FD80B142200EF081FC00062BD452
:100C9000922020603120794628609220C8F8001008
:100CA0000BB0BDE8F08301279DF811004FF000065E
:100CB00041074FF0870903D4C4F800902E606DE01F
:100CC000400654D506A8F9F7F1FE000674D49DF845
:100CD00018000E2801D0002FEED060200EF057FC37
:100CE000000602D505F054FB66E001F0F0FA0006BC
:100CF00062D4684600F03FF900065DD40DF10200B1
:100D000000F01DF9000657D41E208DF80400684637
:100D100001F056FB00064FD48DF800606846F9F7E5
:100D2000AAFE000648D4684601F003F9000643D441
:100D3000BDF80000401E80B201F025FD00063BD446
:100D4000214D0121204805F0F6FF000606D5F3F7F6
:100D50007DFA00F0D7FFF3F78EFA2DE001F082FD67
:100D6000000629D495F800010028EAD11BE0079875
:100D7000C00707D08DF800606846F9F77CFE0006D2
:100D80001AD410E06846F9F780FE000614D49DF8E6
:100D9000000040B10420C4F8009028607946872004
:100DA000C8F800107CE733200EF0F1FB000603D4F6
:100DB00001F079FB000695D4206871E708C0072090
:100DC0000CC0072010C007206CC5072038B54FF0B5
:100DD0000040F9F7F3FB104D000617D400248DF8FE
:100DE00000406846F9F7CFFF000606D48DF80040B2
:100DF0006846F9F798FE000602D5F9F7DAFC38BD27
:100E000068460094F9F7D0FF000601D5286838BD80
:100E1000F9F73AFC38BD000008C007201CB54FF0B8
:100E20000040F9F7CBFB000602D51D4800681CBD49
:100E300001A8FAF730F900062CD46846F9F78EFEBF
:100E4000000627D46846F9F751FA000622D468460E
:100E5000F9F77AFE00061DD46846F9F790FE000601
:100E600018D46846F9F71BFA000613D46846F9F758
:100E70007CFE00060ED400248DF8044001A8FAF789
:100E800000F9000606D48DF800406846F9F74BFEDD
:100E9000000602D5F9F78DFC1CBDF9F7F5FB1CBD6A
:100EA00008C007202DE9FC5F9B4D9C4E9C4C894659
:100EB00007004FF086084FF0140A03D048F6AD60E3
:100EC000874204D9C4F80080C5F800A008E04FF0BC
:100ED000170BB9F5B46F08D3C4F80080C5F800B09B
:100EE000784630608620BDE8FC9F01A8FAF7CAFA70
:100EF00000060BD4BDF804003F1A4FF4B46047431A
:100F0000E0D46846FAF7CEFA000601D52068EAE791
:100F1000BDF80010A9EB0100C019DDD40021B0F527
:100F2000B46F06DB8A2020607846296030608A2012
:100F3000D9E721607846296030600020D3E738B5D2
:100F40000446684619F0D9FC0106754801D50068C9
:100F500038BD9DF800209DF80110C2EB021201EB94
:100F600082012180002101606B48016078466B4955
:100F70000860002038BD38B50446684619F0EEFC1C
:100F8000000602D56648006838BD21466846F3F77A
:100F90009DFD38BD7CB50025ADF800506846FFF7D3
:100FA000CEFF5F4C000604D401A8FFF7E4FF000663
:100FB00001D520687CBDBDF80010BDF80400FFF726
:100FC00071FF5549554A38B191202060882008604A
:100FD0007846106091207CBD256078460D601060D9
:100FE00000207CBD2DE9FE43DFF8388181464A4E62
:100FF00098F80000494F4A4C002510B188F800507D
:1010000062E069463D200EF038FD000651D49DF89F
:101010000000E8B3012188F8001001A8FFF78FFF56
:10102000000646D402A8FFF7A6FF000641D4BDF88B
:101030000800BDF80410C0EB001000EB400001EB0D
:10104000401801A8FAF709FC000632D402A8FAF702
:10105000F3FB00062DD4BDF80800BDF80410C0EB6A
:10106000001000EB400001EB40109DF80010C1EBB8
:10107000011100EB8101414526D8B9F1000F1BD0C9
:1010800062200EF084FA000613D46946532000E073
:101090001AE00EF027FC00060BD49DF8000010F0BB
:1010A00002008DF8000007D0012005F0BBFD00060E
:1010B00002D52068BDE8FE838720206005203060CF
:1010C000784638608720F5E72560784635603860D7
:1010D0000020EFE71CB56846FFF731FF104C000613
:1010E0000ED401A8FFF747FF000609D401A8FAF7BC
:1010F00099FB000604D46846FAF7A5FB000601D563
:1011000020681CBD0449002020600860784603491F
:10111000086000201CBD00000CC0072010C0072084
:1011200008C00720D601001010B5044690B04FF05B
:101130000040F9F743FA000603D53648006810B0BE
:1011400010BD201DFAF78FFA000617D404F108002D
:10115000FAF79AFA000611D4207A0EA9FAF7B2FA31
:1011600000060BD4211D0EA8F8F770FE000605D46A
:10117000207A0EA9FAF799FA000602D5F9F719FBB9
:10118000DDE70DA94B200EF0ADFB00063CD49DF829
:101190003400C00703D005F0FFFC000634D4132050
:1011A0008DF80100207A8DF802006068CDF8030008
:1011B0009DF83400800704D5684602F02DF900063A
:1011C00022D49DF83400C00704D0684603F0A6FA84
:1011D000000619D4F9F73FFA000615D49DF834003B
:1011E000800704D5684602F042F900060CD49DF849
:1011F0003400C00704D0684603F0C8FA000603D4E0
:10120000F9F735FA000602D505F0C2F8B6E7F9F7A6
:101210003BFA94E708C0072010B5044690B04FF0A1
:101220000040F9F7CBF9000603D53648006810B046
:1012300010BD201DFAF717FA000617D404F10800B4
:10124000FAF722FA000611D4207A0EA9FAF73AFA30
:1012500000060BD4211D0EA8F8F719FE000605D4D0
:10126000207A0EA9FAF721FA000602D5F9F7A1FAB9
:10127000DDE70DA94B200EF035FB00063CD49DF8B0
:101280003400C00703D005F0A7FC000634D41420B6
:101290008DF80100207A8DF802006068CDF8030017
:1012A0009DF83400800704D5684602F0B5F80006C2
:1012B00022D49DF83400C00704D0684603F02EFA0B
:1012C000000619D4F9F7C7F9000615D49DF83400C3
:1012D000800704D5684602F0CAF800060CD49DF8D1
:1012E0003400C00704D0684603F050FA000603D467
:1012F000F9F7BDF9000602D505F04AF8B6E7F9F7A7
:10130000C3F994E708C0072070B592B000260446E0
:101310008DF840604079B74DA0B110A8F9F7CDFD28
:10132000000674D49DF8400008B110280AD9862020
:10133000B1492860032008607846B04908608620DB
:1013400012B070BD4FF00040F9F738F90006E8D44C
:101350006079002875D06846F9F730FD00066CD436
:10136000A07921460028684652D0F8F790FD000683
:1013700063D46846F9F718FD00065ED469469DF807
:101380004000F9F750FD000657D4A0792146002807
:10139000684640D0F8F77BFD00064ED469469DF8BC
:1013A0004000F9F734FD000647D410A8F9F7F2FD24
:1013B000000642D42046F9F7DCFD00063DD4207932
:1013C0006946FAF7D3F900067FD421466846F8F754
:1013D0003DFD000679D420796946FAF7BAF900068E
:1013E00073D4A0790028684618D0F9F7FFFE0006EC
:1013F0006BD421466846F8F729FD000665D4684697
:10140000F9F7EBFE000660D405F0DBF973E0BFE00E
:10141000F8F71CFDABE7F8F719FDBDE7F9F70CFF8E
:10142000000652D421466846F8F710FD00064CD459
:101430006846F9F7F7FEE5E703E046E004F0A8FFA9
:1014400043E00FA8F9F7BAFC00063ED40FA8F9F75D
:10145000E5FD000639D40F980090A07921460028B8
:10146000684635D0F8F713FD00062ED46846F9F724
:101470009BFC000629D42046F9F7BFFD000624D4C2
:10148000A0790028684626D0F9F7F5FC00061CD4A0
:1014900021466846F8F7DAFC000616D46846F9F7E4
:1014A000E0FC000611D420796946FAF75FF90006DE
:1014B0000BD421466846F8F7C9FC000605D420790C
:1014C0006946FAF746F9000613D5F9F772F937E7D6
:1014D000F8F7BCFCC8E7F9F7DFFC0006F5D42146B5
:1014E0006846F8F7B3FC0006EFD46846F9F7CAFC83
:1014F000D7E705F086F90006A0D4A079A8B10820A6
:101500008DF8050020798DF80A00617901A871B184
:10151000CDF80660C01DF9F714FD00068ED46846AC
:10152000F9F720FD000689D40EE00720E8E70F99BF
:10153000CDF80610C01DF9F748FD000628D468460E
:10154000F9F754FD000623D4BDF80000ADF80C00F7
:101550002068CDF80E000EA94C200EF0C3F900064D
:1015600016D49DF83800800704D501A801F054FF77
:101570000006C1D49DF83800C00704D001A803F0CC
:10158000CDF80006B8D46846FAF734FA000601D55B
:101590002868D5E69DF8000060B11948007848B188
:1015A00020681190A079002811A820D001F037FA06
:1015B0000006A1D4F9F74FF800069DD49DF8380035
:1015C000800704D501A801F052FF000694D49DF8CD
:1015D0003800C00704D001A803F0D8F800068BD467
:1015E000F9F739F8000687D4F9F74EF8A8E601F0C4
:1015F0006DFADDE708C007200CC0072010C00720E7
:101600000844000071B581B04FF00040F8F7D6FFF4
:101610007A4C00063CD403208DF800006846F9F7A8
:1016200082FA000662D419208DF800006846F9F7A6
:1016300084FF00065AD472490220087001A91920BB
:10164000F9F78CFF000623D4012005F0EBFA000621
:101650004CD402F0C2F8000648D4BDF8040002F0F1
:1016600022F8000642D420680025052807D0654EE0
:1016700002F000F9000639D42068D8B913E0F9F770
:1016800098F8000604D4012022F07FFE000601D560
:1016900020687CBD812020605B48056078465B49FE
:1016A000086081207CBD7078062803D0052801D011
:1016B0000B28DDD123F028F9000617D4012022F0F1
:1016C00064FE000612D4012005F0ACFA00060DD429
:1016D0008DF800506846F9F726FA000606D48DF812
:1016E00000506846F9F729FF000602D5F9F761F8BE
:1016F0007CBDF8F7C9FF7CBD2DE9F8430646894655
:101700004FF00040F8F75AFF3C4C00066CD496B1FD
:1017100003208DF800006846F9F705FA000622D488
:1017200019208DF800006846F9F707FF00061AD463
:101730003349022008706846F9F721FA000653D4AD
:1017400069461920F9F70AFF00064DD4012005F07B
:1017500069FA000607D403F023F9000603D403F066
:1017600031F9000603D5F9F724F8BDE8F8832068BD
:10177000254FDFF89880002505280FD1F9F719F8D3
:10178000000631D4012022F000FE00062CD4812076
:10179000206079463D60C8F80010E6E703F057F98D
:1017A000000606D420680028F8D023F0ADF8000623
:1017B00002D504F0EDFDD6E7F8F766FF000613D476
:1017C000A6B1484605F02EFA00060DD48DF800505B
:1017D0006846F9F7A8F9000606D48DF80050684667
:1017E000F9F7ABFE000601D52068BEE72560794613
:1017F0003D600020C8F80010B7E7000008C00720CF
:10180000000000109EC707200CC0072010C0072052
:101810002DE9FC412F4C90460F460026C0B3FAF745
:10182000AAF840B1F2F712FD00212BA022F0A0FE91
:10183000F2F721FD43E08DF800606846F9F70CF9F6
:101840006846F9F718F902208DF800006846F9F7A4
:1018500045F9000633D46846F9F72FF900062ED46F
:101860006846F9F719F9000629D40120ADF80400FB
:10187000054601A92846F9F771FE00061FD46D1C24
:101880001B2DF6D901F00CFDFEF732FC000616D434
:10189000C7B140460FF061F8000610D400200EF0EA
:1018A0005AFC00060BD40FF09FF820B900200FF06F
:1018B000FBFA000603D4F3F716FD000602D52068F4
:1018C000BDE8FC810B482660066078460A4908603E
:1018D0000020F5E708C007208EE8A8A1AAA020A84C
:1018E000ADA8E6A8A0ABA8A7A0E6A8A8208E8793DD
:1018F0000A0000000CC0072010C007202DE9F041AD
:101900008AB0BB48F8F73CFBBA48F8F739FB06A8A1
:10191000FAF770F8B84C000652D49DF81800052765
:10192000B64EDFF8DC82002510B307A912200DF0B7
:10193000D9FF000644D408A92E200DF0D3FF0006DD
:101940003ED405A8F9F703FE000639D49DF81C1013
:10195000C80705D09DF814000E2812D0142810D006
:101960009DF814000F2803D19DF82000800708D4AB
:101970002760794635600520C8F800100AB0BDE838
:10198000F081A04F880715D5002002F0C6F90006A7
:1019900016D46946002002F084F9000610D4BDF880
:1019A0000210022002F0A3F9000609D4BDF80200DB
:1019B000788008E00021022002F099F9000601D5A4
:1019C0002068DBE77D803D7025607946356000202A
:1019D000C8F80010D2E72DE9F04F89B04FF00005AC
:1019E000854CDFF81C82854F06008DF814504FF0AF
:1019F000050B04D0012E02D0022870D09DE0DFF844
:101A000004A24FF000096946022002F04AF920B111
:101A1000052830D093287DD152E09AF8000060B1BB
:101A2000BAF80210BDF80220481C824211D00220F0
:101A300002F05DF9000674D44AE001218AF8001032
:101A4000BAF80210BDF802204B1C9A42EFD1AAF856
:101A50000220684801A9F8F788FB000661D46448B1
:101A60000DF10901F8F781FB00065AD4BDF8021008
:101A7000AAF802102CE0012E1FD105A8F9F705F8ED
:101A800000064ED49DF81400B8B106A90120F9F75C
:101A900016FB000645D406A95648F8F766FB000673
:101AA0003FD406A90220F9F70AFB000639D406A99B
:101AB0004F48F8F75AFB000633D48AF8005034E058
:101AC000BAF80210491CAAF802103868082828D170
:101AD00009F10109B9F1640F95DB2EE0FFE705A8D4
:101AE000F8F7D3FF00061CD49DF81400E8B106A94E
:101AF0000120F9F7E4FA000613D406A93D48F8F7E7
:101B000034FB00060DD406A90220F9F7D8FA000626
:101B100007D400E005E006A93548F8F726FB0006E3
:101B20000BD5206809B0BDE8F08FC4F800B0794645
:101B30003D600520C8F80010F4E7256079463D6057
:101B40000020C8F80010EDE72DE9F04F83468DB076
:101B50008A460846F8F714FA5846F8F711FA0AA820
:101B6000F9F748FF244C000630D49DF82800DFF830
:101B70009080224F002578B3002002F0CEF80006B6
:101B800024D46946002002F08CF800061ED4BDF86B
:101B90000210022002F0ABF8000617D405AE0DF1DA
:101BA0001D0905A9022002F07CF8206810B19328D5
:101BB0000FD015E0311D5846F8F7D7FA000605D4C6
:101BC00049465046F8F7D1FA000606D520680DB010
:101BD000A9E738680828E4D002E020680528E0D1A9
:101BE000256079463D600020C8F80010EFE700004E
:101BF000F3010010EC01001008C007200CC0072002
